:020000040800F2
:1000000000A00020AD3C0108F5E50008E12C010846
:10001000F3E50008F1E50008EFE500080000000046
:10002000000000000000000000000000EDE50008F6
:10003000EBE5000800000000E9E50008FDBA000853
:10004000153D0108153D0108153D0108153D010844
:10005000153D0108153D0108153D0108153D010834
:10006000153D0108153D0108153D0108153D010824
:10007000153D0108354B00089BD60008153D0108C9
:10008000153D0108153D0108153D0108153D010804
:1000900055E60008153D0108153D0108153D01080C
:1000A0008D1B0108B91B01087D1B0108C91B010834
:1000B000AD1B01089D1B0108153D0108153D0108F8
:1000C000153D0108153D0108153D0108153D0108C4
:1000D000153D0108851D0108791D01086D1D0108E8
:1000E0000DBB0008153D0108D9E50008153D0108C4
:1000F000153D0108153D0108153D0108153D010894
:10010000000000000000000000000000153D010894
:10011000153D0108153D0108153D0108153D010873
:10012000153D0108153D0108153D0108153D010863
:10013000153D0108153D0108000000000000000009
:10014000153D0108153D0108153D0108000000009E
:10015000000000000000000000000000000000009F
:100160000000000000000000153D0108153D0108D9
:10017000153D010800000000000000000000000024
:0801800000000000153D01081C
:100188002DE9F04F2DED028B6F4E704B3360AFB001
:100198000023736010F034FF18B910F055FF09F010
:1001A8008BFC09F029FD6A4B6A4C1A7842F001026F
:1001B8001A70694A4FF47001C2F888100022099237
:1001C8000A92226842F4803222600493236803F47E
:1001D80000330A93099B013309930A9B1BB9099BB6
:1001E800B3F5A04FF2D1236813F4003318BF0123ED
:1001F8000A930A9B012B70D0574F584BFB60636AD8
:10020800B360636ADFF884A1DFF88481DFF8849142
:1002180043F080736362636943F4FC032EAD63614A
:1002280003238DF86A3041F6FF7325F8503D4FF0EF
:100238009040294604F070FD4FF6FF73504629465A
:10024800ADF8683004F068FD4548294604F064FDBF
:100258004448294604F060FD4348294604F05CFD03
:100268002946424804F058FD284607F0BBFF1A9B70
:100278003F4AB3FBF2F33F4A3F4913603F4B00222A
:100288001A603F4B5960F02187F823109A603D4F60
:1002980007221A60BB68C8F8003099E80F0085E8A3
:1002A8000F0063691A9843F480236361636943F418
:1002B800802363614FF0200B1023CAF818301BA964
:1002C800CAF818B004F028FD1DA91C9804F024FDF4
:1002D800D8F80030190729D464E02B4B12221A6091
:1002E8006368636063686360636843F48063636042
:1002F800636823F47C136360636843F4E813636002
:10030800236843F0807323602268124B9201FBD567
:100318005A6822F003025A605A6842F002025A6090
:10032800636803F00C03082BFAD165E797F892315C
:10033800012B37D8044B97F893219B6813F080530F
:1003480000F0A7842EE000BF780100203B9300084E
:10035800C02F00200010024000ED00E00005FA0563
:1003680000080048000C004800100048001400482D
:1003780040420F00541F00203F190100901F002029
:1003880010E000E050120020002002400004004865
:10039800582E0020F0800108B54B002283F89321E5
:1003A80009F0E4FD64200BF02EFAC822B1480021C0
:1003B80015F0D7FCE369B04A43F00303E361A3698E
:1003C80043F4A123A361636943F4C023636102F189
:1003D800B00C937B506892F80FE003F00701DB083C
:1003E80000EB83038900186A4FF00F0A0EFA01FE2A
:1003F8000AFA01F120EA01011962196A10324EEA7B
:10040800010162451962E4D10023DFF894A20AF1E0
:100418000C020021995401330B2BF6D1FF23974A84
:100428008AF817308AF818308AF819308AF81A309A
:100438008AF81B30924BDFF86CB21360914A039331
:10044800042010705846302215F08BFC142202212B
:100458008BF800208BF8241001228B49039B8BF822
:10046800182097F805B081F800B0A3F5F071CAF824
:100478001C108649D8F80080A3F590730B60844B54
:1004880003EBCB0318F0200F5B78CAF8203018BFB5
:10049800CAF8202000237F4A40F2DC5122F81310CA
:1004A8000133082BF7D113A800211C2215F059FCA1
:1004B800BBF10E0F03D00BF0EF03082B02D1012381
:1004C8008DF85C3002200BF00DF818B14088003030
:1004D80018BF0120C8F340038DF85230C8F38013C9
:1004E8008DF85430C8F340338DF84C30C8F3C0331E
:1004F80000F001008DF84F3018F400638DF85100BA
:1005080007D097F8863103F1FF3EDEF1000343EB95
:100518000E038DF85030C8F300438DF85530336A18
:10052800B7F84801ADF86000003318BF01238DF813
:100538005630C8F300538DF85730B7F84A31ADF844
:100548005A3018F4805FB7F8563118BF4848ADF8EC
:100558005830C8F380438DF85330B7F854311CBF76
:10056800B0F85001ADF86000B3F5FA7FADF85E3031
:1005780084BF0023ADF86030474897F8D63186F835
:100588002430002386F8253043709DF85C3008F04D
:100598000101002BC8F3C0028DF84D108DF84E20D4
:1005A8000CBF0023022301B902B1013309EB83090F
:1005B8004FF0000AD9F810309A1E143303920593AD
:1005C800039A32F8023F03924FF6FF72934200F00B
:1005D80089819DF85100190ADAB2CBB280B1264F51
:1005E800DFF8C4E007EB02177868704508D138894E
:1005F800B0F5806F00F07181B0F5006F00F06D818B
:100608009DF8550090B11001DFF86CE00EEB000783
:100618005EF800E02148864500F05F817868B0F117
:10062800904F03D1B87B062800F057819DF85200FF
:1006380050B1114F07EB02177868B0F1904F03D112
:100648003889102800F049819DF8500050B10A4FB0
:1006580007EB02177868B0F1904F03D138898028EA
:1006680000F03B81022921D19DF84C1022E000BF07
:1006780050120020C81F0020D0A301081C2B002006
:1006880044140020251200209C0900200C21002081
:1006980070B10108941100209D0100200044014020
:1006A80078010020202B002000040048012904D1F3
:1006B8009DF84D10002900F010819DF85600BF49A3
:1006C8004FEA021850B19DF85C0038B9012A05D8E4
:1006D80051F80800BA4FB84208BF04239DF85700E4
:1006E80001EB080730B19DF85C0018B9043A032AF9
:1006F80040F2DC80012B53D19DF85330DFF8D092C3
:100708003BB151F80830B3F1804F04BF032389F897
:100718002730AA4AC9F87C7002EB0801FF2391F838
:100728000DE089F86C3089F86D3048688DF86AE01A
:1007380001F108030989ADF868104FF0000B022198
:100748008DF86B1089F870B01AA90792069389F88A
:1007580028B0C9F82CB0C9F830B0C9F834B0C9F815
:1007680068B089F86EB089F86FB004F0D5FA069BC6
:10077800079A997852F808005A4604F021F9384641
:1007880011F0E8FC8F4B9049C9F880308F4BC9F8BD
:100798008430C9F888B038460A1D11F089FA9CE0FF
:1007A800022B49D15FFA8AF21C2101FB02FC884A1C
:1007B800CDF81CC002EB0C09804A89F871A0012110
:1007C80089F8701002EB08014FF0000B91F80DE06A
:1007D800486889F872B001F108020989ADF8681013
:1007E80089F87AB01AA9C9F87C708DF86AE006927F
:1007F8008DF86B3004F090FA704B069A53F80800A5
:1008080091785A4604F0DCF8384611F0A3FC704B96
:10081800DDF81CC06F4AC9F8802003EB0C016E4A52
:10082800C9F884208031C9F888B038460A1D11F00B
:100838003FFA0AF1010A50E0032B35D19DF85330F5
:10084800DFF88C81DFF8C4913BB198F826B03846C0
:1008580008214FF6FF7200231AE0BDF85E2098F8D1
:1008680026B0BDF86030B2F5FA7F0BD95B49B1FB11
:10087800F2F23846082192B204F077FA584B49F858
:100888002B000AE05749B1FBF2F23846012192B237
:1008980004F06BFA544B49F82B00C36098F82630E3
:1008A800013388F8263018E0042B16D196F82580F5
:1008B800BDF858204B4B93FBF2F23846BDF85A303E
:1008C800012192B204F051FA96F8253006EB880817
:1008D8000133C8F8500186F82530039B059A9342E6
:1008E8007FF46EAE96F8252086F870213F4A404B7B
:1008F80092F800E0AEF117020027022A1F709C460A
:100908001AD8F3693B44D3ED007AF5EE407AF1EE5C
:1009180010FA02D1336A63BB26E0364A07EB0208B5
:100928000FCB88E80F009CF8003010370133C02F38
:100938008CF80030E5D1EDE72F4B13F83E908CF89A
:10094800009003EBCE03D3F804A0BAF1000FE1D076
:100958004F45DFDA274A3B0103EB020853440FCB2C
:10096800013788E80F00F3E7244F3B68DE0451D4D1
:100978001DE0234B234A13F83E00107003EBCE030F
:100988005E68002EF0D000238342EDDAC3EBC3018A
:100998007218DFF87C80D2F8009041F8089001EBDB
:1009A80008079188B9809279BA710133ECE70EF0A3
:1009B800EF03082B144B4DD14FE000BFD0A3010823
:1009C8000040014051470008F80100203D48000858
:1009D80078010020C54A00082947000800127A005B
:1009E8005D48000840420F004D4800089C0900205F
:1009F800C41F0020D808002070B10108582E00201C
:100A08009489010898200020441A0020941F00208F
:100A1800992000209CF80020012AC8D9B94B03EB83
:100A28000212103210339342C1D053ED047AB6EE5D
:100A3800007A67EE877A43ED047A53ED057A67EE1C
:100A4800877A43ED057A53ED037A67EE877A43EDAB
:100A5800037AE7E7BEF10E0F09D11A7842F01002C7
:100A68001A70BEF1180F09D10BF0FEF906E01A78DA
:100A780022F010021A70BEF1190FF4E70BF0D8F942
:100A88003B68A14E58035EBFA04B01221A70049B1D
:100A9800049A1B7843F0040313709D4B1E6063692E
:100AA80043F400336361E36943F48003E361236B38
:100AB80023F020032363236B43F080534FF09048C7
:100AC80043F020032363D8F8243023F0F003C8F858
:100AD8002430D8F8243043F04003C8F82430D8F83C
:100AE800243023F47063C8F82430D8F8243043F451
:100AF8008063C8F824304FF0000902234FF40072D5
:100B080029464FF0030B40468DF86C3004931A9237
:100B18008DF86E908DF86F908DF86DB007F0D0FC61
:100B28004FF48062294640461A9207F0C9FC3268A1
:100B380022F0010232603168764A0A403260764A11
:100B48003261326842F001023260C6F80890C6F895
:100B58000C90C6F80890B26842F40042B26032685D
:100B68003260726822F0784222F400427260326881
:100B780042F0010232603D68684E4FF0100A05F4F9
:100B88000063524630464946039315F0EAF84FF69B
:100B9800FF72049B0E9215F002058DF83D308DF81A
:100BA8003E908DF83F908DF83CB00CD02EA9404671
:100BB80041F880AD07F084FC01250723357086F8DD
:100BC8000190F370B570039B83B12EA9802341F87F
:100BD800803D4FF0904007F073FC042333730723E4
:100BE800F373012375731D44B373EDB2E36A4C4884
:100BF80023F4F873E362E36A43F4D873E362636946
:100C080043F0805343F00203636107F020FA1AA807
:100C180007F0F2F9434B1A93434B1B93022D4FF005
:100C2800000314BF1A4680221F924FF480723C4C76
:100C380020924FF4806221922022204622921AA903
:100C48004FF400521C931E9323922493ADF87450D2
:100C580007F0DFF9236843F001032360334CA368EE
:100C680023F04053A360A36843F08053A3600A2095
:100C78000AF0C9FDA36823F08043A360A368A360BA
:100C8800A36843F00043A360A368284A002B51DA05
:100C9800FAE7013A092A3FF685ABD9F8240003930D
:100CA8002946AAF828B028604FF0904004F034F89C
:100CB8004FF09042082191613C200AF0A4FD039B6B
:100CC800CAF818B09A4697F893319A45BFF664ABBC
:100CD800174A4FF0904B1021082391617820069114
:100CE8000592ABF8283003930AF082FD059A06991D
:100CF800039B11857820CBF818300AF079FD0AF1AA
:100D0800010AE0E7E008002000580040080E002033
:100D180060110020FFE0CF007A25E000C41D00200C
:100D28000804024040010050D41D0020000100507A
:100D3800000400489368AC4923F0405393609368DB
:100D480043F0005393608868A84B034043F468332A
:100D58008B60D168A64B0B4043F40053D360136BF0
:100D6800013D23F00F031D431563002401233219AD
:100D78009178002972D05D1C042B16F804E0D07815
:100D8800DFF870C2EDB20ED803EB43035A00DCF86B
:100D980030101F23934021EA03010EFA02F30B439C
:100DA800CCF8303031E0092B0ED8053B06225A43E7
:100DB800DCF834101F23934021EA03010EFA02F3F2
:100DC8000B43CCF8343020E00E2B4FF006010ED840
:100DD800A3F10A024A43DCF838801F23934028EA2B
:100DE80003010EFA02F30B43CCF838300DE00F3B49
:100DF80001FB03F2DCF83C801F23934028EA03013F
:100E08000EFA02F30B43CCF83C30BEF1090F794AD5
:100E180011D993699169AEF10A0303EB43034FF0CB
:100E2800070E0EFA03FE21EA0E01916191699840BE
:100E38000843906111E0536951690EF1FF3303EBE8
:100E480043034FF0380E0EFA03FE21EA0E015161FA
:100E5800516903339840084350612B460434102CE1
:100E680085D1644B9A6842F001029A601A4611686B
:100E7800604BC907FBD5DA685F4C22F00202DA60E2
:100E8800DA6842F00202DA60DA6842F00102DA60F7
:100E98009A6842F004029A60B4F85C31002B40F082
:100EA800B887B4F95E21002A40F0B387B4F960210D
:100EB800002A40F0AE873B689B0320D5C8200AF083
:100EC800A2FCAE2010F0C1FD08B110F0C3FD4B4DDF
:100ED80085F87101C8200AF096FC494BC5F87431B1
:100EE800484D00210C22284614F03BFF0223EB70EA
:100EF8000BF0A3F90AF060FC434B0344AB6094F891
:100F08006B310393414B42481B68B4F86461B3F8F2
:100F18005630049300210C2294F863B194F86C5174
:100F2800B4F80C9094F80FA014F01BFF394B0693FB
:100F380018460021142214F014FF374A00211170BA
:100F48002E4A0592C2F8781110F041FD059A8046A4
:100F5800002833D0069B314919603149596031491D
:100F6800D960B6F5807F30491961304B01D1002135
:100F780016E0BB2E01D9012112E0612E01D9022110
:100F88000EE0292E01D903210AE0132E01D90421EC
:100F980006E0092E01D9052102E0002EE7D006213E
:100FA80019701D4B04211970214B02211970214918
:100FB8000B6843F001030B6059460FE003200AF069
:100FC80067FD35E24FF0010B0BFA01F040F2B23346
:100FD80003409BB3012940F28D800021164800236D
:100FE80009290370F9D8EDE700030050E010FCFF71
:100FF80007C0FFFD000100505012002078010020BA
:10100800DA13002048210020404B4C00A411002096
:10101800702B00204C28002060280020B9180108F7
:10102800C91701084918010890C1793D000000203E
:1010380004010020401A0020EE2F002010F04D0F70
:10104800C8D00691C2F87831059210F0C0FC059A14
:1010580006990028BED0062168200A460DEB000339
:1010680003F070FF9DF86D1001EA0B029DF86B10FC
:1010780001EA0B0101FA0BF343EA82019DF86920AA
:1010880002EA0B030B430BD05BB25B4501D1002294
:1010980002E0022B0FD10122AF4B83F87C2111E033
:1010A8000EAB68200C215A4603F04CFF9DF83830EF
:1010B80013F00F0303D105200AF0EAFC02E0042B29
:1010C800E9D1E4E7A54BA64A1A60A64A5A60A24AA3
:1010D80092F87C21002A0CBF6F226E221A72A24B52
:1010E80004221A70A14B03225A70A14A136843F0D4
:1010F80002031360042D00F2A380DFE805F003BEAD
:101108006B036B000A200AF07EFB7720A0210122E6
:101118000EAB03F017FF00285CD01E2101227720B8
:1011280003F08CFF4FF42F600AF062FB4FF0000BC6
:10113800ABF160010025C9B202221AAB77208DF805
:1011480068508DF8695003F0FDFE9DF869309DF8F0
:10115800682043EA0222804B03F5BF712BF8012077
:101168000BF1020BBBF1100FE2D1B3F88C2102F0A6
:101178000F0E02F47F42A3F88C2101202B4629464A
:10118800DFF8D4C121F001056544B5F87E51002D82
:1011980018BF002011F0010F03D0EDB26B400825F5
:1011A80002E083EA1523FAE713F4004F18BF83F42B
:1011B800C053013D4FEA4303F6D101311029DFD175
:1011C800654942EA0E02A1F88C2118B9C3F303332A
:1011D8009E4538D0604D95F88EB1BBF1000F40F0B8
:1011E8000E8614200AF00FFB05F28F137620D0210B
:1011F800012203F0A7FE95F88F31582B3DD105F554
:10120800C87388211822762003F09CFE31227620AC
:10121800F42103F013FF012385F88E31554B564A0C
:101228009A60564A5A6045F6D8125A80544ADA608B
:10123800544A1A61544AA3F800B05A6100F0DFBD5D
:10124800012D13D119E04B4B42F210721A805A80CB
:101258004E4A5A604E4A9A604E4ADA604E4A1A61BD
:101268004E4A5A61B8F1000FB4D003253F4B404AAB
:101278009D70136843F0040313603D4D2B689B0772
:1012880002D5364B1B6898473349454ABAF1000FD7
:1012980025D016F0FF0F0AD12B6813F0020F4FF07C
:1012A8007D0040F2712308BF4FF4FA7302E04FF457
:1012B8007A731846994505DBB9F57A6FA8BF4FF4DC
:1012C8007A6900E09946431E4B44B3FBF0F3013BB7
:1012D800DBB203FB000081F8AC31106003E081F859
:1012E800ACA1C2F800902F4B1B689847DDF80CA002
:1012F8002D4E00233370BAF1000F04D0AAF1020278
:10130800012A00F27F852EAB4FF0000903F8509DAB
:101318000C204946012203F015FE002800F0A185A3
:101328009DF86830482B13D1204B214A1A60214A76
:101338005A604046B8F1000F00F0938505233370DA
:101348000A4B0322DA702B6843F008032B6033E062
:10135800484600F086BD00BF78010020702B0020B1
:101368002919010809180108EE2F0020040100209E
:10137800401A0020D8060020516D0008536D00085F
:10138800E16F000877700008556B000877170108AF
:10139800B91701086D170108A9170108556D00084C
:1013A800982C00204C280020E82F0020B4060020AC
:1013B800C1700008EB6F0008174B93F858210AB169
:1013C80016490A7093F859210AB115490A7093F819
:1013D8005A3103B133702B68124913F0080F25D026
:1013E800BDF91000DFED106A642290FBF2F302FBF6
:1013F800130212B207EE902AB8EEE77A07EE903A97
:10140800F8EEE77AE7EE267AB2EE047A67EE877AA4
:10141800C1ED007A0CE000BF5012002060280020C7
:10142800EE2F0020B42700208988883C00230B6019
:10143800BA4D2B7843F002032B70B94B20221A8542
:1014480010229A610A26DFF8D882B8F814309BB2C5
:1014580083F02003A8F81430B8F814309BB283F056
:101468001003A8F8143019200AF0CDF9013E19200C
:101478000AF0C9F916F0FF06E5D110234FF020094C
:10148800A84EC8F81830C8F818903368180709D556
:10149800A54BA8F828901B689847A44BC8F8189043
:1014A80001221A70A24B9FEDA38A1B68DFF8CC8239
:1014B8001B7B00EE103AB8EEC00A20EE080A08F0CE
:1014C80005FAB8F8003007EE903AF8EEE77A27EE1A
:1014D800800A14F055FE984B9FED987A1880B8F85A
:1014E800003007EE903AF8EEE77A954BC7EE277A88
:1014F800FF211B229FED937AC7EE877A9FED927AA0
:10150800C3ED007A914BD3ED047A914B67EE887A5C
:1015180067EE877AC3ED007A8E4B184614F021FCEB
:10152800002202703268DFF858E2012112F0020F3F
:101538008EF800101FBF417003218EF800100221A1
:1015480018BF8170510741BF9EF800104E1C8EF8DD
:101558000060032648BF465412F00A0F73460ED0A7
:101568009EF8002004218154511CC9B20526465416
:10157800D11C0232D2B28EF80010062181543A688A
:10158800960641BF19784E1C1E70072648BF465460
:10159800110608D51978092646548E1C0131C9B29E
:1015A8001E700A2646546C4E7779082F01D00E2FEC
:1015B80008D1197801F1010E83F800E04FF00B0E05
:1015C80000F801E0197812F4803F4FF00C0C00F895
:1015D80001C001F1010E1CBFDFF8A4C102315FFA9E
:1015E8008EFE83F800E01FBF8CF8001059494FF0B9
:1015F8000E0C01F80EC0510741BF197801F1010E18
:1016080083F800E04FF0100E48BF00F801E01978A9
:1016180001F1010E5FFA8EFE4FF0120C12F4806F8A
:1016280083F800E000F801C00ED096F818C2BCF1AB
:10163800000F09D0DFF848C102318CF80010454985
:101648004FF0130C01F80EC0197812F4007F4FF018
:10165800140C00F801C001F1010E1CBFDFF820C115
:1016680002315FFA8EFE83F800E01FBF8CF800108D
:1016780038494FF0150C01F80EC0182F13D11978FE
:101688004FF0160E00F801E001F1010E5FFA8EFE30
:101698004FF0170C00F80EC001F1030E0231C9B269
:1016A80083F800E04754110341BF19784F1C1F709D
:1016B800192748BF4754D20541BF1A78511C1970E1
:1016C8001A2348BF835400219822244814F049FB68
:1016D8000EF031FF224B234A1A60234BB4F8521103
:1016E8001980224900230B808B7021490A60B4F8C5
:1016F800982190B21F4921F813000133122BF9D118
:101708001D48036813F4805F804604BFB6F89E0145
:1017180008801B0740F1FE8034E000BFC02F002086
:1017280000040048401A0020B4060020CC0600201F
:10173800F428002035FA8E3C102900200AE81C41C4
:10174800EC07002000401C46BD3786354C28002099
:10175800F02800206D11002050120020782A002067
:101768003C0F0020DA130020400F0020DC2E002060
:10177800B42F0020942E0020582E002004000020B2
:101788006C11002096F89231062B00F2BD80DFE83C
:1017980003F004070E3D5878780045F2F05201E056
:1017A80042F6F822854B1A800EF062FFABE007EE96
:1017B800902ADFED836A814BB8EEE77ADFED817A14
:1017C800E7EE267A42F6F82119800023FCEEE77A44
:1017D8007D4A17EE901A42F823100133122BF7D1E5
:1017E8007A4A7B4911607B4A4020137009F0B2FEA7
:1017F800002800F0898001234FF0070990F90000C4
:10180800754A8DE808024021744B77E06B4B42F62D
:10181800F8221A806D4B724A1A606E4B10224020D3
:101828001A7009F097FE00286ED001234FF0000CC3
:1018380090F900006B4A8DE8081040214FF4E1331D
:101848005CE05E4B42F6F8221A80604B664A1A60EA
:10185800604B082240201A7009F07CFE002853D003
:1018680001234FF0000E90F90000604A8DE808400F
:1018780040214FF4E13309F0D0FF5D4BC3F8B001CC
:101888003EE04E4ADFF89C91DFF89CC1DFF89CE10E
:10189800584F594C594842F6F82111804D490C22AD
:1018A800062B0A700ED0002389F800308CF800301F
:1018B8008EF800301B233B700523227003704FF411
:1018C800E1340BE0002189F800108CF800108EF844
:1018D8000010227021214A4C397003703B4B494A51
:1018E8001A60402009F036FE70B101230027464AED
:1018F80090F9000040218DE88800234609F08DFF0B
:10190800003018BF012028B9082008F0A3F82F4B91
:101918003E4A1A60D8F800302E4A13F4804F1FBF91
:101928000821117029493A4818BF086042F201019C
:10193800194003F0010003F4005479B11F4944F63B
:1019480020670F8024B1082111702049314C0C60A8
:1019580020B10C2111701D492F4808601178180614
:10196800A1F10401517040F19D802148DFF8C09039
:101978002A4FC0F8B47100242146152200F5DC7006
:10198800DFF8B0A089F80140C9F80440C9F8084058
:10199800053F14F0E6F92046CAF8007005F0CAFEC3
:1019A8001F4B02201B68C9F80C3009F0D3FD002832
:1019B80042D1802008F04EF86CE000BF44080020B7
:1019C800CDCCCC3F0000B0C4042F0020F400002090
:1019D800CD2A0108142B0020D92B0108A08601006C
:1019E800317C0008312B0108197C0008657D00084E
:1019F800780100205A1D0020DB1C00205B1D002000
:101A080090D00300357B0008457C00082D2B010889
:101A1800012B01081D2B01080D2B0108441400207F
:101A28007C2E0020DC1C0020591D0020581D0020A1
:101A38000008002020080020447999F80130C649A0
:101A48000C2202FB03125278A24204D00133DBB20B
:101A5800042BF4D9002389F80130DAF8003099F81A
:101A680001201B7890F90000002B4FF00C0303FBBA
:101A7800021314BF0324012400225B78009401920E
:101A8800022109F0CAFEB54B1860002891D0012048
:101A980005F050FEB24B1868B24B00F5C5721A60DB
:101AA80005F0F6FEB04AB14B1360B14AB14F80332E
:101AB8001360D8F800300024D9033C7040F1AD80A1
:101AC8000DF04CFFDFF810C3DFF810A3CDF810C0FD
:101AD80040F22A3B4FF00109604621465A4687F8F2
:101AE800009014F03EF9DAF81430A34F4FF090400C
:101AF80043F40033CAF81430036A23F070630362B6
:101B0800036A43F080730362402302220C930CA9FA
:101B180003238DF8342003928DF835308DF8364044
:101B28008DF8379006F0CCFCDAF81830039A43F4B5
:101B38000033CAF818303B8823F440731B041B0C8D
:101B48003B801D23FB620EA93A8560233C863846FC
:101B5800C7F814900E93ADF83E401094ADF8444089
:101B6800ADF84640ADF84840ADF84A40ADF83C9075
:101B780006F0FAFABB6943F00803BB617B6C43F4D7
:101B880000437B64DAF8143043EA0903CAF81430D6
:101B9800AAF57D6A504606F05AFA1AA806F02CFAF9
:101BA800764B1A9310231C9380231F934FF4807352
:101BB800DDF810C020931AA94FF400535046CDF811
:101BC8006CC02393ADF874B01E942194229424948D
:101BD80006F01FFAFB6843F40073FB60DAF8003084
:101BE80043F00203CAF800300BA80D238DF82C30FF
:101BF8008DF82D908DF82E408DF82F9010F08CFADE
:101C080021465F4B1A685F4B43F821200131202998
:101C1800F7D102F0A3FF02F0A1FFD8F800305A056F
:101C280056D5594F594BD7F8F894C3F8009004206B
:101C380009F090FC0421C7F8FC0409F067FC544B38
:101C480087F800050820C3F8009009F083FC514B81
:101C5800514C1860082109F059FC002187F801054A
:101C68002C22204614F07DF88E2363704FF07C0BF5
:101C7800E0234FF07D0AE37084F800B084F82BA0CD
:101C8800464C2C220021204614F06BF88A236370FE
:101C98001020A023E37084F800B084F82BA0C7F8C4
:101CA800049509F057FC1021C7F8080509F02EFC27
:101CB80087F80C052020C7F8109509F04BFC202167
:101CC800C7F8140509F022FC87F818050AF08CF902
:101CD800D8F80030324A13F4002318BF01231370D8
:101CE80009F06AFD2F4B18607379052B02BF2E4B44
:101CF8004FF4C8721A802D4B4FF47A721A802C4B0D
:101D0800C8221A802B4A137843F0080313702A4A12
:101D1800137823F002031370D8F8002040F602036A
:101D280013406BB1254B26491960264B03211970C6
:101D3800254B01211970254900230B8024490B806C
:101D4800930341BF234B04221A71DA7844BF42F04F
:101D58000102DA7044E000BF4C81010844210020F0
:101D6800A4110020900F0020902700207814002054
:101D780088210020090E002000440140344401401D
:101D8800108101080A0E002078010020341A002072
:101D98008C1A0020D81A00205C1A0020911A002002
:101DA800942C00208C0E0020BC280020E62F002058
:101DB800E02F0020441A0020EA2F00202C1A0020CF
:101DC800CC130020901A0020FC00002030100020C6
:101DD8003210002048210020450300200010024056
:101DE800B368C8F80030234B01221A702B7863F0CF
:101DF8007F032B702FB0BDEC028BBDE8F08F04255C
:101E0800FFF734BABAF1010F7FF6D6AA9A46FFF760
:101E18006FBA1BB207EE903ADFED176AB4F95E317C
:101E2800164AF8EEE77A07EE103A67EEA67AB4F9A2
:101E38006031CDED1A7A07EE903AB8EEC77AF8EE2F
:101E4800E77A002127EE267A67EEA67A11701AA89B
:101E58000B498DED1B7ACDED1C7A07F03FFDFFF79E
:101E68002AB8BAF1010F7FF6A7AA4FF0000A30701E
:101E7800FFF749BA080E002035FA8E3C38000020DA
:101E8800A01D0020924A2DE9F04F1368914C03F5EC
:101E98009C4320332DED028B23608F4B196889B04A
:101EA80011F4804F0592984605D110F0E3FE10B961
:101EB8002379013323716779A7B1864B013F5F719D
:101EC800DBE0D9F800308548072D98BF595D844B71
:101ED80088BF29461B689847032D0BD904EB450595
:101EE8000137E8807D4BDFF814921E78FDB2AE42D0
:101EF800E7D820E0D9F8002005F10E0302EB8303B0
:101F08009988DA880028E9D04FF47A73401A584340
:101F1800531A90FBF3F040F6C90300F57A70984223
:101F280005DC40F2EE239842B8BF184601E040F6BF
:101F3800CA0080B2D2E70F23277984F82A3094F8B0
:101F48002B300193032594F82C30B7FBF5F505EBFE
:101F580045057D1B0393D9F800300293DFF8A4A14F
:101F6800EBB204930025B54254DA5E49019B31F87F
:101F780015B04FEA450953B910F07CFE28B1039B10
:101F8800002B08BF4FF0000B01E0DDF804B0029B06
:101F9800988A584502D8D88A58450ED2E8B210F027
:101FA8003FFE032D8346DFBF94F82AE00120A840B6
:101FB8002EEA0000D8BF84F82A0010F05BFE18B1A2
:101FC800494829F800B021E0049B94F876002AF8E3
:101FD80013B028B9022F15D93E49012081F876009F
:101FE800BAF80210BAF800000844BAF80410084415
:101FF8003E4980B229F8010000B2032190FBF1F0BC
:1020080080B200E05846384929F8010001350AF144
:10201800060AA8E794F82A203548364BA2F10F01A2
:102028004A424A4184F890206AB1334A1268520100
:1020380009D40268D9689A60521AC82A1DD901229F
:1020480083F8212019E002689868DA605B68121A40
:102058009A4288BF274B4FF0000184F82B1088BFA5
:1020680083F821100025B54207DAE8B210F0D8FD50
:102078001D4B23F815000135F5E7D8F80030DF04CB
:1020880005D51D4B1B68DE0701D410F011F8059B20
:1020980019681A4B1868837AB3B3013B124D027B57
:1020A80035F813301AB1C3F53B6308339BB21BB242
:1020B800A3F57A73B3F57A7FA8BF4FF47A7323EA4E
:1020C800E37307EE903A9FED0E7AF8EEE77A54E064
:1020D800C82F0020900E0020582E0020142B00201E
:1020E800F4000020960E0020942E0020080F0020F7
:1020F8007C2E0020DC2E002068110020B42F002048
:1021080000007A44BE0E0020D8F80020150440D5FF
:10211800D4F89420934E8A1A002A3ADB01F59C429F
:102128002032C6F89420904AC07A55798F4A32F8FE
:10213800152096F89850013592B292FBF0F205F00E
:102148000F0086F89800304480F899201A4688488D
:10215800185C01330244102B92B2F8D112B292FBF0
:10216800F3F31BB2642BA8BF642323EAE37307EEDF
:10217800903A9FED807AF8EEE77AC7EE877A7E4A42
:102188009FED7E7A67EE877AFCEEE77A17EE903A53
:102198001380D8F800307A4F13F4807F00F009815B
:1021A800784BDFF8E491994205D999F8022012B9E1
:1021B800012289F8022099F80220002A00F0F9800B
:1021C800714A3E7892F821506A1E554255416F4A2D
:1021D8001168002DC1F38063C6F38006019392460F
:1021E80014BF4FF0000B4FF0030B99F82020052A7D
:1021F80000F2D980DFE802F0034D527584A1002E69
:102208003AD0D4F8AC00B4F8B01009F044FA012878
:1022180009D15F495F4A09681268C988642000FBD0
:102228000122C9F81020019B6BB1594A1268127932
:102238004AB110F02BFC032289F820204FF47A725F
:10224800C9F81C20D1E7002D40F0AD80514AD9F8DB
:10225800101010684C4A88420AD9029210F016FCF5
:10226800029A032182F8201040F6B831D161BCE708
:10227800012182F82010B8E7019B4FF4806013B168
:1022880007F0D8FB01E007F0C4FB0022C9F81020D2
:1022980089E0002D46D110F0F9FBA6E725B105220B
:1022A80089F82020012000E0284666B1D4F8AC2047
:1022B800D189394A11805180918035490968498806
:1022C800D1804FF0020B334A1168D9F8142091429B
:1022D80001D8002E64D147F23052C9F81C200322DD
:1022E80021E03A7842F002023A700FF0E1FE294A02
:1022F800D9F81C1012680A44C9F81820042212E000
:10230800244A9DB11168D9F8182091424BD9234A23
:1023180012781AB9DAF80020D30744D43A7822F0B0
:1023280002023A70052289F820205EE71268D9F87F
:102338001C100A44C9F8182035E01549154A0968DF
:102348001268C988642000FB0122C9F810204FF4E4
:102358008060002289F8202089F8032007F059FBC3
:1023680043E700BF900E0020C41D0020D41D0020AC
:10237800290F00200000C842C411002000C07F447B
:10238800EA2F0020404B4C00DC2E00206811002072
:10239800002F00207C2E0020942E00200300002017
:1023A80000287FF422AFBBF1000F02D0584609F095
:1023B800C9F9924D05F5C570B5F8521109F06BF9D8
:1023C800834668B910F054FB8D4BC3F800B0C3F8CE
:1023D80004B0C3F808B08B4B00221A605A609A60A8
:1023E8003B785E0736D5D8F80030D80632D5864B0C
:1023F8001B78D9062ED4854B1B7893B195F8E2311A
:10240800BBF1000F15D17BB1814B1A68D4F8B430F9
:102418009B1A002B08DA0FF04BFE7E4B83F8B8B0FE
:1024280018E0BBF1000F0DD1102009F08BF9012342
:102438000EE03BB1764A12684FF47A7101FB032330
:10244800C4F8B43094F8B83023B109F069F900231E
:1024580084F8B830002295F8E0A195F8E111B5F8B4
:102468009AE1B5F89CC113466B4E019636F91200F5
:102478009B087045C4BF63F07F03DBB2013260453F
:10248800B8BF43F04003042AEED194F8B92061485C
:102498009A4205D190F8BA20F92A04D8013200E00E
:1024A800002280F8BA2084F8B930584B5B4E1A786D
:1024B8009946E2B93368DA0708D5BBF1000F16D19F
:1024C8003B78DB0713D50FF05FFC10E03B7858072B
:1024D8000DD5504B93F82B304BB1514BDB7833B9BA
:1024E80011B10FF0E5FD02E0BBF1000FF9D094F84F
:1024F800BA30484ADFF844B1142B40F0B18099F85B
:1025080000301AF1000A18BF4FF0010A6BB392F8B5
:10251800B9305F2B11D13B7803F0040303F0FF01BE
:1025280013B10FF0C5FD08E00B200391029209F0EA
:1025380009F9029A039982F8BA10BAF1000F14D077
:1025480094F8B9307D2B10D13B7803F0040303F0E5
:10255800FF0213B10FF0ACFD07E00B20029209F067
:10256800F1F82C4B029A83F8BA203B7803F0040365
:1025780003F0FF01002B73D194F8B930254A572B8B
:1025880016D1284B4FF47A721A80D8F80030190601
:1025980001D505F0DFF9244B1B685A0742BF234ACF
:1025A8000A21118013F008035AD1214A138057E0F9
:1025B800D8F80000400716D55A2B14D11D4B1878AF
:1025C80020B119701C4B01221A7049E092F8BB30F7
:1025D80083F0010382F8BB300BB10C2000E00D2022
:1025E80009F0B0F83CE05D2B00F02F855B2B00F084
:1025F8002E855E2B24D1032000F02ABD5012002026
:10260800D8270020B01E0020441A00200300002014
:102618007C2E0020900E0020942E002068110020AF
:10262800DC2E0020E62F0020401A0020E02F00209A
:1026380040120020E9280020EA280020A4110020E8
:10264800562B03D1029307F091FC029B99F80020C6
:10265800002A00F012856F2B40F009850FF094FBDB
:10266800D8F80030580732D594F8BB30A3B13B787E
:10267800590711D5019BB3F90620B5F89A319A424A
:102688000ADD336813F0010301BFAF4A322111801C
:10269800AE4A08BF82F8BB303368DA030AD5AC4BC0
:1026A8001A782AB9AB4A127812B9A74A322111808E
:1026B80001220BE0A74A13784BB13B7803F00403DF
:1026C80003F0FF011BB9A44B117001221A70DBF84B
:1026D80000A0002333600AF17B090AF1CB0B99F8BB
:1026E800002099F8013019F8010C9A420BD249469A
:1026F80008F09AFF38B119F8022C012303FA02F204
:1027080033681343336009F10409D945E7D1934B82
:102718001B7853B1924B934E1A68DFF860A212F0FF
:10272800020F994640F048833FE30AF1CA060AF5CA
:1027380089793278737816F8010C9A4225D2314695
:1027480008F072FF08B3B37896F804E0864A96F862
:1027580003A07E480C21013B01FB0E4103EB430320
:102768001344D1F8C0209A420FD0C1F8C0300023DA
:1027780090F8EC20C1F8C430012303FA0EF322EAE2
:10278800030381F8BCA080F8EC3006364E45D0D162
:10279800764B1E68764B1B68039394F82B30049392
:1027A800744B029300230193029B1B68002B00F0DB
:1027B800F18293F800A0BAF1000F00F0EB82029AC0
:1027C800039952688A1A002A0CDB01F5FA720299F9
:1027D8004A60019901228A4094F8EC1021EA020229
:1027E80084F8EC20049A002A00F0D482029A5978DE
:1027F80012F8042C0432D2B2002940F08A825E49D1
:1028080031F91210B5F8982102F1C800814202DDB1
:1028180093F802B015E0C83A914203DA9978C1F109
:10282800000B0EE0019A0123934094F8EC2022EA71
:10283800030384F8EC30039B029A03F5FA735360A0
:10284800A8E294F8EC30019A1341DB0700F1A28268
:10285800BBF1000FCCBF0220012008F095FF0AF160
:10286800FF33DFF8E890132B00F28C82DFE813F0D7
:102878001400250037004B0064008E00F500580155
:10288800BF01EF011F028A024B005A008E00F500BB
:102898005801C5002A018F0196F80090D944B9F172
:1028A800FA0FA8BF4FF0FA0929EAE979304686F805
:1028B800009008F09FFE01200FE096F80190D9449F
:1028C800B9F1640FA8BF4FF0640929EAE9793046E5
:1028D80086F8019008F08EFE02204946E4E196F859
:1028E80003A0DA44BAF1640FA8BF4FF0640A2AEAD9
:1028F800EA7A86F803A03046D9F8F01008F030FEDE
:1029080003205146D0E1717959446429A8BF642154
:1029180021EAE17171710D2008F0EEFEBAF10D0F98
:1029280000F03082317959446429A8BF642121EA32
:10293800E17131710E20B7E1B179594481F3080191
:10294800B1710520B0E100BFD0280020900E002012
:10295800E8280020E9280020EA280020EB2F0020A2
:1029680068110020401A002038850108C81100208D
:102978007C2E0020500F0020942E0020081B0020E1
:1029880000007A440000C84200000000D9F8F43082
:102998001A78022A22D107EE90BAF8EEE77AB2EE58
:1029A800040A87EE800AD3ED097A30EE270AB5EEDD
:1029B800C00AF1EE10FA09D45FED0E7AB4EE670A98
:1029C800F1EE10FAC8BFB0EE670A01E01FED120A77
:1029D80083ED090A0F2008F079FE0AE09978594436
:1029E800C829A8BFC82121EAE17199700F2008F011
:1029F80083FEBAF10F0F00F0C581D9F8F4301A78C8
:102A0800022A20D107EE90BAB8EEE78AB2EE040A9D
:102A180088EE008A93ED080A38EE000AB5EEC00A7F
:102A2800F1EE10FA09D45FED297AB4EE670AF1EEF7
:102A380010FAC8BFB0EE670A01E01FED2D0A83ED5A
:102A4800080A122058E159785944C829A8BFC82152
:102A580021EAE1715970122026E1D9F8F4301A7888
:102A6800022A20D107EE90BAB8EEE70A5FED3B7A6A
:102A780093ED0C7A80EE270A30EE070AB5EEC00A0D
:102A8800F1EE10FA07D4B4EE670AF1EE10FAC8BFF7
:102A9800B0EE670A01E01FED440A83ED0C0A10202E
:102AA80008F014FE0AE0197B5944C829A8BFC821B8
:102AB80021EAE1711973102008F01EFEBAF1100F17
:102AC80000F06081D9F8F4301A78022A1ED107EE96
:102AD80090BAB8EEE78A5FED557A93ED0B0A88EE67
:102AE800278A38EE000AB5EEC00AF1EE10FA07D4CC
:102AF800B4EE670AF1EE10FAC8BFB0EE670A01E05B
:102B08001FED5F0A83ED0B0A1320F5E0D97A5944CB
:102B1800C829A8BFC82121EAE171D9721320C3E0EE
:102B2800D9F8F4301A78022A22D107EE90BA1FEDAC
:102B38006C0AF8EEE77A87EE800AD3ED0F7A30EE6A
:102B4800270AB5EEC00AF1EE10FA09D45FED737AE0
:102B5800B4EE670AF1EE10FAC8BFB0EE670A01E0FA
:102B68001FED770A83ED0F0A112008F0AFFD0AE088
:102B7800997D5944C829A8BFC82121EAE1719975EE
:102B8800112008F0B9FDBAF1110F00F0FB80D9F857
:102B9800F4301A78022A20D107EE90BA1FED880A7D
:102BA800B8EEE78A88EE008A93ED0E0A38EE000A3E
:102BB800B5EEC00AF1EE10FA09D45FED8E7AB4EEE4
:102BC800670AF1EE10FAC8BFB0EE670A01E01FED20
:102BD800920A83ED0E0A14208EE0597D5944C829C3
:102BE800A8BFC82121EAE171597514205CE0D9F821
:102BF800F4301A78022A20D107EE90BAB8EEE78AA4
:102C0800B2EE040A88EE008A93ED0A0A38EE000A4A
:102C1800B5EEC00AF1EE10FA09D45FEDA67AB4EE6B
:102C2800670AF1EE10FAC8BFB0EE670A01E01FEDBF
:102C3800AA0A83ED0A0A09205EE0D9785944C8290E
:102C4800A8BFC82121EAE171D97009202CE0D9F880
:102C5800F4301A78022A1ED107EE90BAB8EEE78A45
:102C68005FEDB87A93ED0D0A88EE278A38EE000AF0
:102C7800B5EEC00AF1EE10FA07D4B4EE670AF1EE29
:102C880010FAC8BFB0EE670A01E01FEDC10A83ED74
:102C98000D0A0A2030E0597B5944C829A8BFC82129
:102CA80021EAE17159730A2008F026FD6AE0D9F893
:102CB800F4301A78022A22D107EE90BA1FEDD00A12
:102CC800B8EEE78A88EE008A93ED100A38EE000A1B
:102CD800B5EEC00AF1EE10FA09D45FEDD67AB4EE7B
:102CE800670AF1EE10FAC8BFB0EE670A01E01FEDFF
:102CF800DA0A83ED100A0B2008F0E8FC42E0D97DDF
:102D08005944C829A8BFC82121EAE171D9750B2007
:102D1800CAE7012936D19878B84B33F91230B3F5A0
:102D2800617F05DB40F633029342A8BF134601E0FA
:102D38004FF46173BAF10C0F24D14FF4966292FBF1
:102D4800F0F0AF4AA3F5617393FBF0F35FFA83F9F0
:102D580013784B4516D0B9F1040F34BF4B46022304
:102D68001370A84A0AFB035303F2B27313600EF000
:102D780023F95046494608F0BFFC09F10100C0B2EA
:102D880008F002FD019A0123934094F8EC201343C4
:102D980084F8EC30019B01330193029B0C330293BE
:102DA800019B042B7FF400ADB4E4D8F80030D805BB
:102DB80010D5954BDB786BB1336899070AD5BAF80B
:102DC800003013F0010B0AD10FF052FE012006F07B
:102DD80031FE04E0012006F01CFE012300E0002380
:102DE800D9F8002052070DD563B1012006F011FE75
:102DF800BAF800309B0708D40FF03AFE022006F01C
:102E080019FE02E0022006F004FEBAF800307F4AFC
:102E180013F0030F4FF020010CBF91611185326848
:102E280012F00A0F27D0D9F80020D00609D5590783
:102E38000AD4042006F0FEFD754B1B88A4F8F83070
:102E480002E0042006F0E5FDD9F800309A0607D51F
:102E5800BAF800305B0606D4402006F0EBFD02E02D
:102E6800402006F0D6FDD9F80030580642BF684B1E
:102E78001B88A4F8FA303368990609D4D9F80030C9
:102E88001A0540F191804FF4807006F0D3FD8FE071
:102E9800604B1B789B0753D55F4B1B78042B4FD98E
:102EA800D9F8003013F4007B0FD0BAF80030DE06F2
:102EB8003AD4102006F0BEFD202006F0AAFD57489F
:102EC800011D04F09BFC02232AE0BAF8006006F01A
:102ED8001006B6B22EB1102006F09BFD012684F82C
:102EE800FCB0D9F80030580512D5D4F800314C4957
:102EF8005A89B1F90030002BB8BF5B42934207DA18
:102F0800B1F90230002BB8BF5B429342C0F2058191
:102F1800BAF80030990608D5202006F07AFD00237B
:102F280084F8FC30012600E0002694F80431BBB98F
:102F38000E2008F007FC3B4B012283F804210FE028
:102F4800BAF8003003F03003002B97D0102006F0B9
:102F580060FD202006F05DFD002384F8FC3001E0D0
:102F6800002E8BD0304B002003F1280603F15004CB
:102F78002E4A002122F810102D4A596022F810100C
:102F88000432716022F8101000221A609A603260D0
:102F9800B26022606160A2601433143614340028D1
:102FA8007FF46CAF0120E3E74FF4807006F031FD49
:102FB8006B79082B01D00E2B02D1402006F029FD99
:102FC800D8F800305A0540F1BE8095F818321BB980
:102FD8003B7813F0040F03E0D9F8003013F4002F06
:102FE8002AD0144B00221A703C200DF08BFB0028CD
:102FF80000F0A9800DF0D6FCF6E700BF942E002063
:10300800502B0020C8110020DC2E002000040048AE
:1030180040120020441A00204A1A0020D011002033
:1030280048120020900E0020980F0020E22F002068
:1030380010100020192B002008F0D6FF09B0BDECB5
:10304800028BBDE8F04F0DF076BA012000E00220B7
:103058005FFA80F909F1FF3385F8B03706F02CFDE7
:1030680006F0CAFD484608F08FFBFFF7F9BABAF137
:10307800000F02D07E2B3FF4F1AA972B05D1344BD9
:103088004FF4C8721A80FFF7EBBAA72B06D1314A62
:10309800137843F004031370FFF7E2BA0022BB2B46
:1030A800079201D1022303E0B72B04D14FF6FE7338
:1030B800ADF81E3009E0BE2B01D1022303E0BD2B81
:1030C8001AD14FF6FE73ADF81C30DBF80030BDF8AE
:1030D8001C10B3F858200A44A3F85820BDF81E1055
:1030E800B3F85A200A44A3F85A2006F03FFF0023F9
:1030F80084F8BA30FFF7B4BA792B04D1164AD378DA
:1031080023F0010306E07A2B7FF4AAAA124AD378A7
:1031180043F00103D370FFF7A3BABAF800309B0657
:103128003FF503AF202006F085FC0C480C4B011D31
:103138001A685B684360026004F060FB094B012673
:1031480083F8FC60F1E609B0BDEC028BBDE8F08FB6
:10315800BC280020441A002048210020D811002053
:103168004C1A0020900E00202DE9F04FC14BB3F906
:103178000610C14B2DED028B1F687A8985B09142EC
:1031880001930EDBB1F5FA6FFC79BDBF8B1A63436F
:10319800A2F5FA64C4F16404BCBF93FBF4F464348C
:1031A80000E06424B54BB64AB3F898B193F962319C
:1031B800126802929BB2154603930022AD4B33F975
:1031C80012E0CBEB0E0303F2F31640F2E630864230
:1031D8004FEA420C03D8002BB8BF5B4201E04FF422
:1031E800FA73022A2ED0029E96F811611EB1B342DC
:1031F800CCBF9B1B0023A34E6FF0630A642093FB94
:10320800F0F836F818900AFB083A08F1010836F980
:1032180018600FFA89F8C8EB060606FB0AF696FB53
:10322800F0F699484E4420F80C60BE1864203679B0
:103238007343964E93FBF6F364339BB2634393FB5D
:10324800F0F02DE0029890F812611EB1B342CCBFA5
:103258009B1B0023DFF860926FF06308642093FBE8
:10326800F0F008FB003A39F910600130002B39F909
:103278001000A0EB060000FB0AFABDF80C009AFB50
:10328800F8FAC6EB0A0A1AFB00FA7F48A0F804A06D
:10329800B879B8BF5B4243437C4893FBF0F0643095
:1032A8006B787B4E4FF06408434393FBF8F3B354B9
:1032B800784EEB7A434393FBF8F3B3546B7D724E2D
:1032C8005843754B90FBF8F0022A9854734B0ED173
:1032D800DE4583F802800DDB684CB4F89A219142F0
:1032E80014DBB1F5FA6FA8BF4FF4FA610FE0DE45C1
:1032F8009C5404DA36F80C305B4226F80C30013264
:10330800032A05F101057FF459AFE5E71146DFF817
:10331800BCE15D4D891A4FF47A736FF06307594326
:10332800C2F5FA626423B1FBF2F191FBF3F23EF8C5
:10333800120007FB0211013207B23EF91220D21B1C
:10334800514391FBF3F30344F380554B1B885F060D
:1033580035D5544B544A1B881288DFED547A9B1A92
:103368001BB208EE103AB8EEC88A28EE278AB0EEEB
:10337800480A06F0ABFAF0EE408AB0EE480A06F0CA
:1033880042FAB5F9023006EE903AB5F90030F8EE97
:10339800E66A07EE903A20EE667AF8EEE77AA7EE4C
:1033A800A87A67EE807ABDEEC77AE6EEA87A17EEBD
:1033B800103AFDEEE77A2B8017EE903A6B803C4D81
:1033C8002B68980740F1A1803A4B3B4F1A687B69FC
:1033D80045F20721D31A8B4240F397807A6105F0B2
:1033E80085F9364BDFF8E8901A78032A9846B9F839
:1033F800003022D10A2B2AD90023282088F800304F
:1034080008F001FA05F072F92D4B188805F058F903
:103418002C4B1A68D37890FBF3F0013008282A4B1C
:10342800A8BF08201870537980B213FB00F33B83C0
:10343800137913FB00F0788309E00A2B07D80323DC
:10344800214A88F80030002313703B837B8398F867
:1034580000301A4A012B3DD002D3022B4CD054E045
:103468003A8BB9F800309A424FDD012388F80030D2
:1034780040E000BF942E0020C81100205012002008
:10348800A4110020361F0020481200200CFEFFFF68
:10349800C41E002026100020C71E0020B8270020C8
:1034A800081B0020401200208A0F002035FA8E3CAD
:1034B800582E0020C82F002018100020901A002035
:1034C800DC1D00202C1A0020FC0000201E1F0020FC
:1034D800301A0020B9F800107B8B8B4202DD0223E2
:1034E80013700FE09D4B1B8B0133994202DD0023C3
:1034F80013700AE0082006E07B8BB9F8002001333E
:103508009A42B2DC072008F01DF92D68290577D505
:10351800934B924F1A68FB69C3EB020845F20723E5
:1035280098456DDD8F4BB6F906B0D3F80090FA6177
:1035380099F80A30B4F852118B4E012B4FF47A7077
:10354800ABF57A7B98FBF0F803D042D3022B20D05E
:1035580041E0864B396A5A7B854B33F812204FF08D
:10356800080E92B291FBFEF3C91A8B18BA843B621B
:1035780040F6E44293FBFEF39BB25343B9F80820AC
:10358800C2EB13335843B9F9063090FBF3F03060BF
:1035980021E0784BB9F808A01B78C6F800A05A07B4
:1035A80019D5754808F077F820B915F0100F18BF2D
:1035B8004FF0000B32220BFB0BF393FBF2F3B9F93C
:1035C80006205B445A434FF47A7392FBF3F3534457
:1035D80000E000233360D7E90A013368674A03FB38
:1035E80008F84FF47A7398FBF3F810EB080041EBF6
:1035F800E8710023C7E90A010FF088FB604B1860E7
:10360800604E3368DB0427D52F0622D55E4B1B7826
:103618009D071ED55D4B187804281AD900225C4BEB
:10362800D7180521951C4FF00A0E122AD154E9B279
:1036380087F801E004D0B0EB510F2A46EFD800E03C
:1036480014215A18322002F8010CFF225A540F2074
:1036580000E00A2008F076F84E4D2A68002A44D087
:103668004D4B4E4F18683968814298463DD84C4BAF
:10367800DFF8389118785168B0B901221A70B9F892
:103688000030CB5CD3B1474B1A700FF0FFFAB9F892
:1036980000309BB92B681B78053B012B0ED808F02E
:1036A8008BF8414B186009E000221A70B9F8003015
:1036B800CB5C1BB13B4B1A700FF0E8FA2A68B9F8DB
:1036C800003052683948D25CFE2A01D100230BE051
:1036D800FF2A02D108F024F807E0D8F800500A21A0
:1036E80011FB02523A6001330380224D2B785807B0
:1036F80003D52F4B10221A8572E03268D1075CBFC0
:1037080043F001032B70204B1B781F075EBF2B78FB
:1037180023F001032B70D60248BF2B78214A44BFFF
:1037280023F001032B70234B1B6813F0040F02D006
:103738002149098851B92149098809B1980705D44F
:103748001F4B1B88003318BF0123DBB30223137000
:103758002B7823F001032B7039E000BF18100020EC
:10376800C82F00202C1A0020381A0020C41D002061
:10377800D41D0020EA2F0020DA130020407E050027
:103788003C1A002068110020441A00204A1A002020
:103798007C2B0020501F00207C2E0020481F00207A
:1037A800441F0020B82F0020382E00204C1F002076
:1037B80000040048401A0020E02F0020BC28002008
:1037C800E62F00202978C90758BF0223137007F095
:1037D800F3FFB34B1B68C01A002801DB0FF056FA41
:1037E80008F002FCAF4B1E789846002E00F0AA8025
:1037F800AD4E3368002B00F0DC86306808F093F992
:10380800002800F0D686A84BA84C186808F088F95C
:10381800092801D03F2850D14FF0000AD4F8009071
:10382800A34D5746B9F1000F05D0A24829684A466A
:1038380012F0E4FA10B9AA4607B92F469E4B103584
:103848009D42EFD3C7B1D7F800E0DAF800C023688B
:103858001EF803501CF80300A8420DD15A1C9549C4
:1038680038B92D2B05D8914D2A602025CD54885480
:1038780002E0CD542260EAE723680BB1574511D026
:103888008E480DF083F9574507D857F8100B0DF0FF
:103898007DF909200DF072F9F5E789480DF076F900
:1038A8004FF0000923689945A7D2824B13F8090005
:1038B8000DF064F909F10109F4E72368002B40F0E1
:1038C8005C86042840F09E867A4809F0B1F900F039
:1038D80070BED9F80000DFF8F8A108F024F938B371
:1038E800DAF8000008F01CF9DBF8003093F848100B
:1038F8000246002934D124286BD1012283F84820BC
:10390800DBF80030DFF8C4A193F84820062AE0D19C
:1039180093F8490001F000FC8346002800F08380FA
:103928003B6898790DF07BF83B68002283F84820C3
:10393800644B93F83530002B40F00D864C36982EAA
:1039480000F03786604BF21892F84A100129F5D139
:103958005E4FF3583A605E4ABB4613609146B8E73B
:10396800012904D14D2814BF00220222C6E70229EA
:1039780004D13C2814BF00220322BFE703290CD13D
:1039880040284FF0000102D983F84810B8E7587171
:103998001971D97198710422B0E7042906D199796F
:1039A80083F849004A409A710522A7E70529A7D15B
:1039B800587919798842987906D950409871481CE5
:1039C80018710B441A729BE790420CBF0622002222
:1039D80094E72B783F49580792D4232ADAF8003025
:1039E80014D1012088F800002F480391036035485E
:1039F8000292036338480DF0C9F831480DF0C6F853
:103A08000399029A0B7843F002030B70334B1B683F
:103A18001B78934201BF324B324A1A60324B04BFC3
:103A2800324ADA606CE7DAF8002092F849304C2B19
:103A380000F0988400F28780332B00F0CE8421D8E0
:103A4800292B00F05B8409D8252B00F01584272B3F
:103A580000F01984232B40F0D1853BE22D2B00F098
:103A68005E8407D82B2B40F0C9850CF0BBFF607132
:103A780000F06CBD2F2B00F01C85312B00F02E853B
:103A880000F0BCBD3E2B00F01B8146D8372B00F060
:103A9800D8842DD8352B00F0718200F0AFBD00BF5F
:103AA800BC2F0020EB2F00206C2B0020842100204D
:103AB8008C870108542100203C8901089EA7010831
:103AC800A3A7010818100020782A0020E81A00206F
:103AD800EC1A0020EA2F0020D3A701081C2B002095
:103AE800FC9F0020EFBEADDE00ED00E00400FA050B
:103AF800392B00F0D5833C2B40F08085DFF84C94BF
:103B0800D9F800A00CF06EFF8AF80000D9F8003050
:103B180018780BF08FFE00F019BD432B00F06E846F
:103B280006D8412B40F06A854FF0000900F05ABCD6
:103B3800442B00F007854A2B40F060850CF05CFFB1
:103B4800A08100F003BDD02B00F00F8355D8CA2BFD
:103B580000F0C08009D8C82B00F0858000F22683C9
:103B68004E2B00F00C8400F049BDCD2B00F00883EB
:103B780004D8CC2B00F02A8200F040BDCE2B00F0F8
:103B88000883CF2B40F03A850CF036FF6FF4AF6214
:103B980083189BB2C62B98BFA4F898010CF02CFF91
:103BA800A4F844010CF028FFA4F846010CF024FF07
:103BB800A4F848010CF020FFA4F8DA010CF012FF79
:103BC80084F8EF010CF00EFF0CF00CFF84F8F00104
:103BD8000CF008FF84F887010CF004FF84F89401C6
:103BE8000CF000FFD94BD3F800900CF005FF00EB68
:103BF80080004000A9F8560052E3D62B00F0398225
:103C08000AD8D22B19D0C0F0F882D32B25D0D42BC8
:103C180000F03B8200F0F2BCEF2B41D005D8D82B46
:103C280040F0EC844FF0000AE6E0F22B00F07582D9
:103C3800FA2B00F0B78200F0E1BC2B78590700F1AD
:103C480085840CF0CFFE022884F8B00740F29382F6
:103C5800BF4B002283F8B0278DE20CF0CDFEBD4BA0
:103C6800188000F073BC92F805904FEA5909B9F131
:103C7800120F03D90CF042FD00F068BC4FF0000AA7
:103C8800CA4507D20CF0B8FEB34B23F81A000AF164
:103C9800010AF5E7B14B012283F8342000F056BC45
:103CA800DFF8A892D9F800A00CF0A6FEAAF85A00EE
:103CB800D9F800900CF0A0FEA9F8580000F046BC16
:103CC8000CF090FE84F8E2010CF08CFE84F8E1011F
:103CD80000F03CBC9D4B1A681278022A824699462D
:103CE8006FD1D9F800B00CF07DFE07EE900AF8EE1F
:103CF800677AB2EE048AC7EE887A0BEB8A0BCBEDB3
:103D0800087AD9F800B00CF06DFE07EE900A9FED26
:103D1800947AF8EE677A0BEB8A0BC7EE877ACBEDCD
:103D28000B7AD9F800B00CF05DFE07EE900A9FED13
:103D38008D7AF8EE677A0BEB8A0BC7EE877A0AF171
:103D4800010ABAF1030FCBED0E7ACAD1BAF1070F07
:103D5800D9F800B01CD10CF045FE07EE900AF8EE39
:103D6800677AC7EE887ACBED117AD9F800B00CF0F3
:103D780039FE07EE900AF8EE677AC7EE887ACBED3F
:103D8800127AD9F800B00CF02DFE8BF84C0012E036
:103D98000CF028FED3448BF80100D9F800B00CF0E1
:103DA80021FED3448BF80B00D9F800B00CF01AFEB2
:103DB800D3448BF815000AF1010ABAF10A0FC5D1EC
:103DC800C4E3D9F800B00CF00DFED3448BF8010021
:103DD800D9F800B00CF006FED3448BF80B00D9F8E4
:103DE80000B00CF0FFFDD3440AF1010ABAF10A0F42
:103DF8008BF81500E5D1A9E3DFF850919FED598ABA
:103E0800D9F800B00CF0F8FD07EE900AF8EE677AE2
:103E18000BEB8A0BC7EE887ACBED087AD9F800B09D
:103E28000CF0EAFD07EE900AF8EE677A0BEB8A0BC6
:103E3800C7EE887ACBED0B7AD9F800B00CF0DCFD30
:103E480007EE900AF8EE677A0BEB8A0BC7EE887AD2
:103E58000AF1010ABAF1030FCBED0E7ACCD1BAF10F
:103E6800070FD9F800B01CD10CF0C6FD07EE900A78
:103E7800F8EE677AC7EE887ACBED117AD9F800B0F8
:103E88000CF0BAFD07EE900AF8EE677AC7EE887A6A
:103E9800CBED127AD9F800B00CF0AEFD8BF84C00DF
:103EA80012E00CF0A9FDD3448BF80100D9F800B05A
:103EB8000CF0A2FDD3448BF80B00D9F800B00CF03D
:103EC8009BFDD3448BF815000AF1010ABAF10A0FD9
:103ED800C5D13BE30CF086FD132883463FF6CAAEF6
:103EE800DFF868A0DAF800900CF07CFD00231E4A89
:103EF8000C2101FB0322117A814222D10FFA8BFB9C
:103F080009EB8B09137889F879300CF06BFD89F887
:103F18007A000CF067FD89F87B000CF063FD134B09
:103F2800134A1A6089F87C00124BDAF8000018600E
:103F38000021793007F09EFB0F4B80F001001870CC
:103F480004E301331C2BD2D194E600BFA411002056
:103F580050120020880F0020942E002018100020F6
:103F68000000C84200007A44A4850108800F0020A0
:103F780094130020840F0020030000200CF032FD71
:103F88000B2882463FF676AECE4BD3F800900CF065
:103F980029FD03283FF66EAE062303FB0A9989F82C
:103FA800CE000CF01FFD89F8C9000CF01BFD89F844
:103FB800CA000CF017FD89F8CB000CF013FD89F846
:103FC800CC000CF00FFD89F8CD00BFE25379092B26
:103FD8007FF650AE019BD3F800900CF003FD019BD7
:103FE80089F80000D3F800900CF0FCFC89F8010077
:103FF8000CF0F8FC019B64281B68A8BF64201871AA
:104008000CF0F0FC019B64281B68A8BF6420587161
:104018000CF0E8FC019BFF281B68A8BFFF209871E3
:104028000CF0E0FC019B6428D3F8009028BF6420C2
:1040380089F807000CF0D6FC019B89F80200D3F838
:1040480000900CF0CFFC019B89F80300D3F8009096
:104058000CF0D2FC3B68A9F80A005B790A2B40F205
:104068007582994BD3F800900CF0BCFC89F80800D5
:104078006CE282460CF0C0FC944B23F81A000AF15B
:10408800010ABAF1080FF5D160E253790F2B7FF4DA
:10409800F1AD0CF0A7FC072881463FF6EBADDFF841
:1040A80024A2DAF800B00CF0A7FC0E2303FB09F9F0
:1040B800CB44ABF81901DAF800B00CF09DFCCB4406
:1040C800ABF81B01DAF800B00CF096FCCB44ABF867
:1040D8001D01DAF800B00CF085FCCB448BF81F0109
:1040E800DAF800B00CF07EFCCB448BF82001DAF84B
:1040F80000B00CF077FCCB448BF82101DAF800B063
:104108000CF070FCCB44DAF800A08BF822010CF01C
:104118007DFCD144C9F8230118E20CF063FC0F2898
:1041280081463FF6A7AD0CF05DFCC9EBC909A14477
:1041380089F8D4000CF056FC89F8D5000CF052FC34
:1041480089F8D6000CF04EFC89F8D7000CF04AFC30
:1041580089F8D8000CF046FC89F8D9000CF042FC2C
:1041680089F8DA0007F080FEF0E12B785B0700F1B0
:10417800ED810CF069FF05F09FFC05F03DFDE5E1E0
:104188002B78580700F1E281514B4FF4C8721A801E
:10419800DCE12B78590700F1D9814E4A137843F0B6
:1041A800040328E02B785A07E5D527E20CF01AFC1F
:1041B800484B1A7810B142F0020201E022F00202E4
:1041C8001A700CF00FFC444BDFF82C9118700CF0AF
:1041D8001DFCC9F800000CF019FCC9F804000CF02B
:1041E8000BFC3E4B18800CF007FC3D4B3D4A1880F9
:1041F800137843F002031370A8E10CF0F3FB02906C
:104208000CF004FC83460CF001FC82460CF0FEFB2B
:1042180081460CF0F1FB0CF0EFFB0CF0E3FB029B8A
:10422800A3B9314B1020C3F800B0C3F804A005F0BF
:10423800F0FB284A137843F001031370B9F1000F1B
:1042480000F08481294BC3F800907FE1102B40F0E7
:104258007D81274BC3F800B0C3F804A0B9F1000F63
:1042680002D0224BC3F800902148224B0222011DA4
:104278001A7003F0C3FA69E1A0600CF0C7FBA368E9
:104288001843A06062E10CF0B7FBA4F85C010CF0E5
:10429800B3FBA4F85E010CF0AFFBA4F8600155E194
:1042A8000CF0A0FB84F87C010CF09CFB84F88001E6
:1042B8000CF098FB84F87F010CF094FB84F88101E2
:1042C80044E100BFA4110020C8110020522B002097
:1042D800BC280020441A00204A1A0020481A00204E
:1042E800461A0020CE110020D0110020E011002035
:1042F800D81100208C0F00204C1A00200CF07CFBF9
:10430800A4F882010CF078FBA4F884010CF06AFB95
:1043180084F886010CF070FBA4F8880116E10CF013
:1043280061FB84F892010CF067FBA4F89C010CF087
:1043380063FBA4F898010CF05FFBA4F89A010CF059
:1043480051FBDAF8003084F893015B79082B40F2CE
:10435800FD800CF051FBA4F89E010CF04DFBA4F875
:10436800A001F3E00CF03EFB84F8D8010CF03AFB16
:1043780084F8D9010CF040FBA4F8DA01E6E092F8E1
:1043880005900323B9FBF3F9B9F1120F3FF672ACAC
:10439800DFF888A34FF0000BCB4580F0D7800CF0F6
:1043A80021FB8AF8A2010CF027FB40F2ED2398428A
:1043B80005DD40F6CA039842A8BF184601E040F25E
:1043C800EE20A0F2EE2019230BF1010B90FBF3F085
:1043D8000AF1020A8AF8A101DEE70CF003FB84F86F
:1043E8009401B3E00CF0FEFA04EB090309F10109AA
:1043F800B9F1080F83F88A01F4D1A7E00CF0F2FABA
:10440800C4F808B060710CF001FBA3681843A06001
:104418000CF0E8FA84F892010CF0EEFAA4F85C01CA
:104428000CF0EAFAA4F85E010CF0E6FAA4F86001D0
:104438000CF0E2FAA4F882010CF0DEFAA4F8840188
:1044480084E053794FF0070AB3FBFAF2C2EBC202D9
:104458009A1A12F0FF0F7FF40DACB3FBFAFA0AF1C7
:10446800FF3A5FFA8AFABAF1FF0F6FD00CF0BAFA86
:104478005FFA80FB4FFA8BF007F034F8814600288A
:104488003FF4F8AB80F800B00CF0B6FAA9F80200D7
:104498000CF0A8FA89F804000CF0A4FA89F80500D1
:1044A8000CF0A0FA89F807000CF09CFA89F80600CD
:1044B800D5E7DFF8689209F1400A0CF09DFAA9F8EF
:1044C800A8020CF08FFA89F8AA020CF08BFA09F10D
:1044D800040989F8A702D145EFD137E00CF082FA38
:1044E8001F2881463FF6C6AB3B685B79082B7FF4F3
:1044F800C1AB0CF081FA09F18A0904EB890A00F0D2
:104508003F00AAF802000CF077FABAF802308001EE
:1045180000F4FE501843AAF802000CF063FA0001F8
:1045280004F829000CF05EFA14F8293000F00F00A6
:10453800184304F829000CF055FA8AF801000BF02A
:104548000DFA03E0624B012283F8352000200CF0BD
:1045580095FAFFF7E5B95F4B985907F0DBFA18B9F8
:10456800322007F050F9F6E707F03EFC05F07AFA3A
:10457800594B5A4ADA60FFF7E1B90C2844D00A28A7
:104588004BD1574D57480CF001FB2846232111F019
:104598001EFC08B1401B20602368002B60D15048E6
:1045A80023600021302211F0DCFB98F80030002B4A
:1045B8002DD14D4B1B689B0615D54C4B44491B68A8
:1045C8008A6B9A1A002A0EDB494A1278042A0AD9F9
:1045D800484A03F5123303F5F8738B63938A9BB249
:1045E80083F020039382444B9B68002B6BD0434895
:1045F80005B0BDEC028BBDE8F04F18470CF07EF813
:10460800FFF78EB90C2804D13D480CF0BFFA3D489D
:104618000DE07F2812D1FFF7F0B80D28B1D07F2820
:1046280009D1013B2E4A384823600021D1540CF0AF
:10463800ADFAFFF7E2B82F2B3FF6DFA8A0F1200272
:10464800D2B25E2A3FF6D9A813B920283FF4D5A8DC
:104658005A1C2260224AD0540CF090FAFFF7CDB8C9
:104668005A1EA95C202901D1134696E71C4A2360EB
:104678000021D154254B264DD3F800A0D5F800B021
:10468800DFF85C90584611F0B0FB07463A464846BA
:10469800594611F0B3FB1F4A28B919F8073053449B
:1046A8005B785B0703D010359542E7D306E0954267
:1046B80004D2781CEB684844984702E016480CF08E
:1046C80065FA00236BE705B0BDEC028BBDE8F08FFF
:1046D80018100020782A002000ED00E00400FA05F8
:1046E800542100207AB40108401A0020C82F002065
:1046F8004A1A0020000400484C28002054100020CA
:10470800A8A70108A3A70108CFA701080C0100204A
:104718008C8701083C890108B3A7010850120020C2
:1047280010F80A3C0133DBB20A2B84BF10F8131CC3
:10473800044A00F80A3C82BF002322F8113000F82E
:104748000A3C70474C2F0020354A70B5136C9068AE
:104758001944344B1B78D940081A40F68C239842E8
:104768009160D060516013463BD9127893F9451097
:104778008A4210460BD1111F082908D893F8461011
:10478800182901D8013103E083F8442002E0002110
:1047980083F8461093F944402149A24219D191F86F
:1047A8004740B4B10C310024944206DA1E4D51F84A
:1047B800046F25F814600134F6E70C2805D01A496F
:1047C800002421F810400130F7E71848017801313A
:1047D800017083F84520002201211A7083F84710E0
:1047E80070BD92F84710C9B1A0F2EF2440F2DA5137
:1047F8008C4208D811780B2905D80B1D013111708E
:1048080042F8230070BD002283F84720084B03F1CB
:104818003002002143F8041F9342FAD170BD00BF53
:10482800A00100209F0100204C2F00209C060020A2
:10483800AC010020024A136C01331944116470471B
:10484800A0010020024B53F820301B681960704704
:10485800941F0020064B53F820301A681B89A1F5D5
:104868007A7159434FF47A7391FBF3F111607047F1
:10487800941F0020054B98420CBF054A054A13882F
:1048880001339BB213800020704700BF00540040E2
:104898006411002066110020F0B5046D8668236855
:1048A80023F0010323608379054613F0020F407952
:1048B8000CBF4FF0000E4FF4005E13F0040F14BF4E
:1048C8004FF48067002710F0010F14BF0421002166
:1048D8008307206820F001002060626822F44052BB
:1048E8004EEA02026260226822F4B05323F00C03FD
:1048F80048BF41F008013B430B432360A36895B0D0
:1049080023F44073A360684603F06CFC284B9C4278
:1049180001D10C9B0EE0274B9C4201D10D9B09E075
:10492800254B9C4201D10E9B04E0244B9C420CBFBA
:104938000F9B109B2268A879170448BF5B00B3FB44
:10494800F6F206FB1233B3EB560F236828BF013289
:104958001E0441BF4FF6F073C2F34201134041EA0F
:1049680003026B7992B213F0020FA28100F00101E9
:1049780014BF4FF400320022DC0748BF42F48032F3
:104988002B6D11B159680A4302E0596821EA020205
:104998005A609A6801074CBF42F0080222F00802E8
:1049A8009A601A6842F001021A6015B0F0BD00BFA3
:1049B800003801400044004000480040004C0040DE
:1049C8003D4B1B78012B30B514BF00240324B1B92B
:1049D800036A23F0010303628169036A21F0F3018A
:1049E80023F00A0341F0010142F001021A4341EAAF
:1049F800041181610262836923F00C031BE004291E
:104A08001DD1016A4FF6EF730B4003628169056A95
:104A1800120121F473414FF65F7342F0100241F422
:104A280080712B4092B2134341EA043181610362E1
:104A3800836923F4406383618369836130BD0829F6
:104A4800016A1AD14FF6FF630B400362C169036A1A
:104A58009BB289B223F4206343F4807321F0F301FD
:104A680043EA022241F0010192B241EA0411C16114
:104A78000262C2694FF6F37319E04EF6FF730B40FA
:104A88000362C369056A40F6FF41194045F6FF73A2
:104A98002B4043F4805343EA023241F4807192B2CE
:104AA80041EA0431C1610262C2694FF2FF33134027
:104AB800C361C369C36130BD9C01002038B510F8DB
:104AC8000E2C50F8043C044652B9012200F80E2C72
:104AD80020F80C1C997A18680222BDE838406FE764
:104AE80030F80C2C20F80A1C891A89B220F8081C06
:104AF800074A10F80F0C002522F8101004F80E5C75
:104B08001868997A2A46FFF75BFF04F8065C38BDF7
:104B18004C2F0020044B53F820301BB107289CBFB2
:104B28001B681960704700BFC8020020084A136854
:104B38009B050BD5074B00211970074908684FF6EC
:104B4800FE7303400B604FF400735360704700BF5F
:104B580000000240E92F0020300002402DE9F04714
:104B6800664D2B6866490A78581C02F0FF068E4687
:104B78000AB10346F6E72B60687BAB6895F80C80B2
:104B8800AA7B374639B2202900F09B80DFF880C124
:104B98000CEB81033CF82110DC789B78C3F1FF0310
:104BA8009BB2002B65D0C3F1FF0363434FF03C0C6D
:104BB8001B12B1FBFCF9B9F1050F5DD8DFE809F06C
:104BC800030B1A293A4AE01ADAB24143B1FBFCF066
:104BD8001044C0B251E0B1FBFCF00CFB101189B2DB
:104BE800DAB2C1F13C01E31A4B432046B3FBFCFCAB
:104BF80094442CE0B1FBFCF00CFB10115FFA83F835
:104C0800E21A89B24A43B2FBFCF24244D2B22046CD
:104C180032E0B1FBFCF90CFB191189B25FFA83F899
:104C2800E01AC1F13C014843B0FBFCF04044C0B27B
:104C3800224621E0B1FBFCF80CFB1811D8B289B26E
:104C4800E31A01FB03F2B2FBFCFC224684445FFA40
:104C58008CF412E0B1FBFCF80CFB181189B2D8B245
:104C6800C1F13C01E31A4B43B3FBFCF20244D2B25C
:104C780003E02246204600E044464FEA042C4CEA72
:104C8800004C4CEA020C172306F117014FF00108FB
:104C980008FA03F8C91A18EA0C0F89B2DFF8748009
:104CA80014BF4FF011094FF0090913F1FF3308F849
:104CB8000190E9D218360137B6B2BFB2114BA046FF
:104CC80060E7AA73AB60104AE98001238EF80030D0
:104CD8000E4985F80C8040F22A336873AE80536021
:104CE80000234B620B889BB243F001030B801368CF
:104CF80043F001031360BDE8F08700BF581000209F
:104D0800E92F0020641000203000024000440140D8
:104D18000A0E00204503002073B506460D46002400
:104D280001232A88A34013421AD0AA78009302F0DC
:104D380003038DF80430EB78022B03D0032B0CBF50
:104D4800032301238DF805303046C2F30113694669
:104D5800C2F381028DF806308DF8072003F0B0FB0E
:104D68000134102CDCD102B070BD2DE9F04F734E28
:104D7800F57B07460C4687B011469A4600686B1CBF
:104D8800914622464FF0020BF3730CF021FF3B894A
:104D98007868ADF8043001A98DF806B08DF807B031
:104DA800FFF7BAFF0023ADF80A30ADF81230ADF8BE
:104DB800163070230193BA7A3C68CDF80CA0012311
:104DC80006F110082D01ADF808304FF48073A8449F
:104DD800ADF810B0ADF814300C2A7ED8DFE802F038
:104DE800077D7D7D0F7D7D7D387D7D7D5E00204644
:104DF80001A903F0B9F9A36943F0080326E0236A7F
:104E08004F4823F010032362236A6168A26922F0E5
:104E1800807222F4E642844242F4E04206D000F571
:104E28000060844202D043F0300307E023F0E0033F
:104E380021F4406143F0300341F480616160A26174
:104E4800C4F838A02362A36943F40063A36144E073
:104E5800236A3B4823F480732362226A6168E3690A
:104E6800844223F0730343F0700306D000F500601A
:104E7800844202D042F4407207E022F4606221F4D6
:104E8800405142F4407241F480516160E361C4F8DA
:104E98003CA02262E36943F008031DE0236A284826
:104EA80023F480532362226A6168E369844223F40D
:104EB800E64343F4E04342F4405203D000F5006077
:104EC800844201D141F480416160E361C4F840A0AB
:104ED8002262E36943F40063E3613A7B3B681AB1F9
:104EE8005A6C42F400425A641A8892B242F00102A3
:104EF8001A80BA7A0C2A18D8DFE802F007171717B1
:104F08000B1717170F1717171300721903F134012E
:104F18000AE0721903F1380106E0721903F13C0145
:104F280002E0721903F14001116135444046A5F8C9
:104F380018906B6107B0BDE8F08F00BF58100020D3
:104F4800002C0140F8B53A4E3A4C4000C7B24FF435
:104F580020453068C4F8D050D0F818E01EF4004F4F
:104F680005D0AE46013DBEF1000FF5D116E0D0F8F0
:104F780004E0314D0EEA050545F490353D434560A2
:104F88004FF42045C4F8D050D0F818E01EF0020FB6
:104F98002DD1AE46013DBEF1000FF5D1C4F8D05079
:104FA8001FE02946013D0029F8D081694906F8D556
:104FB800C4F8D05020494568294041F0007141F4B7
:104FC800105141EA0241394341604FF42041A2B1F6
:104FD800306885696D071ED411F1FF31F9D2C4F824
:104FE800D010FFF747FC003018BF0120F8BD4FF480
:104FF80020458162C4F8D050D7E73068C4F8D01093
:105008000B46826992060CD41A46013B002AF8D155
:10501800C4F8D030E5E7416A03F8011B013AD2B27F
:10502800D3E7C4F8D0302023C3610120F8BD00BF06
:105038006011002058100020009800FC400070B556
:10504800C5B23248324B00684FF42044C3F8D04010
:105058008669360404D52646013C002EF8D113E0B3
:1050680046682C4C344044F0807444F490342C430B
:1050780044604FF42044C3F8D0408669B60729D469
:105088002646013C002EF8D1C3F8D0401CE021464A
:10509800013C0029F8D081690E06F8D544681D49FD
:1050A800214041F0007141F48031294341604FF4BF
:1050B8002041C3F8D0108469A40711D40C460139E3
:1050C800002CF8D1C3F8D010FFF7D4FB003018BF7C
:1050D800012070BD4FF420448162C3F8D040DAE764
:1050E80082624FF42042C3F8D0208169890606D431
:1050F8001146013A0029F8D1C3F8D020E4E7C3F8F3
:10510800D0202023C361012070BD00BF60110020A2
:1051180058100020009800FC2DE9F0474D282DED8F
:10512800028B044600F05E8600F2B980302800F059
:10513800D98651D8222800F09D8423D8032800F06E
:105148000B8214D8012800F0FB81022840F0028766
:1051580004200BF093FC43200BF061FC4C200BF077
:105168005EFC46200BF05BFC4C2000F061BE04287E
:1051780000F0FB81052840F0ED861A200BF07EFC3C
:10518800002402E2282800F0EC8515D8242800F035
:10519800D385262840F0DE86D14C06200BF06EFC25
:1051A800B4F85C010BF06DFCB4F85E010BF069FC1F
:1051B800B4F8600100F0BDBD2C2800F0E5852E286C
:1051C80000F060862A2840F0C58601200BF056FCC6
:1051D800C34B587900F02CBE3D2800F0FD821ED844
:1051E800362800F036860BD8322800F01B86342883
:1051F80040F0B08648200BF041FC002500F05CBC74
:105208003A2800F0C0823B2800F02D84382840F06E
:10521800A18604200BF032FCB14C00F093BD452868
:1052280000F0858627D8402800F00586422840F0FF
:105238009186AB4C10200BF021FC60790BF0EFFB52
:10524800A0680BF027FC94F892010BF0E8FBB4F887
:105258005C010BF016FCB4F85E010BF012FCB4F81C
:1052680060010BF00EFCB4F882010BF00AFCB4F8F4
:10527800840100F05EBD492800F0B9824B2800F097
:10528800A285462840F066860D200BF0F7FB00202B
:105298000BF0C5FB00200BF0FDFB00F053BE70289F
:1052A80000F0F68200F2E580692800F04C8200F2F6
:1052B800B680662800F0A68100F2A680642800F077
:1052C8007D81652840F04686864C0B200BF0D6FB86
:1052D80020880BF0D6FB6268834B9A420CBF20896A
:1052E800608980B20BF0CDFB804B1B68C3F3C00014
:1052F800C3F38002800040EA4200C3F34002104337
:10530800C3F3401240EAC20003F0100318430BF045
:10531800B8FB774B1A88E368247C02F0080103F491
:10532800475949EA010903F4804149EA010903F4AC
:10533800004149EA010903F4803149EA010903F40B
:10534800003149EA010903F4802149EA010903F41B
:10535800002149EA010903F4801149EA010903F02F
:10536800007349EA0303DFF8A89199F8009012F056
:10537800010FC9F3800914BF4FF002084FF000086D
:1053880043EA090312F0020F43EA080314BF4FF07F
:10539800040C4FF0000C12F0040F43EA0C0C14BF7D
:1053A8004FF0100E4FF0000E12F0400F14BF2027E0
:1053B80000274CEA0E0E12F0100F14BF4FF40076BF
:1053C80000264EEA070712F0200F14BF4FF480653D
:1053D80000253E4312F4807F14BF4FF40060002084
:1053E800354312F4007F14BF4FF400110021284305
:1053F80012F4806F41EA000114BF4FF0806300236C
:10540800002019430346E9E0672800F02381682853
:1054180040F0A08510200BF031FB00248AE16C28B5
:1054280000F0A48117D86A2800F008846B2840F09F
:10543800918505200BF022FB2E4B18880BF021FBE1
:105448002D4B18880BF01DFB264B93F8720000F0CB
:10545800010000F0EDBC6E28224D00F0988100F2AA
:10546800EF8106200BF00AFB686E0BF013FB234B51
:1054780087E1782800F0FB8018D8742800F03D8375
:105488000AD8722800F09A83732840F063850820B0
:105498000BF0F4FA0124CAE3762800F0EF8300F257
:1054A8006D832F200BF0EAFA154CD4E2A42800F003
:1054B8000C842FD87B2800F07482A02840F04A85FD
:1054C8000C200BF0DBFA0F4B18680BF0E3FA0E4BCD
:1054D80018680BF0DFFA0D4B186800F037BD00BFF5
:1054E800501200205C11002000540040401A002097
:1054F800081B0020BE1A0020C01A00203812002005
:1055080073850108ACF7FF1FB0F7FF1FB4F7FF1F43
:10551800EA2F0020F12800F0E680FE2800F0FC8346
:10552800F02840F01785B54C04200BF0A7FAA36CBF
:10553800B3F85A000BF0A5FAA36CB3F85800F8E3D7
:1055480003200BF09BFA00200BF069FA20460BF0C1
:1055580066FA0D2000F06CBC0BF090FA01200BF0FD
:105568005EFA0A200BF05BFAADE306200BF086FA30
:1055780053200BF054FA50200BF051FA4B200BF04B
:105588004EFA59200BF04BFAD2E39D4B185D0134CB
:105598000BF045FA0B2CF8D100249A4B185D013416
:1055A8000BF03DFA082CF8D10024974B185D013414
:1055B8000BF035FA072CF8D100F0CABC07200BF025
:1055C8005DFAE7200BF02BFA904B58790BF027FA8D
:1055D80000200BF024FA042000F0B8BCA3420AD241
:1055E8008B4A9D5C012202FA05F50D421CBF9A40C8
:1055F80010430133F2E70BF04DFA844B93F8B007F0
:1056080000F016BC12200BF039FA824B1B88B3F558
:10561800806F8CBF0825012500247F4B33F91400C7
:1056280090FBF5F0013480B20BF02BFA032CF4D187
:10563800724CA08D0BF025FAE08D0BF022FA208E2B
:105648000BF01FFA608E0BF01CFAA08E0BF019FA03
:10565800E08E6EE310200BF011FA00246F4B185DFA
:1056680001340BF0DCF9102CF8D100F071BC70207B
:105678000BF004FA0026614D0E24AB6C74432344EE
:105688000136B3F819010BF0FCF9AB6C2344B3F8FD
:105698001B010BF0F6F9AB6C2344B3F81D010BF0BA
:1056A800F0F9AB6C234493F81F010BF0B8F9AB6C1D
:1056B800234493F820010BF0B2F9AB6C234493F820
:1056C80021010BF0ACF9AB6C234493F822010BF0E9
:1056D800A6F9AB6C1C44D4F823010BF0DBF9082EB7
:1056E800C9D100F035BC7020484C0BF0C7F904F163
:1056F800700594F8D4000BF092F994F8D5000BF0EB
:105708008EF994F8D6000BF08AF994F8D7000BF0CC
:1057180086F994F8D8000BF082F994F8D9000BF0C8
:105728007EF9073494F8D3000BF079F9AC42E0D154
:1057380000F00EBC3A4B185D01340BF070F9102CD8
:10574800F8D100F005BC374D2878400000F0FE0085
:105758000BF094F900242B789C4280F0F983324BAB
:1057680033F814000BF08DF90134F4E72F4C0620C0
:105778000BF084F920880BF084F960880BF081F92C
:105788002B4B1888D5E204200BF078F9DDE30720CD
:105798000BF074F9274B1888FF28A8BFFF20C0B268
:1057A8000BF03DF9244B186880F3100080B20BF021
:1057B80068F9B5F868000BF064F9144B93F8872181
:1057C8001E4B186822B10A23584380F3100001E0E9
:1057D80000F30F0080B2ACE20C4C02200BF04EF943
:1057E80094F8E2010BF01BF994F8E10120E30220A0
:1057F8000BF044F9054B98899BE200BF5C1100202F
:10580800D8A40108E4A40108B9A401085012002092
:105818006D11002004000020321200209411002095
:10582800A8110020142B0020942E00204E2E0020BA
:1058380040120020301A00203C1A0020381A00209C
:105848000B200BF01BF9EB6E18780BF0E8F8EB6EF9
:1058580058780BF0E4F80026EB6EC44C334401365C
:1058680018790BF0DCF8032EF6D1E36ED8790BF03B
:10587800D6F8E36E98780BF0D2F8E36ED8780BF090
:10588800CEF8E36E58890BF0FCF8E36E187ACFE295
:10589800B64C1E200BF0F2F8A36C1B78022B4FF0CD
:1058A80000056BD1A36C03EB850393ED080AB2EEF8
:1058B800048A20EE080A10F063FC80F30800C0B2E6
:1058C8000BF0ADF8A36CDFEDAA7A03EB850393ED3B
:1058D8000B0A20EE270A10F053FC80F30800C0B230
:1058E8000BF09DF8A36CDFEDA37A03EB850393ED32
:1058F8000E0A20EE270A10F043FC80F30800C0B21D
:1059080001350BF08CF8032DCCD1072DA36C23D1D6
:1059180093ED110A20EE080A10F032FC80F308001B
:10592800C0B20BF07CF8A36C93ED120A20EE080AC3
:1059380010F026FC80F30800C0B20BF070F8A36CDE
:1059480093F84C3000EE103AB8EE400A10F018FC0C
:1059580080F30800C0B20BE02B4458780BF05FF8D6
:10596800A36C2B44D87A0BF05AF8A36C2B44587DBF
:1059780001350BF054F80A2DC7D1E9E2A36C2B448A
:1059880058780BF04CF8A36C2B44D87A0BF047F8F6
:10599800A36C2B440135587D0BF041F80A2DEDD14D
:1059A800D6E23C200BF06AF80024704D9FED718A16
:1059B800AB6C03EB840393ED080A20EE080A10F0A1
:1059C800DFFB80B20BF05DF8AB6C03EB840393ED67
:1059D8000B0A20EE080A10F0D3FB80B20BF051F846
:1059E800AB6C03EB840393ED0E0A20EE080A10F06B
:1059F800C7FB013480B20BF044F8032CD5D1072C37
:105A0800AB6C16D193ED110A20EE080A10F0B8FB22
:105A180080B20BF036F8AB6C93ED120A20EE080A50
:105A280010F0AEFB80B20BF02CF8AB6C93F84C0086
:105A38000BE0234458780BF024F8AB6C2344D87A55
:105A48000BF01FF8AB6C2344587D01340BF019F8A8
:105A58000A2CD4D17CE214F8010F002800F07882D7
:105A68000AF0DDFFF7E701200BF008F83F4B9B6CCD
:105A78001878DDE150200BF001F800253B4B9C6CB9
:105A88003D4B04EB85040C2194F8792001FB02338B
:105A9800013593F838000AF0C2FF94F87A000AF04A
:105AA800BEFF94F87B000AF0BAFF94F87C000AF075
:105AB800B6FF142DE2D14BE22C4B9C6C062303FB62
:105AC8000544013594F8CE000AF0A9FF94F8C900FE
:105AD8000AF0A5FF94F8CA000AF0A1FF94F8CB00D9
:105AE8000AF09DFF94F8CC000AF099FF94F8CD00D5
:105AF8000AF095FF0C2DDFD12AE24FF000080126AD
:105B080000271A4B1A7C974227DA11330024FA5CD3
:105B1800194D0C2305F130016343595C914207D1BB
:105B28002B44586B10F061F982462EB9B14605E056
:105B380001341C2CECD10EE080440CE0D1450ADA8B
:105B48000C2303FB04535B6B13F809000AF067FF8F
:105B580009F10109F2E70137D3E7002E00F0F881D7
:105B68005FFA88F00AF08AFF0026C9E75C11002076
:105B78000000C84200007A4474850108CC4D287C96
:105B88000AF07CFF00242B7C9C4280F0E181C94B09
:105B9800E65C0021C8480C2200F1300702FB01F343
:105BA800DA5DB24205D1034493F838000AF037FFB2
:105BB80002E001311C29EDD10134E4E7BF4C162085
:105BC8000AF05CFFB4F898010AF05BFFB4F84401EE
:105BD8000AF057FFB4F846010AF053FFB4F8480139
:105BE8000AF04FFFB4F8DA010AF04BFF94F8EF011E
:105BF8000AF015FF00200AF012FF94F8F0010AF0ED
:105C08000EFF94F887010AF00AFF94F894010AF04D
:105C180006FF00200AF003FFA54B9B6C0A20B3F98E
:105C2800563093FBF0F080B20AF02BFF8AE0E0B226
:105C380001340AF0F4FE092CF9D189E110200AF0A8
:105C48001DFF9F4B9F4C187800F002000AF0E7FEFA
:105C58009D4B18780AF0E3FE20680AF01BFF606885
:105C68000AF018FF994B18880AF00BFF984B188810
:105C78000AF007FF8E4BB3F870005AE00AF0B2FE44
:105C8800074612200AF0FAFE894C17B9666FA56F0D
:105C980006E0102F13BF0025E66FD4F880502E467B
:105CA80038460AF0BCFE30460AF0F4FE28460AF0F0
:105CB800F1FED4F884000AF0EDFE00200AF0E1FEBF
:105CC80000200AF0DEFE0020B2E0794D95F8880049
:105CD80080000130C0B20AF0D1FE95F888000AF0C1
:105CE8009EFE00242E4696F888309C4280F0308133
:105CF800784D285D0AF093FE05F11003185D0AF04F
:105D08008EFE05F120033035185D0AF088FE285D07
:105D18000AF085FE0134E6E708200AF0AFFE00200D
:105D28000AF0AFFE00200AF0ACFE00200AF0A9FE3F
:105D380000200AF0A6FE0BE104200AF09FFE5F4B4C
:105D4800986803E194F87C010AF069FE94F88001F0
:105D58000AF065FE94F87F010AF061FE94F881016B
:105D680066E0564C07200AF089FEB4F882010AF072
:105D780088FEB4F884010AF084FE94F886010AF0DB
:105D88004EFEB4F88801D4E74C4C0C200AF076FE9D
:105D980094F892010AF043FEB4F89C010AF071FEEF
:105DA800B4F898010AF06DFEB4F89A010AF069FE99
:105DB80094F893010AF033FEB4F89E010AF061FEEC
:105DC800B4F8A001B5E73D4C04200AF057FE94F85A
:105DD800D8010AF024FE94F8D9010AF020FEB4F89C
:105DE800DA01A6E73C4C3D4D207800EB4000C0B2FC
:105DF8000AF044FE002623789E4205F1020580F051
:105E0800A78015F8020C0AF00AFE15F8010C00EB41
:105E1800800000EB800000F2EE2080B20AF031FE34
:105E28000136E8E701200AF029FE244B93F8940193
:105E38000AF0F5FD8CE008200AF020FE00241F4B34
:105E48002344013493F88A010AF0E9FD082CF6D1BD
:105E58007EE0174B194C93F8C900C0EBC000C0B2E4
:105E68000AF00CFE04F1200594F8F60100231C4A00
:105E7800D25C904270D00C33302BF8D10834AC424D
:105E8800F2D165E040200D4C0AF0F8FD04F1400520
:105E9800B4F8A8020AF0F5FD94F8AA020AF0BFFDCA
:105EA800043494F8A7020AF0BAFDAC42F0D14FE0EE
:105EB8005C1100206D11002074850108501200202B
:105EC800441A00204C1A00204A1A0020481A0020C0
:105ED800461A0020E5110020142B0020F2130020A0
:105EE800202B0020E0202A4C0AF0C8FD04F1800590
:105EF800B4F82A0200F03F000AF0C3FDB4F82A0201
:105F0800C0F386100AF0BDFD94F8280200090AF0D3
:105F180086FD94F8280200F00F000AF080FD043492
:105F280094F825020AF07BFDAC42E1D110E0132081
:105F38000AF0A4FD0024174B185D01340AF06FFD28
:105F48000B2CF8D100200AF0A5FD00200AF0A2FDD4
:105F5800012018E0002016E00AF061FDB4F8F8010D
:105F68000AF08FFD94F8FA010AF059FD94F8FB0144
:105F78000AF055FD94F8FD010AF051FD94F8FC0172
:105F88000AF04DFD7AE7BDEC028BBDE8F08700BF53
:105F980050120020D8A401082DE9F047D14CD24F67
:105FA800237886B00646002B00F0F8813A686368CB
:105FB800D31A7C2B40F2F281237A62600133237278
:105FC8004FF0000808F12400C64DC0B205F0FCFFF0
:105FD80005F10A0333F9183007EE903AC34B1B88D2
:105FE800B8EEE77A07EE903AF8EEE77A08F101089A
:105FF800C7EE277A9FEDBE7A67EE877AFDEEE77ADD
:10600800CDED037ABDF90C0005F0CCFFB8F1030F14
:10601800D8D1302005F0D8FFB5F9100005F0C2FF3F
:1060280005F0CAFF2B7A9A072CD16A6841F28833A7
:106038009A4218D9102005F0C7FF4FF06408686924
:1060480090FBF8F000B205F0ADFF212005F0BCFF91
:10605800686990FBF8F308FB13000028B8BF4042BA
:1060680000B205F09FFF142005F0AEFFB4F9180048
:1060780005F098FF1C2005F0A7FF002005F092FF0F
:1060880005F09AFF237ADFF85C825B0740F06381B2
:10609800022005F099FFD8F81C00DFF86C92642301
:1060A800323090FBF3F000B205F07CFF0320B8F922
:1060B800265005F089FF8F4B1B7813F0040F4FF023
:1060C800050A95FBFAF5ADB20DD008F5D970314641
:1060D80005F0E1FA28B9D9F8003013F0100F18BF0D
:1060E800002528B205E0D8F804389889B0FBFAF002
:1060F80000B205F057FFD9F800309E076ED5DFF8DB
:106108000C92B4F80A6899F80030B4F80828754D6C
:1061180036014FF06408B6B208FB02325B00B2FBEE
:10612800F3F346EA0326B6B2C3F303231E4306205D
:1061380005F04AFF30B205F035FFB4F80A3899F88F
:10614800001001339BB293FBF1F201FB1233A4F868
:106158000A38D4F80C389B7B012B05D1392005F07F
:1061680033FFB5F908081AE0B5F808586E233A2045
:106178005D43152605F028FF95FBF6F5AEB2B6FB94
:10618800F8F528B205F00EFF08FB15653B2005F071
:106198001BFFA8B2451D0A2095FBF0F000B205F0E0
:1061A80001FF282005F010FFD4F810380A2093FBCF
:1061B800F0F000B205F0F6FE042005F005FFD4F873
:1061C80004389B8913B102F053FA04E0454BD3F825
:1061D800140880F3100000B205F0E4FED4F8183873
:1061E800404E9D0640F1AC8096F81C3898071DD5A6
:1061F800112005F0E9FEB6F81E083F4B4FF4F36591
:10620800684390FBF3F000B205F0CCFE192005F0CE
:10621800DBFEB6F81E084543642095FBF0F595FBB8
:10622800F0F300FB135000B205F0BCFE94F81C38E4
:10623800B4F8205813F0020F08BF0025012005F01C
:10624800C3FE28B205F0AEFE092005F0BDFE002011
:1062580005F0A8FE294B94F822581A88B2F5967FC3
:106268000AD9204B1B7A03F00F03072B04D842F2FC
:106278000F75954228BF1546052005F0A5FED4F8F0
:106288000C385B7B0BB928B21CE0A5F1200307EEA4
:10629800903A9FED1B7AF8EEE77AF6EE006AC7EEC1
:1062A800877ABEEE007AF5EEC07AF1EE10FA58BFA2
:1062B800B0EE667A77EE877AFDEEE77ACDED037A6F
:1062C800BDF90C0005F06EFE94F81C28054B9107EB
:1062D80003D493F82328012A1CD1012384F82338F6
:1062E800084834E0281200207C2E002004000020FA
:1062F80000007A44EA2F0020A0860100FE0000205A
:106308006666E63F4C1A0020582E0020FC0000204C
:106318008096184BD3F80C385FED036A93ED017A39
:10632800D3ED027A27EE267A67EEA67ABDEEC77A13
:10633800FDEEE77A8DED047ACDED057A04A806E046
:10634800B74A92E8030004AB83E80300184602F05A
:1063580037FF05F031FE237A282B1FD1B14B0022DD
:106368001A723C263B684FF47A70B3FBF0F817209A
:1063780005F02AFEB8FBF6F5B5FBF6F006FB105063
:10638800000200B205F00EFE182005F01DFE06FB07
:10639800158000B205F006FE05F00EFE94F82C38C4
:1063A800A04D002B00F05D8105F006FAD5F83038D5
:1063B8009D4AC31A9342064640F2C680002385F8D8
:1063C800363885F83838B5F80838DAB21B0A85F84F
:1063D800522885F8533885F8482885F84938D5F87B
:1063E80060283B689A1AD5F86438D97B4FF47A73D9
:1063F8004B439A420ED38D4B1B68C5F8603895F80D
:106408006838013B012B9FBF102385F836380223DB
:1064180085F838380A20D4F8102892FBF0F284F86E
:106428005028121284F8512894F81C28D4F81438EB
:1064380093FBF0F384F854381B1284F8553892070C
:1064480094F82238774984F8833803D42D2381F8C7
:10645800843877E0042BD4F82498D4F82878DFF827
:10646800DC81734A8CBF3323322381F884384FF0A0
:10647800060C704B99FBF3F097FBF3F308FB0091C4
:1064880008FB037803EB83030CFB01F103EB8303A5
:1064980091FBF2FE642502FB1E119B0091FBF5F1B6
:1064A80084F8751809120CFB08FC84F876189CFB14
:1064B800F2F143FA81F39BB202FB11C292FBF5F2AF
:1064C80084F87A28121284F8783884F87B281B0A12
:1064D800B4F81E2884F879382423534393FBF5F540
:1064E800B4F8963884F87C3800EB80001B0A00EB7F
:1064F8008000800084F87D380A22B4F82038B3FB85
:10650800F2F303F5FA739BB240FA8EF080B284F886
:106518007E381B0A4FEAD97984F87308FF0F000AFE
:1065280084F8705884F87F38C5F30725B4F898388C
:1065380084F8729884F8740884F8777884F8715825
:1065480084F88538C4F8306894F89A88354DB8F1DD
:10655800000F0DD1D5F8A00805F0E5FA012807D9F4
:106568000228354F00F05D8202F01CFE0123BB704B
:10657800D4F8A4282B4D002A73D095F89A783FB107
:10658800D5F8AC3840F6B731F31A8B4219D868E021
:106598000123D5F8A00885F89A3807F0E6FFD5F862
:1065A800B03893F9000002238DE8880008213A46A4
:1065B8004FF4964305F031F985F8B478C5F8A0088A
:1065C8004DE095F8A878CFB9D5F8A008C5F8A47813
:1065D80085F89A7807F0C9FFD5F8B03893F9000024
:1065E80001238DE8880008213A464FF4964305F0C8
:1065F80014F9C5F8A00802F0D5FD30E0013FFFB25C
:1066080085F8A87895F8B41895F8B538C7B94A1C2C
:10661800013385F8B42885F8B538D5F8A0081CE00A
:1066280000870108281200203F0D03007C2E00205F
:1066380040420F008096980004000020806967FFA0
:1066480012F8017BC5F8A428781885F8B408013336
:10665800D5F8A00885F8B538394605F067FAC4F8C2
:10666800AC6894F8B638A24DF3B1D5F8B838DBB1B8
:10667800D5F8BC38C3B1C5F8C0381B689D4AC5F801
:10668800C438D5F8C8381344187AFEF745FDD5F84C
:10669800C03898790AF0C3F9D5F8C8380133092BFE
:1066A80088BF0023C5F8C838934D94F8CC282E68C5
:1066B8008F4B002A00F0F081D3F8D028002A00F090
:1066C800EB8193F8D438013B012B00F2E581D4F833
:1066D800D008874F05F027FAE0B1D7F8D00805F0C1
:1066E8001FFA97F8D538D5F800907E2B80460ED142
:1066F80002231B2887F8D43809D1D7F8D00805F029
:1067080012FA20B90123C7F8D89887F8DC3884F83A
:10671800D588DCE7D7F8D8282B689B1A41F6583279
:1067280093421ED9032387F8D438B5E1734A32F867
:10673800130010B903464FF403600133B0F5C06F7E
:10674800DBB279D01ED9B0F5006F7FD032D9B0F561
:10675800036F3FD184F8DD38D4F81838644F9906B0
:106768003FD494F8DC1894F8DD38002900F05681FD
:106778002A68921B012AD9D984F8DD38002384F8C5
:10678800DC3889E1B0F5007F43D007D8B0F5807FC9
:1067980049D0B0F5887F00F08D80E6E7B0F5806FCE
:1067A80000F0B080B0F5826F00F0F580B0F5047F9E
:1067B800DBD123E0B0F5E26F00F08D80B0F5E46F37
:1067C80000F08E80B0F5E06FCFD184F8DD38B4F9F1
:1067D8000A1089E0B0F5046F76D0B0F5026FC4D125
:1067E80005E197F81C389A07BBD5B7F81E1824237B
:1067F8004B431233642193FBF1F109E184F8DD384E
:106808003F4B3B4F1B689B07ABD5B7F808380A21AD
:10681800FDE084F8DD383A4B354F1B681905A0D5E3
:10682800D7F81018F4E084F8DD38D4F81838304F69
:106838005A0796D57969EBE084F8DD38304B2C4F50
:106848001B681B058DD5D7F81418E1E0D4F8181883
:10685800274A84F8DD388F0683D592F81C188807F4
:106868007FF57FAFD90712D5D2F8283883EAE371CC
:10687800002BA1EBE37101EB51014FF01902B1FBC1
:10688800F2F1ACBF41F0004141F040410FE0D2F8D5
:10689800243883EAE371A1EBE371002B01EB51018A
:1068A8004FF01902B1FBF2F1B8BF41F080414FF44B
:1068B80000608BE084F8DD38D4F818380C4F5B079B
:1068C8007FF54FAF3969A3E0B4F9181084F8DD38C3
:1068D800642359437AE084F8DD38B4F90C1003E0F6
:1068E800B4F90E1084F8DD382C2391FBF3F16DE038
:1068F80028120020008701087C2E0020F0A801083B
:10690800582E002084F8DD3894F8DE38644A0133C4
:10691800DBB2032B88BF012382F8DE3894F8DE1837
:1069280042F2107359435F4B1B78D80748BF0131B7
:106938009A0748BF02315F07B4F8E03848BF04310E
:10694800D80748BF0A319A0748BF14311F0648BF05
:106958002831D80548BF28315A0748BF64311F0776
:1069680048BFC831980548BF01F5C8719A0648BFA5
:1069780001F57A71DF0648BF01F5FA61580648BF8C
:1069880001F57A614FF4806002F0D8FB444B002295
:1069980083F8DC28E5E6D4F81818DFF8048184F8D1
:1069A800DD3811F0200717D098F81C2812F0020FD4
:1069B80014BF4FF47A71002112F0010F14BF4FF485
:1069C800FA6300230B4494F82218194402F0B6FB2A
:1069D800002384F8DC38C4E6334B1B6819067FF5BE
:1069E800C0AE394602F0AAFB88F8DC78B9E684F82C
:1069F800DD38D4F818382A4F9A067FF5B2AE97F8E2
:106A08001C389B077FF5ADAEB7F820386421594391
:106A180002F094FB002387F8DC38A2E684F8DD381E
:106A28003AE0BB7823B1C5F89C6887F802809FE5F7
:106A3800D5F89C38F31AB3F57A6FFFF499AD0123B2
:106A4800D5F8A008BB7005F06BF80746D5F8A00884
:106A580005F066F87F067FF48BAD8A2802D08E2871
:106A68000DD085E5D5F8183898067FF581AD95F8ED
:106A78009A38002B7FF47CAD05F6690306E095F89B
:106A88009A38002B7FF474AD05F63403C5F8A438A2
:106A98002D2385F8A8386BE506B0BDE8F08700BF60
:106AA80028120020EA2F0020582E002082B01B4B0D
:106AB8001B4A8DF807101968106860B31268052A18
:106AC80029D1184A106810BB9DF808109DF80730A6
:106AD80043EA012314490B80144B1968144B89B2FB
:106AE8000B445B0019680121196013680B4413609B
:106AF800104A136823F4E04323F040039BB283F069
:106B0800300343F4004343F08003136003E01A6842
:106B1800521A312AD5D902B0704700BF7C2E002006
:106B2800D02F0020702A002080610040505C004077
:106B38000A300020045C0040014B1868C0B270475E
:106B48002C2A002001207047704770476D4B6E4A11
:106B58009FED6E7AD2ED007ADFED6D4ADFED6D3A8A
:106B680030B51C88B3F90AE01D8A06EE904AB8EEE3
:106B7800E76AF8EE666ADFED687AB3F9044067EE13
:106B8800E67AB7EE004AE6EE077A9FED647A67EE9A
:106B9800666A9FED637AE6EE076A27EEA77A07EE44
:106BA800904AB3F902409FED5F6AF8EEE77A67EE24
:106BB800277A07EE104AB8EEC77ADC89E6EE877ABC
:106BC800B6EE007AFDEEE76A87EE866AC3ED066ADE
:106BD800F8EEE66AD2ED017A9A89E6EE874A06EE81
:106BE80090EAB3F908E09FED507A05EE90EAF8EEE6
:106BF800E66AF8EEE55A66EEA46A65EEA45A66EE11
:106C0800A46AB3F806E0E6EE875A65EE875AA5EE61
:106C1800A34AF0EE445A04EE10EAB8EE444A25EED0
:106C2800844AB5EE404AF1EE10FA5BD02DB205EE7B
:106C3800905A24B224EEA45A07EE104AF8EEE55A08
:106C480012B265EE255AB8EEC75A65EEA35A64EE3D
:106C5800854AB0EE007AE4EE875AB5EE007A65EE22
:106C6800875A07EE102AB8EEC75A9FED307ADFED43
:106C7800306AB3F91620E5EE075AF8EEE77A9FED89
:106C88002D7A76EEE77ADFED2C6AE5EEC77A05EE27
:106C9800902AB0EE677ADFED297AB3F91420B3F9B8
:106CA800123067EE277A07EE102AC7EE847AF8EEDC
:106CB800E55AB8EEC77A65EEA75A27EE877A65EEE9
:106CC800A75A27EE237AA5EEA67AF0EE476A07EED2
:106CD800103AB8EEC77A36EE877ADFED196AE7EE32
:106CE800267A01E0DFED177A18B1FDEEE77AC0EDFC
:106CF800007A31B1FDEEC67A642217EE903A53431A
:106D08000B6030BD080300200C1B0020000000377A
:106D180000007AC700000038000000390000803AFF
:106D2800000080380000A0450000003600008047C1
:106D38000000804900008039000000300050C34541
:106D48000000803D00000000704770476C4B6D4AA2
:106D58002DE9F04F5E8994684FEA062AB4EB0A0AD7
:106D68009C884FEA04481C894FF000054FF0000B3F
:106D780065EB0B0BA4FB0A6704FB0B77F40944EAE9
:106D8800476418EB04065C884FF000094FEAE715E2
:106D98004FEAC438DC8849EB050787B0CDE90467BA
:106DA800A4FB0A6704FB0B77340A44EA076418EB70
:106DB80004064FEA27259C894FF0000949EB05078F
:106DC800CDE90067AAFB046704FB0B77F40D44EADE
:106DD800472414F5FA664FEAE75545F10007B6F57A
:106DE800FA6F77F10003CDE90267964667DAA4FBEC
:106DF800046704FB05F34FF0050C07EB4307DDE9D7
:106E08000489A6FB0C230CFB07335F104FEA3206FC
:106E1800B8EB06084FEA920669EB070946EA83765B
:106E28009F10DDE90023921B63EB0703DDE902678E
:106E3800CDE90023344A4FF0FF33964277EB030342
:106E4800CDE9048928DA40F6AC52A4184FF00003C3
:106E58005D4104FB05F3A4FB044505EB43056FF016
:106E68000602664202FB0566A4FB0223334418EBC4
:106E7800020649EB0307CDE904670B26A4FB0623AA
:106E880006FB0533DDE900455B104FEA3202A41A20
:106E980065EB0305CDE900450AFB0BF3DDE9024587
:106EA800AAFB0AAB0BEB430B4FEADA7242EA4B023E
:106EB800A41A4FEAEB7365EB0305CDE90245DEF84A
:106EC8000C40009B019DA4FB032304FB05334FEA00
:106ED80052584FEA635948EAC328DDE90423B8EB5E
:106EE800020269EB03039946D30B43EA494300B115
:106EF800036009B1029B0B6007B0BDE8F08F00BFCB
:106F0800F60200200C1B002024FAFFFF07EE900A6F
:106F1800F8EEE77ADFED0C6A9FED0C0AF5EEC07A21
:106F2800F1EE10FAD4BFB1EE677AC7EEA67A08B5CB
:106F3800D8BFC7EE267A27EE800A02F0C7FC044BBA
:106F480083ED000A08BD00BF8096184B35FA8E3CC9
:106F58006C000020F7B51C4B1A680AB91C6800E0E1
:106F680001241A490E7C0022D0B2A04202F101028B
:106F780007D202AD2F18164D3544285C07F8040CCB
:106F8800F2E71A68121B1A600A7C1D6822440A7408
:106F98009DB90320402100F07BFF0E4A136823F4BB
:106FA800804323F070039BB283F4405343F40043BF
:106FB80043F080031360054B1D74002CCBD09DF863
:106FC800040003B0F0BD00BF2C2A00200C1B0020D9
:106FD800302A00200C5C00407620F4213122FEF794
:106FE8002DB81FB5044602210C2001220DF107031C
:106FF800FDF7A8FFC8B39DF80730DB0735D5032197
:10700800062202AB0C20FDF79DFF0C20092101226E
:107018000DF10703FDF796FF38B39DF8073013F01D
:107028000C0F22D19DF809209DF8083043EA02236D
:10703800C3EB83339B009DF80B2023809DF80A3017
:1070480043EA0223C3EB83339B009DF80D20638042
:107058009DF80C3043EA0223C3EB83339B00A380E3
:107068000C200A210122FDF7E9FF04B010BD07B585
:10707800F7216B4606227620FDF764FF9DF8003065
:107088009DF801100B4A1B0343EA01139DF80210F7
:1070980043EA111353609DF803309DF804101B0355
:1070A80043EA01139DF8051043EA1113136003B076
:1070B8005DF804FB0C1B002007B50A2100220C20F8
:1070C800FDF7BCFF142004F09EFB0A210F220C20C0
:1070D800FDF7B4FF0A2004F096FB01AB1021032250
:1070E8000C20FDF72FFF0A2004F08DFB0A21002257
:1070F8000C20FDF7A3FF0A2004F085FB0DF1030324
:10710800022101220C20FDF71DFF0DF103030921C7
:1071180001220C20FDF716FF0A2101220C20FDF7A1
:107128008DFF03B05DF804FBF8B59F4B1B68044660
:10713800187818B1012800F07181EDE2242C9B4DDC
:107148000CD006D80A2C00F0DD800D2C00F0DA8077
:107158004EE12A2C06D02C2C04D049E16874A8747E
:10716800E87457E1924BA97C6F7C904A00205854F0
:107178002FBB19781775472921D1597850291ED165
:107188009978472907D1D978472904D1197941290C
:1071980001D1012111759978854A522903D1D178F5
:1071A8004D2900F0BB829978814A472907D1D178C7
:1071B800532904D11279562A04BF03222A752A7D3D
:1071C8007A4E022A3AD0032A4DD0012A40F088800C
:1071D800BA1E072A00F28480DFE802F004080F13C1
:1071E8001A25822B0BF070F9A86179E01B78532BD4
:1071F80076D1AB695B42AB6172E00BF065F9E8618F
:107208006EE01B78572B6BD1EB695B42EB6167E053
:107218001B78302B674B1A788CBF42F0020222F0A1
:1072280002021A705CE000200BF0AEF985F820002D
:1072380056E000200BF0A8F9688451E0072F06D02B
:10724800082F4DD101200BF09FF9F08448E0012070
:107258000BF09AF941F2184358434FF47A73B0FB94
:10726800F3F0B0843CE0022F07D0032F0BD10020AD
:107278000BF08AF9504B187032E000200BF084F9BB
:1072880086F828002CE02BD93A1F921096F828305F
:107298000132D2B2013B02EB8303DBB2102B1FD8C1
:1072A800F91EC2F1010201EB8202D2B2012A0BD00F
:1072B800042A11D100205E1E0BF066F93F4B985549
:1072C8003F4B00229A5507E05E1E3E4A0020935528
:1072D8000BF05AF93C4B98553C4A1368013313603C
:1072E800324B2A2C18BFDA7C07F101074FF0000057
:1072F8000CBF012254406F74A8740CBF83F8292076
:10730800DC7487E095F82900002848D0304B13F842
:10731800012D30495A708B42F9D1254A234C1378F4
:107328005278402B85BF373B1B011B01DBB298BF4E
:1073380003F0F003402A8CBF373A303AD2B21344F4
:10734800EA7CDBB29A4227D121230B702249207DA7
:107358000B68204A013301280B600AD002281DD18E
:10736800722313701D4BA28C1A801D4BE28C1A805D
:1073780014E0672313700F4B1B789F070FD5194B29
:10738800A2691A60E2695A60174B94F820201A70B3
:10739800164B628C1A8002E03F230B7000200023FA
:1073A80085F8293036E000BF200800200C1B00209B
:1073B800842E0020441A0020E41100201512002019
:1073C80005120020E5110020F511002030210020D1
:1073D80044030020300300203C210020461A0020EE
:1073E800CC1100204C1A00204A1A0020481A00200C
:1073F800AB7C95F829000E2B9FBFAB4A591C9174A2
:10740800AA4A98BFD454A84A18B9D37C5C40D4740B
:1074180000E00020003018BF0120F8BDA24B93F80F
:107428002A100022082900F27781DFE801F0050C14
:10743800101A2B3B5F7B8800B52C40F06D8183F8D8
:107448002B2001224FE0622C08BF02224BE00322CE
:1074580083F82A2083F82C4083F82D4083F82E40A7
:107468005AE1042283F82A2093F82D2093F82E104D
:1074780083F82F402244D2B283F82D200A4483F89F
:107488002E2049E1052283F82A2093F82D2093F82D
:107498002E101C862244D2B283F82D200A4483F889
:1074A8002E2039E1062283F82A2093F82D2093F81C
:1074B8002E102244D2B283F82D200A4483F82E20BD
:1074C8001A8E02EB0424A4B2B4F5AC7F88BF764AC6
:1074D8001C8684BF012182F82B1000225A86002CBA
:1074E80040F01A81072283F82A2015E193F82D200D
:1074F80093F82E102244D2B283F82D200A4483F840
:107508002E205A8EB2F5AC7F3CBF6749891802F12C
:10751800010238BF81F83440198E92B291425A86DE
:10752800E0D9F9E0082283F82A2093F82D30A34205
:1075380000F0F2805C4B012283F82B200FE05C4DB9
:1075480083F82A2015F8012D6A705A4A9542F9D114
:1075580093F82E10544AA14206D03F232B70564A66
:10756800536801335360D7E0544801680131016022
:1075780092F82B0010B13E232B70CDE02121297009
:1075880092F82F10062941D004D8022907D00329E0
:1075980023D0F8BD122959D0302967D0F8BD502121
:1075A80029704749946B4C60D46B0C60516C4FF454
:1075B8007A7491FBF4F1434C218092F88C11424A81
:1075C80019B1117841F0020102E0117821F00201AD
:1075D8001170012283F88D2190E05321297092F8CF
:1075E8003910CE0705D592F83820D51E6A426A416F
:1075F80000E0024602F0010183F88C11002A7DD1D7
:1076080031490A7822F002020A7077E04F21297086
:1076180092F83F10CC0705D592F83E20D11E4A4279
:107628004A4100E0024602F0010183F88C1122B9B8
:1076380025490A7822F002020A70244A93F8631056
:107648001170234AB3F86010118057E05621297051
:107658002049946C0C8042F21074D16C91FBF4F1C7
:107668001D4C2180012182F88E1147E049212970A3
:1076780092F83810194A102988BF1021117018493A
:1076880014780022A24235D2164D0E7A5655164D60
:107698004E7A5655154DCE7A5655154D11F80C6F34
:1076A80056550132EEE700BF0C1B0020842E002047
:1076B8004403002030030020000800203C21002063
:1076C8004C1A0020481A0020441A00204A1A0020A8
:1076D800FE000020461A0020CC110020E4110020F2
:1076E800401B0020E5110020F511002005120020A4
:1076F800151200200D490A6801320A6093F88D318D
:107708000B4A93B192F88E317BB1002182F88D112A
:1077180082F88E111846F8BD0020F8BD1279432A68
:107728007FF441AD02222A753DE5F8BD30210020E5
:107738000C1B00200449054B0968187000225A6187
:1077480099611A77704700BF7C2E0020000800203E
:1077580010B5121A07EE902A5B1A2DED028BF8EE7F
:10776800E78A07EE903A184B059CB8EEE78AD3ED06
:10777800007A28EE278A28EE080AA8EEA80A0EF052
:10778800A5FFDFED127A049B20EE270AF0EE480AE7
:10779800BCEEC00A83ED000AB1EE680A0EF0F2FDF5
:1077A800DFED0B7A9FED0B7AE0EE077ABDEC028BEA
:1077B800FDEEE77A17EE903A002BBCBF03F50C43B9
:1077C800A033236010BD00BF6C0000202C7D8E3FCD
:1077D80000A00C46A00CB34544F25063984203DD68
:1077E800A0F50C40A0387047034B9842BCBF00F589
:1077F8000C40A030704700BFB0B9FFFF73B51A4CFA
:10780800036823600B686360184D0068184EFFF723
:107818007DFB184B009395E8030094E80C00019653
:10782800FFF796FF144B32681A606868636813495B
:107838001B1A07EE903A124B286893ED007A2368DA
:107848001B1A0B600F4BF8EEE77A1A600E4B67EEC7
:10785800877A1B68FDEEE77ADA880C4BC1ED017A6E
:107868001A8002B070BD00BFAC2900204C1A00205D
:10787800B8290020B4290020F4290020BC290020C0
:107888006C000020EC290020900F0020E82900203F
:107898004279DFED2A5A2A4B9FED2A5A07EE902AA1
:1078A800F8EE677AC27BC7EEA57AB2EE047AC3ED2A
:1078B800007A07EE902AF8EE677A234ADA60C7EE74
:1078C800A57AC3ED017A8179204B07EE901AF8EE7C
:1078D800677A017CDA60C7EE877AC3ED007A07EE33
:1078E800901A817E06EE101AF8EE677AB8EE466AAC
:1078F800C7EEA57A86EE056AC3ED017A83ED026AC2
:10790800C179134B06EE901A417CDA60F8EE666A8C
:10791800C6EE876A07EE101AC17EC3ED006A07EE4D
:10792800901AB8EE477AF8EE677A87EE257AC7EEAE
:10793800857A83ED017AC3ED027A70470000C84268
:10794800C429002000007A440000FA44D429002009
:10795800F829002010B50C4C23789B0713D50B4B46
:107968001B78042B0FD90A4A0A4B106852685A60D0
:107978001860FFF7CBFA084B1A88084B1A8023784F
:1079880043F00103237010BD441A00204A1A002056
:107998004C1A0020D011002040120020082A002094
:1079A8001C4B1B681B0307B530D51B4A1B4BD2ED7C
:1079B800007A1B788DF80030B2EE047A67EE877A89
:1079C800174B9FED187A1B788DF80130FCEEE77A9B
:1079D8000A2017EE903AD2ED017A8DF8023067EE60
:1079E800877A6946FCEEE77A17EE903AD2ED027A8A
:1079F8008DF80330FCEEE77A17EE903A8DF80430F4
:107A0800094B1B788DF8053001F008F803B05DF8D4
:107A180004FB00BF582E00206C2E0020482E0020AA
:107A2800682E002000007A444C2E0020054A137866
:107A380083F001031370044A00231360034A1360A0
:107A4800AEE700BF4C2E0020642E0020602E0020E0
:107A580010B5214A18B9136802221A8210BD1F48AE
:107A6800146800230380217811F07F0102460DD1AC
:107A7800637A990644BF0221017013F0400F03781E
:107A880014BF43F0010323F0010315E0012921D0BD
:107A980002291ED1637913F0800F03F00F034FEA18
:107AA800830303F1804303F5B8431B6806D003F052
:107AB8003003102B07D10123137004E003F4405363
:107AC800B3F5805FF6E7064B1B681B6998470348C8
:107AD80010BD184610BD00BF0C2A0020A01C0020B5
:107AE8009C27002010B5064C18B9236801221A8279
:107AF80010BD044B1B689B68984720680C3010BD6C
:107B08000C2A00209C27002010B5064C18B92368C1
:107B180001221A8210BD044B1B681B689847206815
:107B28000A3010BD0C2A00209C27002003788B42C5
:107B380083BF034B03EB410148880020704700BF17
:107B4800A01C002070B500221346244914180C44C8
:107B5800A47E83EA0423082413F4004F4FEA430366
:107B680018BF83F4815304F1FF3418BF83F0010375
:107B780014F0FF049BB2EFD10132192AE5D100F1CC
:107B8800190200F11A050A440D44967EAA7E02EBFA
:107B9800062292B29A421FD1104B93F83B50E2B2A0
:107BA800AA4216D2431C03EB4203DBB2CA180133C4
:107BB8000B44927E9B7E03EB02239BB24FF4AF6291
:107BC80053431B13064A03F5487322F81430013453
:107BD800E5E7012381F83C3070BD00BFA01C002000
:107BE800A21C002003788B420BD9074B1A78074B4D
:107BF80089001944086C02B1400800F5777080B21A
:107C080070470020704700BF182B0020A01C0020E0
:107C180007299DBF034B03EB8101B1F870000020D9
:107C2800704700BFA01C0020034B03EB4101B1F8D3
:107C38009000C008704700BFA01C002070B5334CEE
:107C4800054603F0B9FDD4F8B030C4F8B000C31A43
:107C5800B3F5FA5FC4F8B43082BF002384F8B830B3
:107C680084F8B93094F8B8302BB9A12D02BF274A4F
:107C7800012182F8B91094F8B910244A29B1D11811
:107C8800EDB201338D7682F8B83094F8B85094F894
:107C9800BA30AB4239D11D4B93F8BB30052B02D01B
:107CA800062B03D02CE00020FFF74CFFE37E1E2BB1
:107CB80026D100200246C1B26B1E994219DA21442E
:107CC8008B7E0821DBB283EA0206F60744BF83F005
:107CD8001803C3F3460301F1FF3154BF5B0843F0B7
:107CE800800311F0FF01C2F34702ECD101301A46BC
:107CF800E1E723449B7E9A4202D10320FFF722FF4B
:107D0800002384F8B93084F8B83070BDA01C002076
:107D180010B5044603F050FD0F4BD3F8BC20C3F850
:107D2800BC00821A41F288318A42C3F8C02084BF5D
:107D3800002283F8C42093F8C420074913440F2A6B
:107D4800E4B218BF013283F8C54012BF81F8C420DD
:107D5800012381F8D53010BDA01C002010B50446C1
:107D680003F02AFD0F4BD3F8D820C3F8D800821AA5
:107D780041F288318A42C3F8DC2084BF002283F8AC
:107D8800E02093F8E02007491344142A18BF013271
:107D980083F8E14012BF81F8E020012381F8F63032
:107DA80010BD00BFA01C00202DE9F843324F3D68EC
:107DB8002A8A2E7AB2B9042E14D1304C304823784E
:107DC800012B0BD12F4B19682F4B89B20B445B0049
:107DD80019681A6030230380227048E0102303805A
:107DE800072644E0AC8AAB69A24294BF0426022667
:107DF800944228BF14461FFA84F840469847214AFF
:107E080013689BB203F1005303F540535B0004F180
:107E1800010E1B689BB203F1005303F540534FEA70
:107E28006E0E5B000021714500F1020009D010F8C8
:107E3800019C10F802CC4CEA092C23F821C001312E
:107E4800F1E71268104B92B213445B001A681C6089
:107E58002B8AC8EB03032B826B8A9844084BA5F83E
:107E6800128030221A80094B4FF440521A803B6826
:107E78001E72BDE8F88300BF0C2A0020EC2F0020FA
:107E880096270020505C00400230002094270020F4
:107E98000E4B0F4A1B689BB203EBC00002443E29FD
:107EA8004FEA420209D94B09C80604BF03F1FF3360
:107EB8009BB29B0243F4004304E04B08C90748BF48
:107EC80001339B0211681360704700BF505C00408B
:107ED8000630002010B5454B1A68107810F07F0066
:107EE80004D1537A23F02003537210BD02287AD1AB
:107EF8005388002B78D11379002B75D1537923F04F
:107F08008000840004F1804101F5B84113F0800F2E
:107F1800096814BF01F0300101F44051032862D808
:107F2800002960D0927A002A5DD004F1804404F5DB
:107F3800B8441906226825D502F03002102A4CD11F
:107F480003F07F039B0003F1804303F5B8431A68ED
:107F5800510641BF196840F60F720A4042F40042C8
:107F680044BF42F0C0021A601A6822F4E04222F0CC
:107F7800400292B282F0300242F4004242F08002A3
:107F88001A602AE002F44052B2F5805F25D128B980
:107F9800174B93F82C10FFF77BFF11E09B0003F1C0
:107FA800804303F5B8431A68520441BF196840F684
:107FB8000F720A4042F4404244BF42F080021A6005
:107FC800236823F4804323F070039BB283F4405367
:107FD80043F4004343F080032360064B1B685B694E
:107FE8009847002010BD022010BD00BF0C2A0020B9
:107FF800A80000209C2700200023036043608360C2
:108008008381036143618361C36103624362836265
:1080180070478A68036810B50C6A14430A691443E8
:108028004A6914438A691443CA6914434A6A14435F
:108038008A6A23F4FF4323F0700322431343036047
:108048008B8943600B6883604B68C36010BD02680E
:108058004FF6FE73134003600023036043608360A0
:10806800C360294B984201D1284A27E0284B9842FF
:1080780001D1264A2AE0274B984201D1234A2DE014
:10808800254B984201D1214A30E0244B984201D136
:108098001E4A33E0224B984204D11C4A536843F4E9
:1080A80070032EE01F4B984204D1184A536843F0DE
:1080B800706326E01C4B984204D11C4A536843F075
:1080C8000F031EE01A4B984204D1184A536843F034
:1080D800F00316E0174B984204D1144A536843F44E
:1080E80070630EE0144B984204D1104A536843F46D
:1080F800704306E0114B984204D10C4A536843F48C
:1081080070235360704700BF08000240000002401F
:108118001C00024030000240440002405800024067
:108128006C00024080000240080402400004024043
:108138001C04024030040240440402405804024037
:10814800084BDA68D10709D4DA68D20608D4DB68A4
:1081580013F0040F14BF0320042070470120704758
:108168000220704700200240036A23F001030362E3
:10817800036A70B5446882690D6822F4803222F07F
:10818800730215438A8923F0020313438A88134331
:10819800134A90420FD002F5006290420BD002F5CC
:1081A8004062904207D002F58062904203D002F507
:1081B800806290420DD1CA89CE8823F00803134308
:1081C8000A8A24F4407414434A8A23F0040333438C
:1081D80014438A68446085614263036270BD00BFCE
:1081E800002C0140994A536803F00C03042B2DE935
:1081F800F04105D0082B06D095490160B3B916E0C7
:10820800934B036012E053685468C3F38343991C8B
:10821800E30349BFD36A8F4B8D4C03F00F0344BF70
:108228000133B4FBF3F34B43036000E000235168D0
:10823800894FC1F303117D5C0168EDB221FA05F4A1
:1082480044605668C6F30226BE5D24FA06FEC0F8EE
:1082580008E05668C6F3C226BE5DF6B2F440C460B4
:10826800D2F82C80C8F3041808F00F0C07EB4C0C5C
:1082780018F0100FBCF810C01FFA8CFC07D0BCF126
:10828800000F04D0B3FBFCFCC0F810C000E0016193
:10829800D2F82CC0CCF3442C0CF00F0807EB48079D
:1082A8001CF0100F3F8ABFB204D01FB1B3FBF7F721
:1082B800476100E04161176BFF065ABF644F876151
:1082C8008161176BBF065ABF614FC761C161176BE8
:1082D8007F065ABF5E4F07620162176BFF0506D51E
:1082E800994204D1AE4202D14F00476200E0446295
:1082F800176BFF0406D5994204D1AE4202D14F0054
:10830800876200E08462176BBF0506D5994204D1E5
:10831800AE4202D14F00C76200E0C462176B7F050E
:1083280006D5994204D1AE4202D14F00476400E01D
:108338004464176B3F0506D5994204D1AE4202D179
:108348004F00876400E08464176BBF0406D5994228
:1083580004D1AE4202D14B00C36400E08464156BC3
:108368003A4BAD0701D1046315E01C6B04F003041C
:10837800012C01D101630EE01C6B04F00304022CF4
:1083880002D14FF4004305E01B6B03F00303032BFA
:1083980001D12F4B0363146B2C4B14F4403F02D1D3
:1083A800C0F834E018E01C6B04F44034B4F5803FA6
:1083B80001D1416310E01C6B04F44034B4F5003F74
:1083C80002D14FF4004306E01B6B03F44033B3F5CE
:1083D800403F01D11E4B4363146B1C4B14F4402FD8
:1083E80002D1C0F838E018E01C6B04F44024B4F55E
:1083F800802F01D1816310E01C6B04F44024B4F594
:10840800002F02D14FF4004306E01B6B03F4402316
:10841800B3F5402F01D10E4B8363146B0B4B14F44F
:10842800401F02D1C0F83CE020E01C6B04F440146B
:10843800B4F5801F01D1C16318E01C6B04F440142B
:10844800B4F5001F0AD14FF400430EE000100240BB
:1084580000127A0000093D00080000201B6B03F49D
:108468004013B3F5401F01D1134BC363126B134B79
:1084780012F4400F03D1C0F840E0BDE8F0811A6B58
:1084880002F44002B2F5800F02D10164BDE8F08128
:108498001A6B02F44002B2F5000F02D14FF4004308
:1084A80006E01B6B03F44003B3F5400F01D1024B08
:1084B8000364BDE8F08100BF00127A00001002409A
:1084C800F0B500230E681C460125A54005EA060EF6
:1084D800AE452BD10F797A1E012A15D8856803225B
:1084E8009A4025EA020282604D7982689D401543D0
:1084F8008560828892B222EA0E0282808A79858813
:10850800A2402A4392B28280032205689A40D2434D
:108518001540056005689F402F430760C7681740EE
:10852800CA7902FA03F547EA0502C2600134102C41
:1085380003F10203C8D1F0BD38B52DED048B4A4CC8
:108548000368C4F8F8308388A4F8FC30013A0D4673
:10855800072A42D8DFE802F0040A101822292F352A
:10856800B4F8F8300B80B4F8FA3013E0B4F8FA3005
:108578000B80B4F8F83005E0B4F8F8305B420B80B3
:10858800B4F8FA305B4205E0B4F8FA305B420B808D
:10859800B4F8F8306B80B4F8FC301DE0B4F8F8306B
:1085A8005B420B80B4F8FA3012E0B4F8FA300B8072
:1085B800B4F8F8300CE0B4F8F8300B80B4F8FA30BE
:1085C80005E0B4F8FA305B420B80B4F8F8305B424F
:1085D8006B80B4F8FC305B42AB80244B93F83030AE
:1085E800002B3ED1B5F9003094ED430AD4ED407A22
:1085F80009EE103AB5F9023008EE103AB8EEC88A1A
:10860800B5F90430B8EEC99A28EE000A08EE903A97
:10861800A7EE890AF8EEE88AD4ED467AA7EEA80A0A
:108628000DF0AEFD94ED440AD4ED417A288028EE91
:10863800000AA7EE890AD4ED477AA7EEA80A0DF03A
:108648009FFD94ED450AD4ED427A688028EE000A31
:10865800A7EE890AD4ED487AA7EEA80A0DF090FD96
:10866800A880BDEC048B38BDA01C002008000020A9
:10867800104BDFED117A1B689A89104B1B6883F346
:108688001003D31A07EE103AB8EEC77A27EE277A06
:1086980007EE902AF8EEE77AC7EE277AFDEEE77A3A
:1086A80017EE900A6428A8BF642020EAE070C0B2E0
:1086B800704700BF2C1A00200000C8423C1A002056
:1086C800094B1A68137844F6FB7103EB431300FB5C
:1086D80003135078C0EB0030B3FBF0F39078B3FB92
:1086E800F0F080B2704700BF2C1A002008B50A4885
:1086F80090F8253100EB43030A22B3F8341189B20C
:10870800A0F83C1100F5A07003F013FA80B2FFF74F
:10871800D7FF024B188008BDA01C0020301A00208B
:108728002E4B2F4A1B68126810B51A602D4A116823
:10873800596051689268DA602B4A9960116819612A
:10874800516892689A61294A59611168D9615168DA
:1087580092685A62264A1962118819855188598582
:108768009188D288DA85234A998511881986518893
:10877800598692889A86204A1188D98651881987FD
:108788001946928821F83A2F1C4A10780022824212
:1087980006DA1B4C34F8124021F8024F0132F6E792
:1087A800184A1288A3F86420174A1288A3F866208A
:1087B800164A1188A3F86C1051889288A3F8702083
:1087C800134AA3F86E1012689A66124A1288A3F820
:1087D8007220114A5289A3F85E2010BDB82C0020DF
:1087E800C82F0020282800203428002040280020F6
:1087F800481200208811002032120020C41F0020D7
:10880800A8110020DC1D00203C1000208E11002043
:108818003C120020C4110020941100202DE9F843D7
:108828000E4B93E8800305460E460024B44213DA43
:108838007B1933F9140008EB050333F9142009EB0D
:10884800050333F914301344022293FBF2F3C01AE0
:1088580008F081FF0134E9E7BDE8F883B82C00206F
:1088680070B5472008F0C6FE174B1B681B0307D5D9
:10887800164B174A5B6810681B68C01A08F05CFF43
:10888800144E154C154D307808F056FF23682868AB
:10889800C01A08F060FF63686868C01A08F05BFFD8
:1088A8000F4B188808F048FF0E4B188808F044FF53
:1088B8000D4B188808F040FF337823742B68A360A9
:1088C8006B68E36070BD00BF242E0020B82C002028
:1088D800C82F00204A1A0020A42C00204C1A00207F
:1088E800481A0020461A0020CC1100207FB5264CDB
:1088F800264E274D2749284A284B20B1284800886A
:10890800B0F5805F31D23088ADF8040028781E4D6C
:1089180091F8201012788DF806008DF807108DF860
:1089280008201B788DF8093001A8294606220DF089
:10893800FDF930B30198BDF808302860AB805320AA
:1089480008F058FE208808F0F7FEA07808F0F4FE3A
:10895800E37801932379029301A86379039308F0DC
:1089680051FE0F4B00221A800BE03088208091F8CE
:108978002010287812781B78A070E170227163713A
:10898800DDE704B070BD00BF681E0020081B002092
:10899800441A0020DC2E0020BB0E0020200F0020EF
:1089A800442E0020A0F17D03012B70B504460D462E
:1089B8000A4E05D830687D2103F0B8F884F0200409
:1089C8003068214603F0B2F835B12B881C4404EB1B
:1089D800142404F0FF042C8070BD00BFF81A002096
:1089E8000A4A138801331380094A13680133136054
:1089F800084A138801339BB2202B01BF0023138040
:108A0800054A138808BF013313807047442E00209D
:108A18002C2E0020302E0020322E002038B53A4B64
:108A28001B78083B012B05460C466BD8452008F0FF
:108A3800E1FD284608F0DEFD0C2D23D004D80A2DD0
:108A48000AD014D835B138BD0E2D4BD02ED3FF2DFA
:108A580050D038BD206849E0207808F0CBFD627915
:108A68006378002A14BF80200020184300E0207893
:108A780008F0C0FDA07808F0BDFDE07808F0BAFD68
:108A880020793BE0B4F9000008F04CFEA07808F02B
:108A9800B1FDE07808F0AEFDB4F9040008F042FE3C
:108AA800B4F90600BDE8384008F03CBE6378207889
:108AB8008BB180F0800008F09DFDA468E0B208F05A
:108AC80099FDC4F3072008F095FDC4F3074008F0AA
:108AD80091FD200E12E008F08DFD6068BDE8384079
:108AE80008F039BE206808F027FE6068BDE8384005
:108AF80008F022BE054808F05BFD0020BDE83840BC
:108B080008F078BD38BD00BF942C002010A90108DA
:108B18002DE9F04FB74BB84F1A888BB00193002A54
:108B280040F0A380B7F8D607B44E42F20103C21A48
:108B380050425041FFF7DAFEFFF7F2FD3468492052
:108B480008F058FDAE4B2546186808F0F5FD55F8B5
:108B5800040B08F0F1FD284607F0E0FC04F11000D2
:108B680007F0DCFC04F11C094FF01008A54D0123A7
:108B78002A6803FA08F3134203D0D9F8000008F072
:108B8800EAFD08F10108B8F1130F09F10409EDD164
:108B980004F1280007F0B2FCB7F84431B4F92E000C
:108BA800C01A08F0C9FD2B68DB0408D5964BB4F849
:108BB80064001B88181AC0F30D0008F0BDFD2B686F
:108BC800980403D5B4F8660008F0B6FD2B6859057B
:108BD80003D504F16C0007F091FC2B681A0502D547
:108BE800A06E08F0B8FD2B681B0403D5B4F872001A
:108BF80008F0A2FD04F13000A04607F07FFC04F164
:108C0800360007F07BFCB7F8443138F93C0FC01A3E
:108C180008F092FD01277D4B1B789F4208DA38F94E
:108C2800020FB4F93C30C01A08F095FD0137F2E79D
:108C38002B68980505D5B4F95E00A0F2DC5008F061
:108C48008AFD326872487260B260121A9110714AD5
:108C58004A43531C032293FBF2F202EB42029A1A94
:108C6800742303FB02033360C9E16B4B6B4A1B6837
:108C780011688B4206D00AA9002041F8203D1360F4
:108C8800FFF7CCFE019B97F8D6171B8897F8D707F4
:108C98000B44013BB3FBF0F200FB12338B4280F034
:108CA8007981564C0120FFF721FEFFF739FD50204E
:108CB8002668656808F09EFCA268236810681B682F
:108CC800626803441068A3EB400008F044FD6A683A
:108CD80073689B1A0293AA68B3689B1A0393EA689D
:108CE800F36802A89B1A049307F018FC2A693369F1
:108CF8009B1A02936A6973699B1A0393B369AA69F9
:108D080002A89B1A049308F07DFC06F11C0905F1E2
:108D18001C0B1027A0463B4801210368B9401942A3
:108D2800824606D0D9F80000DBF80030C01A08F0F7
:108D380012FD0137132F09F104090BF1040BEAD1D5
:108D480006F1260005F12601002331F9024F30F91A
:108D5800022F121B02AC44F823200133042BF4D158
:108D68000322002702ABBF0053F82230FFB26BB1D9
:108D780003F108010F2902D847F0010706E0803304
:108D8800FF2B94BF47F0020747F0030712F1FF32A9
:108D9800E8D2384608F02EFC00240DF10809A34655
:108DA80007F00302022A10D0032A17D0012A4AD159
:108DB800BBF1000F41D0D9F8000000F00F002043AC
:108DC80008F018FC4FF0000B3DE0BBF1000F0CD091
:108DD800D9F80000C0F3031020432CE0BBF1000FCA
:108DE8001ED199F8010008F005FC99F8000008F078
:108DF80001FC28E0302E002050120020B82C002062
:108E08002C2E0020242E0020202E0020C41F0020FD
:108E1800C42C002035C2724F382E0020342E00207A
:108E2800D9F80000C0F30330204308F0E3FBD9F879
:108E38000000C0F3071008F0DDFBD9F8004024015A
:108E4800E4B24FF0010B09F1040906AB99454FEA6A
:108E58009707A5D1BBF1010F02D1204608F0CAFB44
:108E6800DAF8003013F480541FBFB6F86420B5F860
:108E78006410521A029218BF012499040AD50AAA4A
:108E880002EB8401B5F86600B6F86620121A41F8BC
:108E9800202C01345A0513D502AA02EB840E06F1E0
:108EA8006A0705F16A00002237F9021F30F902CF7C
:108EB800CCEB01014EF822100132032AF4D103341D
:108EC8001F0508D50AAA02EB8400A96EB26E521AD1
:108ED80040F8202C013418040BD50AAB03EB8402AC
:108EE800B5F87210B6F872305B1A42F8203C0134BB
:108EF80000E0F4B1012C03D1029808F02CFC18E032
:108F0800631E002002AA400052F82320C0B20AB112
:108F180040F0010013F1FF33F4D208F06BFB002797
:108F280002AB53F8270008B108F015FC0137A74237
:108F3800F6DB30200321FFF771FC36200321FFF711
:108F48006DFC314B3C201978FFF768FCDAF80030EB
:108F5800990506D5B6F95E00B5F95E30C01A08F075
:108F6800FAFBD8F800202948D8F80430C8F80420BB
:108F7800121A9110264AC8F808304A43531C032293
:108F880093FBF2F202EB42029A1A742303FB0203E8
:108F9800C8F800301F4B1B681A0630D51E4C1F4DF1
:108FA80022682B689A420BD162686B689A4207D193
:108FB800019B1B88102B11D1194B1B885B060DD107
:108FC800482008F017FB206808F0C5FB606808F027
:108FD800C2FB23682B6063686B600EE0114A0F4B7D
:108FE80011782A7C914208D10F4A99681068884202
:108FF80003D15268DB689A4201D0FFF731FC08F0D0
:10900800C9FA0BB0BDE8F08FC41F0020C42C0020A3
:1090180035C2724F582E0020D0110020A42C0020F9
:10902800322E00204A1A00204C1A00202DE9F84F51
:109038000C9E3A4CC2EB030B0B9BF61A6368002993
:1090480014BF4FF0060A4FF0040A01330546904654
:1090580013D1236853455ED2314A324852F823204F
:10906800032B98BF294608F0B3FA6368013363609D
:109078002D4B002205469A7113E0002511E02B4A7A
:109088001278954240DA0B9BE3B109FB06F2995C32
:1090980001228A40264909680A4213D163680133CC
:1090A8006360D4F804900A9B1C4F9945E7DB2BD1E9
:1090B8000A2008F09FFA3B6801333B604FF0FF330A
:1090C8007B6021E0184A917921B12C2008F092FAAE
:1090D800013501E001219171226809FB0BF308EBCE
:1090E800030752B958F8030008F062FA97F9041018
:1090F8004B1C0544D2D00F4802E03A440E4811797F
:1091080008F066FA0544C9E7206850452CBF0020DE
:109118000120BDE8F88F0020BDE8F88F3C2E002024
:10912800148701081BA90108681E002008010020F7
:10913800242E00202AA901085EAA010830B585B0AE
:1091480004AC002524F8025D0091ADF80600214624
:109158001020FFF727FC9DF806002146FFF722FCA8
:109168009DF807002146FFF71DFC9DF800002146E9
:10917800FFF718FC9DF801002146FFF713FC9DF846
:1091880002002146FFF70EFC9DF803002146FFF779
:1091980009FC9DF80E00C043C0B22946FFF702FC47
:1091A80005B030BD10B5054C206802F0BCFC18B104
:1091B800206802F0B5FCF6E710BD00BFC81A002011
:1091C80013B5044601A9006802F0C2FE132002F09C
:1091D800FBFEBDF9040002F0E5FE1B2002F0F4FEE0
:1091E800BDF9060002F0DEFE232002F0EDFE236842
:1091F800002BB4BF53204E2002F0D4FE01A96068B2
:1092080002F0A6FE122002F0DFFEBDF9040002F013
:10921800C9FE1A2002F0D8FEBDF9060002F0C2FE0F
:10922800222002F0D1FE6368002BB4BF57204520EE
:1092380002F0B8FE02B010BDF0B50124B0FBF4F5A1
:109248008D4201D34C43F9E70026D4B1B0FBF4F5C5
:1092580004FB1500B4FBF1F41EB9002D01DC002C51
:10926800F3D1092D03F1010EEFB204DD002A14BF7A
:109278003725572500E030253D441D7001367346DB
:10928800E3E71C70F0BDF0B50124B0FBF4F58D42A6
:1092980001D34C43F9E70026D4B1B0FBF4F504FB45
:1092A8001500B4FBF1F41EB9002D01DC002CF3D13C
:1092B800092D03F1010EEFB204DD002A14BF372592
:1092C800572500E030253D441D7001367346E3E71D
:1092D8001C70F0BD03685A1C0260197070472DE9B4
:1092E800F843089E002B07468846144614BF4FF0E3
:1092F80030094FF02009334613F8012B0AB92546E7
:1093080003E0002CFBDD013CF6E7002D04DD3846C8
:109318004946C047013DF8E724EAE4743546A01BF6
:10932800284415F8011B11B13846C047F7E7BDE8D6
:10933800F883024B186802F0F9BB00BF4810002000
:1093480090ED017A07EE901AB5EE407AF1EE10FA38
:1093580001BFF8EEE77A9FED0E7A67EE877AB7EEEF
:10936800007A04BFC7EE277AC0ED017A90ED017A42
:10937800D0ED007A30EE877A30EE670AC0EE870AC1
:10938800E0EE807AB0EE670AC0ED007A704700BF61
:10939800DB0FC94010B50278202A034600F101000E
:1093A800F9D0092AF7D02D2A03D10346BFEE000AC7
:1093B80004E02B2A08BF0346B7EE000ADFED387A2F
:1093C8001A46134612F8010BA0F13001CCB2092C51
:1093D8000AD807EE101AB8EEC77AF2EE046AA7EEBA
:1093E800A67AF0EE477AECE72E2816D1F2EE046A58
:1093F8001146B0EE666A0B4611F8012B303AD0B22E
:1094080009280AD807EE102AB8EEC77A87EE267A16
:1094180066EE866A77EE877AEDE71A7802F0DF0261
:10942800452A35D15A782D2A02D10233012004E089
:109438002B2A14BF013302330020013B002213F80A
:10944800011F3039CCB2092C03D80A2404FB0212BC
:10945800F5E7B2F59A7F28BF4FF49A721346B7EE34
:10946800007A072B05D9DFED0F6A083B27EE267A2D
:10947800F7E702F007032BB1F2EE046A27EE267A2B
:10948800013BF8E7F0EE476A20B1C7EE877A03E0C0
:10949800F7EE006A67EEA67A20EE270A10BD00BF35
:1094A8000000000020BCBE4C30B52DED028B87B00B
:1094B800B0EE408A0C220021054603A80CF051FCAE
:1094C800B5EEC08ADFED2A7AF1EE10FACCBF38EE9D
:1094D800278A38EE678ADFED277A28EE278A6946D9
:1094E800FDEEC87A17EE904A84EAE470A0EBE470C7
:1094F80009F096F8002CACBF20232D2368468DF880
:109508000C300CF072FC012807D130238DF80D3097
:109518008DF80E308DF80F300CE0022805D130237D
:109528008DF80D308DF80E3004E0032804BF302389
:109538008DF80D30694603A80CF03AFC03A80CF02E
:1095480054FC0338C4B2224603A928460CF07AFC1E
:1095580000232B55284608490CF02AFC03AB284663
:1095680019190CF025FC284607B0BDEC028B30BD5C
:109578006F12033A00007A444EA9010870B50646F6
:1095880015460846B6FBF2F414B12046FFF7F6FF7D
:1095980005FB1464024B1B5D00F8013B70BD00BF66
:1095A80050A901082DE9F04F814689B08A46164630
:1095B8001C4600253178002900F0DD80252902D0DD
:1095C8000136484675E07278302A08BFB278A2F1B1
:1095D800300319BFB71C4FF0000BF71C4FF0010BFD
:1095E800092B4FF0000819D8A2F13003D9B2092984
:1095F80005D80A2202FB083817F8012BF4E7A2F174
:109608006103052B02D8A2F1570305E0A2F141033B
:10961800052B03D8A2F137030A2BEADD6C2A31D1D6
:109628003A78642A07F1010600F083800BD8252ACE
:109638003DD003D8002A00F09E80BBE7582A0CD002
:10964800632A19D0B6E7732A22D002D86E2A37D0F7
:10965800B0E7752A5CD0782AACD1271D2068A2F122
:10966800580462424FF01001624155E02CD9582A43
:1096780032D0632A2AD13E4648462178271DD04752
:1096880001350FE0642A64D00ED9732A14D13E46FE
:10969800236800934846514642460023FFF71FFEC1
:1096A800271D05443C4685E7252ADFD13E46484626
:1096B8002521D04701357DE70AD86E2A06D13E46D6
:1096C800236804341D6075E7002A54D03E4671E7CC
:1096D800752A26D0782AF9D1A2F1580304F1040C8E
:1096E8005A422068CDF80CC04FF010015A4105AB22
:1096F800FFF7A2FDDDF80CC03E46644605AB0093BB
:109708004846514642465B46FFF7E9FD054451E7A6
:109718002068271D0A21002205ABFFF7B4FD3C464F
:10972800ECE704F1040CCDF80CC020680A210022F3
:10973800DDE72068002804F1040708DA2D238DF8F6
:10974800143040420DF115030A210022E5E705AB6C
:10975800FAE72068002804F1040C0ADA2D238DF8B2
:10976800143040420DF11503CDF80CC00A21002237
:10977800BEE705ABF8E7284609B0BDE8F08F0EB4A0
:109788000FB505AB019053F8042B0649039301A8C4
:10979800FFF708FF019B00221A7004B05DF804EB84
:1097A80003B07047DD9200080FB413B50B4904AB42
:1097B80008680B4953F8042B09680193FFF7F2FE78
:1097C8000446084B186802F0A5F90028F9D020468D
:1097D80002B0BDE8104004B0704700BF7C01002013
:1097E800780100204810002080EAE073A3EBE073C2
:1097F8008B4206DB002801DD401A704702D008447E
:10980800704700207047FDEEC07A17EE903A20337B
:10981800402B43D8DFED237AB4EEE70AF1EE10FAD5
:1098280004DDDFED217A30EE670AF3E7DFED1F7A1A
:10983800B4EEE70AF1EE10FA04D5DFED1B7A30EE4C
:10984800270AF3E7DFED1A7AB4EEE70AF1EE10FA29
:1098580004DD30EE670A37EEC00A0AE09FED157A9C
:10986800B4EEC70AF1EE10FA44BF30EE270A37EE1D
:10987800400A60EE007ADFED106A9FED107AA7EEDD
:10988800A67ADFED0F6AE7EE876A9FED0E7AA7EEFC
:10989800A67A20EE276AA6EE070A70479FED0A0A05
:1098A800704700BFDB0F4940DB0FC940DB0F49C0E1
:1098B800DB0FC93FDB0FC9BF9A7C2E36FAAF4FB911
:1098C8003587083CA4AA2ABE00000000DFED027A12
:1098D80030EE270A97E700BFDB0FC93F38B52DEDFB
:1098E800068B90ED008AB0EE480A0C460546FFF755
:1098F800EDFFB0EE40AAB0EE480AFFF784FFD5EDC1
:10990800018AB0EE409AB0EE680AFFF7DFFFB0EECA
:10991800408AB0EE680AFFF776FFD5ED02AAF0EEAE
:10992800408AB0EE6A0AFFF7D1FFF0EE409AB0EE37
:109938006A0AFFF768FF60EE0A6A69EE297AF0EEB4
:10994800665AE7EEA85A29EE8A6A29EE007A69EE85
:10995800889A29EE489A28EE400A28EE0A8AC4ED29
:10996800035AF0EE465AE7EE685AE6EEA87AA6EEF3
:10997800687AC4ED009AC4ED028A84ED059A84EDF4
:10998800088ABDEC068B84ED010AC4ED045A84ED07
:10999800067AC4ED077A38BD10B52DED048B8AB070
:1099A80090ED009AD0ED028A90ED018A04460846AF
:1099B80001A9FFF793FFDDED047A9DED017A68EECA
:1099C800277AE9EE077A9DED077AE8EE877A9DED2A
:1099D800027AC4ED007ADDED057A68EE277AE9EEC1
:1099E800077A9DED087AE8EE877AC4ED017ADDED15
:1099F800067A28EE278ADDED037AA9EE278ADDEDBF
:109A0800097AA8EEA78A84ED028A0AB0BDEC048B15
:109A180010BD074B1A8822EA0000904210B5188042
:109A28001C4602D0012001F0AFFE208810BD00BF07
:109A3800081B0020064B1A881043904210B5188066
:109A48001C4602D0012001F09FFE208810BD00BFF7
:109A5800081B0020024A936823EA000090607047C0
:109A68005012002008B5104B1A780023D9B2914241
:109A780007D20E4951F82310096800200860013305
:109A8800F4E7322001F0BFFE094B1B685A0309D5E1
:109A9800084B9B685B0305D440F2DC50BDE80840E6
:109AA80001F0B1BE08BD00BFC41F0020941F0020F4
:109AB800582E0020501200202DE9F743484F494AFC
:109AC8004B233B706923137040F2DC735380BE2331
:109AD8001371EF2382F8D937002382F8DA37194651
:109AE8001646F25C0133514040F2DC729342F8D1E1
:109AF8003C4B83F8DA173C4B1A69120604D53B4AEB
:109B08005A6002F188325A604FF00408002008F1C8
:109B1800FF3818F0FF0850D0334B3422DA600024A5
:109B280044B1002356F80490019306F071FD04280F
:109B3800EDD117E006F06CFD0428E8D12A4D2B6919
:109B480043F002032B612A4B6B612B6943F04003FE
:109B58002B6106F05DFD2B69042823F002032B61BD
:109B6800DFD0D4E7204D2B6943F001032B6104F1CA
:109B7800006303F57E331FFA89F21A8006F048FD68
:109B8800042810D11B4B23440193019B4FEA194928
:109B9800A3F8009006F03CFD2B69042823F001038C
:109BA8002B6105D0B3E72B6923F001032B61AEE7E6
:109BB800043440F2DC739C42B2D10B4A1369042886
:109BC80043F08003136102D107F01AFA10B90A2092
:109BD80001F05EFF02233B7003B0BDE8F08300BFD5
:109BE800950E0020501200200020024023016745F6
:109BF80000F8030802F803082DE9F84307F000FA13
:109C080010B90A2001F044FFB24CB34EB349B44D29
:109C18004B2340F2DC72204633700CF097F894F82E
:109C2800B037022B84BF002384F8B03794F8B027EC
:109C38004FF4CC7101FB02F303F53A70234420443E
:109C4800286093F83C0303F54E73022801FB024297
:109C580084BF0020187192F83C33A24A13700C227A
:109C680002FB0343A04A03F2B2731360A36846F2EF
:109C780009021A401AB9974A43F400539360A3683B
:109C8800D80703D54FF40050FFF7E4FEA368590442
:109C980009D50820FFF7DEFE4FF40050FFF7DAFE83
:109CA8000120FFF7D7FEA3681A0706D54FF4005026
:109CB800FFF7D0FE0120FFF7CDFEA3689B0402D575
:109CC8004020FFF7C7FE94F8E021824B2AB193F8B1
:109CD800E42112B1002283F8E421844B844F1F60F1
:109CE8004FF00008C64604EB0803B3F8F8C14FEA82
:109CF8005C0101F077314FEA9C0303F03333C1EB89
:109D08000C00C11A4FEADC0303F01133CB1A03EB42
:109D180023131CF0010903F00F324FF0FF0392FBED
:109D2800F3F3C3EB032318BF0EF1010EA2EB0303F9
:109D380018BF5FFA8EFE012B0ADD022B40F0C780A8
:109D4800B9F1000F00F0C3801CF0BC0F00F0BF8019
:109D580008F10808B8F1200FC5D10EF1FF3EBEF199
:109D6800010F00F2B48007F027F930220021614882
:109D7800DFF8F4810BF0F5FF5F4BD5F80090C3F8DE
:109D880000805E4B002109F17900C3F8009001F0D2
:109D980071FC5B4B80F0010018705A4B08F12602E9
:109DA8001A60594B08F1D4021A6099F8000005F0BE
:109DB80041FD2868554B00F5C5721A60FDF768FD2E
:109DC800534B94F8D801DFED536A08F194021A60F6
:109DD8006421514BC82211FB00225A6000229A606C
:109DE800DA601A615A619A61DA6183F8202083F88F
:109DF80021204A4B08F12C021A602B68484A93ED3F
:109E0800187A03F219111160464A03F28911116098
:109E1800454A08F108011160444AC2F80080444AE2
:109E280008F1A0011160434A08F1AA0111604249F2
:109E380067EE266A0F60B4F86611B6EE007A07EE90
:109E4800901A87EE267AB4F86811101DF8EE677A32
:109E5800C2ED027A07EE901A93F85C10117193F82C
:109E68007810517194F8E3111174F8EE677AB3F829
:109E78001611C2ED037A07EE901A30490860536153
:109E88002F4A03F1640111602E4A2F4982ED007AAE
:109E9800F8EEE77A9FED2D7A2D4A0B60C7EE277A08
:109EA8002C499FED2D7A67EE877AC2ED007A03F18F
:109EB80068020A60294903F211130B60284BC3F8A2
:109EC8000080284B1A6002233370BDE8F88306F03F
:109ED80073FB48E750120020950E002000F8030895
:109EE800A4110020502B0020C8110020B42F0020FE
:109EF800DA1300204C0F0020800F0020840F002070
:109F0800030000206428002070060020900F002025
:109F1800002F0020DB0F4940DC2E0020C028002045
:109F28008C210020C00900209020002094200020CF
:109F3800D4080020701E002098090020F428002072
:109F48002C29002028290020FC070020000061445B
:109F5800D0080020F00700204C3D0F44C008002026
:109F6800C8080020FC0600209413002008B5FFF75D
:109F7800A3FDFFF741FE0120BDE8084001F004BC45
:109F880008B508480BF031FFC0B209280246054B56
:109F980004DC01302021C0B29954F6E700221A549B
:109FA80008BD00BF1921002008B507480BF01DFFA8
:109FB800C0B21428044B04D8421C20211954D0B232
:109FC800F7E700221A5408BD192100202DE9F74FA0
:109FD800A74C01F0F1FB26686568A768861BF64365
:109FE800451BC71BED43FF43F60F8046ED0FFF0FE0
:109FF8002EB93FB9002D00F08682B9462CE04FF00B
:10A00800000929E0B14627E003EB8A0BBBF80230D0
:10A018001A050ED413F4805F1DBF964A9BF80110F1
:10A028001268954A954B14BF52F82120126843F8DC
:10A038002A20BBF80230D80516D499050AD5904BCA
:10A048001B7813F0040F0CBF8E4A8F4A8B4B126893
:10A0580043F82A2009F10109207B8C495FFA89FA23
:10A0680082450B68D0D326E0894A5046594605F008
:10A0780005FC884B1B885A0603D550465946864A24
:10A0880016E0580703D550465946844A10E0190788
:10A0980003D550465946824A0AE09A0703D55046E6
:10A0A8005946804A04E0DB07D4D57F4A50465946D2
:10A0B80005F0E4FBCEE7DFF808E20093BEF90630CE
:10A0C8007822A3F57A7353434FF47A7293FBF2F331
:10A0D80003F22B1301930022F3465FFA82FE8645B2
:10A0E80017D2009B03EB820EBEF802E01EF4806FCD
:10A0F8000DD0DFF88891019B39F822E040F2671A09
:10A108009E449EFBFAFC0AFB1CEE29F822E0013271
:10A11800E3E74DB308F5C333A0336360637B544A68
:10A1280013BB9373614B1B6813F0020F0AD0DFF85F
:10A1380094E19EF800E0BEF1000F03D04FF0010E4D
:10A1480082F80EE0DA0506D5594BDB781BB1A37B04
:10A1580043F00203A3734A4B1B7813F0050F02BFA9
:10A16800A37B43F00403A37394F80EE0BEF1000F41
:10A1780003D13F4B5B7B002B4FD094F80DC01CF0F4
:10A18800010FACF10C031DD1BCF1030F07D8DFF8A8
:10A19800E8903C4A1EF0040F08BF4A4600E0364AE1
:10A1A800ACF1040CBCF1070F05D8DFF81CC11EF098
:10A1B800010F18BF6246DBB2032B0ED81EF0020F48
:10A1C8003C4B06E0DBB2032B06D82F4B2A4A1EF085
:10A1D800020F18BF1A4600E0274A4FF0000C5FFA3A
:10A1E8008CF383420DD20B6803EB8C035B881B0650
:10A1F80042BF224BD2F8009043F82C900CF1010C8E
:10A20800EDE785B1BEF1000F08D0637B184A013332
:10A21800DBB2142B06D1002304E025B1637B002BAD
:10A22800F3D100E05373002E52D0234AB2F9025002
:10A23800B2F90020002DB8BF6D42002A4FF032035A
:10A24800B8BF524295FBF3F592FBF3F2EDB2D3B2ED
:10A25800AB4238BF2B46194A13B192FBF3F300E027
:10A26800134643442360E37B014A7BBB01232EE072
:10A27800881E00208821002080A401080A0E0020E2
:10A28800EA2F002014A1010804A10108902700204A
:10A298002C870108081B002032870108388701082D
:10A2A8003E870108448701084A870108582E002084
:10A2B800DC2E00201CA1010848120020400D0300DC
:10A2C800942E0020901A002024A101080023D373A3
:10A2D8008E4D8F4B2D78E27BADB9002F00F00E81AB
:10A2E8008C4B267B1A788C4B8C4D93F800C08C4B8A
:10A2F800D3F800E00B6802F004020021D2B203EBAD
:10A3080086060F46B5E01AB9864A1A61002508E0A4
:10A31800854AFAE70A68AB00D6187688760604D428
:10A328000135EBB28342F5D3D7E7804EB6F900602A
:10A33800192E25DD12F803E094F814C026690EF0F2
:10A348000F09E1450CDCDFF8C8C19CF815C0BCEB6F
:10A358001E1FDEBFDFF8D8E1D6F800C043F80EC0F4
:10A3680012F803E094F816C00EF00F09E14533DB4C
:10A37800DFF89CC19CF815C0BCEB1E1F2CDC26E046
:10A38800193629DA12F803E094F814C026690EF099
:10A398000F09E1450CDCDFF878C19CF817C0BCEB6D
:10A3A8001E1FA2BFDFF888E1D6F800C043F80EC030
:10A3B80012F803E094F816C00EF00F09E1450BDB24
:10A3C800DFF84CC19CF817C0BCEB1E1F04DBD6F8A5
:10A3D80000E0574E43F806E0544EB6F90260192ED5
:10A3E8001BDD12F803C094F814E026690CF00F097D
:10A3F800F1450CDCDFF8189199F81590B9EB1C1FA2
:10A40800DEBFDFF82CC1D6F8009043F80C90D25C80
:10A4180002F00F0CF4451EDD82E7193680DA12F8D7
:10A4280003C094F816E026690CF00F09F1450CDB1F
:10A43800DFF8DC9099F81590B9EB1C1FDEBFDFF848
:10A44800F0C0D6F8009043F80C90D25C02F00F0CE4
:10A45800F445FFF665AF94F817E0BEEB121FA2BFF4
:10A46800334A36689E505BE75888000504D40433A5
:10A478000435B342F8D122E04AB101EB0C0A0620B8
:10A488009AFBF0F900FB19A001280DDC01E057B98F
:10A49800012793F801900EEB89003EF829A090F867
:10A4A8000290C07803E017460020814682460131B9
:10A4B80025F802AC85F800906870C9B2D7E7164A4B
:10A4C8001378013B13F0FF0308BF06231370114BE9
:10A4D8001B785B0741BFBBF90630A3F57A7303EB22
:10A4E800C3034FF47A7243BF93FBF2F30133DBB239
:10A4F8000123104A92FBF3F34344A36003B0BDE881
:10A50800F04FFAF72BBB03B0BDE8F08FBB0E00206D
:10A51800881E0020EA2F00203A0000200C0E0020A0
:10A528008821002020A1010880A4010848120020E9
:10A538000A0E0020400D03002DE9F04F2DED0A8B87
:10A5480089B08046059390F85030049102921BB16F
:10A55800322BA8BF322300E0012307EE903AF8EE31
:10A56800E7BADFEDA87AA84B9FEDA8CA1B88C7EE0B
:10A57800ABBA002B08BF012307EE903AB8EEE7AA62
:10A58800A34B03932AEE0CCA1A887BEE8CBA12F0FE
:10A59800020FCCEE2BBA27D09E4AB2F90030B2F99E
:10A5A800022083EAE37182EAE270A1EBE371A0EB97
:10A5B800E27088420446B8BF0C46B4F5E17F16DA6B
:10A5C80088429FED95BA05DD002AD8BF524207EEB2
:10A5D800902A04E0002BD8BF5B4207EE903AF8EED1
:10A5E800E77A87EE8BBA04E09FED8CBA01E0B7EE0C
:10A5F80000BADFF858A2DFED899ACDF804800AF195
:10A60800080B0AF110070AF11C090024F0EE69AAE8
:10A61800834931F914307F4909EE103AB8EEC99AE6
:10A6280031F91430F5EE047A29EE279A08EE103A3B
:10A63800039BBDEEC99A1988F8EEC97A9FED799AFD
:10A6480089074FEA440627EE899AB8EEC88A00F0CF
:10A658008180754931F9143007EE903AF8EEE77ABF
:10A66800B0EE007AE8EE077A029B5842FDEEE77AF0
:10A6780017EE901A814203DB8B42A8BF0B4618469F
:10A688006A49059B715E401A33F91410084407EEB5
:10A69800900AF8EEE78A07F0D5FF48B16449F2EE70
:10A6A800049A88EEA90A085D07F080FD60EE298A01
:10A6B80098F81C30DFED5F6A0AEE903A98F8083097
:10A6C80007EE903AF8EE677AF8EE6AAA68EEA77A8B
:10A6D800B1EE047A67EEA67A2AEE877AFDEEE77A7B
:10A6E80017EE901AF1EE477AFDEEE7AA1AEE903AC5
:10A6F800994208DBFDEEC7AA1AEE903A8B42A8BF32
:10A708000B460AEE903AD9ED007AE8EE8C7ABBEE69
:10A718000E7AF4EEC77AF1EE10FAF8EEEAAA09D446
:10A72800B3EE0E7AF4EE477AF1EE10FAC8BFF0EE07
:10A73800477A01E0F0EE477AC9ED007A98F81230CE
:10A7480009EE903AF8EE699A67EEA97ADFED3A9A3F
:10A7580067EEA99A039B1988CA0779D43048305EF6
:10A768000028B8BF4042B0F5206F02DD00203860F5
:10A7780026E0019B9FED317A5B7868EE077A07EE59
:10A78800103AB8EE477A87EE877AD7ED007A37EE37
:10A79800497AE7EE0C7A9FED2A7AF4EEC77AF1EE61
:10A7A80010FA09D49FED277AF4EE477AF1EE10FA01
:10A7B800C8BFF0EE477A01E0F0EE477AC7ED007ABD
:10A7C800019BD7ED007ADB7A08EE903AF8EE688ABA
:10A7D8008B0768EEA77ADFED1C8A67EEA88A3BD55F
:10A7E80038EE6A8AF0EE6A7AEBEE087A78EEE98A51
:10A7F800B0EE678AF0EE697AEBEE287AF0EE678AB7
:10A808002AE000BF83F9223E5C110020BD3786355F
:10A81800081B0020481200200000E143000000004F
:10A8280088110020CDCC4C40E22F00204E2E002075
:10A83800689001086F12033C0AD7A33D0000A043AB
:10A84800000040C3000040430AD7233CA01E00205C
:10A85800F0EE698AB0EE6A8A89499FED8A7A635C6C
:10A8680098F8511007EE903AF8EEE77A67EEC97A51
:10A87800A7EE878A59B18448844DB0EE480A00EBA8
:10A88800C400D5ED000AFEF75BFDB0EE408A9AEDF4
:10A89800007ADBED007A7E49AAEC019A39EE477A14
:10A8A800635C7C4D87EE0C7A043709F1040909EEE4
:10A8B800103A37EE677AB8EEC99AEBEE877A38EE37
:10A8C800280AEBEC017A67EE897A9FED739A27EEF6
:10A8D800899A30EE490A0BF053FCBDEEC88A6F49DD
:10A8E800A85318EE103AFDEEE88AB1EE499A18EE30
:10A8F800902A41F82430BDEEC99A694B694E43F855
:10A90800242019EE102A46F82420019A06910132D3
:10A91800019207930CB901247AE6049A624B947960
:10A92800B3F90430640028345C43604BB3F9043055
:10A9380000EE103ABAEECF0A0BF022FC6411201A8E
:10A94800002C07EE900AB8BF6442322CF8EEE76A92
:10A95800574A02DD0023936026E0BDEECAAA1AEE2C
:10A96800103A23F0030307EE903AB8EEE7AADFEDBA
:10A97800517A98F80D30CAEE277A07EE103AB8EEF9
:10A98800477A936826EE877A67EE277AFDEEE77AAC
:10A9980017EE901A0B4448498B42A8BF0B4647490B
:10A9A8008B42ACBF9360916093685B13B3F5807F73
:10A9B800A8BF4FF480736FF0FF029342B8BF1346ED
:10A9C80007EE903AF8EEE78AFDEEE67A98F803206B
:10A9D80017EE903A53439B1107EE903A384B1B7889
:10A9E800032BB8EEE78A14D9B8F84E20B2F5FA7FEF
:10A9F8000FD2FDEEC87A534217EE901A994204DB43
:10AA0800914217EE903AA8BF134607EE903AB8EE77
:10AA1800E78A98F8511081B14B0803D09942A8BF32
:10AA2800194600E00121194B2648D3ED000AB0EE83
:10AA3800480AFEF785FCB0EE408A78EE287AFDEEEB
:10AA4800E77ACDED017ABDF80430AB801BB200EE99
:10AA5800103AB8EEC00A0BF093FB069BA880BDEE37
:10AA6800C88AFDEEE88A83ED028A079BC3ED028A55
:10AA78000023B36009B0BDEC0A8BBDE8F08F00BFBE
:10AA8800C41E0020A69B443BBC270020D4270020DE
:10AA9800C71E002020280020F7CC92382828002044
:10AAA8003428002040280020481200208811002067
:10AAB800D827002000803B45FEFFFF0F020000F072
:10AAC800C41F0020CC2700202DE9F04F2DED028B6C
:10AAD80087B000260493C14B0391B3F90280B3F900
:10AAE80000300292B8F1000FB8BFC8F10008002B7F
:10AAF800B8BF5B429845B8BF9846B8F5FA7F074695
:10AB0800A8BF4FF4FA780090B2460196B146344691
:10AB1800B34D2B88990757D0B04BB24A33F814304D
:10AB280032F91420022013FB0022029B5B429A4256
:10AB38004FEA440103DB029B9342A8BF1346AA4A8B
:10AB480031F902B0049A32F91420CBEB030303EB7A
:10AB5800020B07F077FD88B107EE90BAA34BB8EE69
:10AB6800E70AB2EE048A185D80EE080A07F01EFBB9
:10AB780020EE080AFDEEC07A17EE90BA3B7A6422FE
:10AB880003FB0BF393FBF2F33A7F6FF0040909FB25
:10AB980002F94B4504DB02EB82099945A8BF9946A7
:10ABA800934A52F824100BEB010342F210718B42C6
:10ABB800A8BF0B468F498B42B8BF0B4642F82430DA
:10ABC800BA7C53431B1301932D8805F00303012B13
:10ABD80038D0824B884933F914A0009B51F824E0FF
:10ABE80093F801C0854B33F9140080EAE073A3EBB6
:10ABF800E073B3F5206F4FEA840616DC0AEB8A038C
:10AC08001A0192FBFCF3042290FBF2F0181A864416
:10AC1800BEF57A5FA8BF4FF47A5E794B9E45ACBF0C
:10AC280041F824E041F8243002E0002341F82430C0
:10AC38008B597D2693FBF6F6009BDB7A73434026FF
:10AC480093FBF6F6AA0711D50198C8F5FA7208FB26
:10AC58000AF308FB06F54FF4FA7102FB093302FB0D
:10AC6800005593FBF1F395FBF1F505E0EB074DBFBC
:10AC7800019D354653464B46604A32F9141004226A
:10AC880091FBF2F25F49615C4A436FF04F0192FB1E
:10AC9800F1F297F8511013444FEA440B08EE103ABA
:10ACA80059B1594B5948D3ED000AB8EEC80A00EB20
:10ACB800C400FEF745FBBDEEC08A504B544A3BF832
:10ACC80003003BF902302BF8020001B2101D0C32D0
:10ACD800CB1A50F824E0042193FBF1F152F8243008
:10ACE80040F8241073440B4497F8501042F824E0BD
:10ACF8004FEA840C00EE103A79B1434A4548D2ED48
:10AD0800000ACDF814C0B8EEC00A00EBC400FEF784
:10AD180017FBDDF814C0BDEEC00A3F4A3F49125D7B
:10AD28003F4810EE103A5343202293FBF2F318EEFB
:10AD3800102A2A44D21A2BF8012018EE102A4CF8AF
:10AD48000020384A4CF80250374D5B424CF8053029
:10AD5800009B013300930CB90124D9E61F4B97F8E7
:10AD68000DE0B3F90440039B9B790F335B00634309
:10AD78005B11224C002B4FF00406B4F9044094FBFD
:10AD8800F6F41D4EA3EB0404B8BF5B42322BD6F891
:10AD980008C00DDC254B0EFB04CE7345A8BF7346D7
:10ADA800DFF890E07345ACBFB360C6F808E001E097
:10ADB8000023B360FB785C431D4B1B78032B4FEAE1
:10ADC800A4143AD9B7F84E30B3F5FA7F35D25F42BA
:10ADD800BC4231DB9C42A8BF1C462EE04812002032
:10ADE800081B0020E22F00204E2E0020689001084A
:10ADF800CC1E0020F0D8FFFFD827002088110020A3
:10AE080080C1FFFFC41E0020D4270020BC270020DB
:10AE1800D41E002008280020C71E0020202800205B
:10AE2800282800203428002040280020FEFFFF0F9B
:10AE3800C41F0020020000F03C46B368846043F35E
:10AE48004F33B3F5807FA8BF4FF480736FF0FF06D0
:10AE5800B342B8BF3346E618936000238E80AB60D8
:10AE680007B0BDEC028BBDE8F08F2DE9F04F2DED5A
:10AE7800028B85B083460293B84B01911D880092DE
:10AE880005F00205ADB295B1B54BB3F90250B3F96F
:10AE98000030002DB8BF6D42002BB8BF5B429D4209
:10AEA800B8BF1D46B5F5007FA8BF4FF40075D94659
:10AEB8000026AB4BAB4C33F81610AB4B54F826704E
:10AEC80033F9163083EAE37EAEEBE37E08B2BEF5D3
:10AED800206F4FEA460A4FEA40004FEA860812DC24
:10AEE8004FF0040E93FBFEF3C31A1F44B7F57A5FC5
:10AEF800A8BF4FF47A579D4B9F42ACBF44F82670C9
:10AF080044F8263002E0002344F8263054F808704C
:10AF180099F80B3099F80140FF115F438F4B1B885C
:10AF280044439B074FEAA7174FEAA41456D0904B07
:10AF380033F90A30022011FB0031009B5B42994231
:10AF480003DB009B8B42A8BF0B468A493AF90110E4
:10AF5800591A029B33F91630CB1808EE103A07F04D
:10AF680071FB68B1B8EEC80A834BB2EE048A80EE72
:10AF7800080A985D07F01AF920EE080ABDEEC08AA3
:10AF88007E487F4958F8003018EE102A42F2107EA9
:10AF980013447345A8BF73468B42B8BF0B4648F8A5
:10AFA80000309BF808109BF81C00514300EB800010
:10AFB800C911C0F1000E714503DB8142A8BF0146EB
:10AFC8008E469BF812104B431B13FF1ACEEB04045A
:10AFD8006F436C4303EB67270EEB6424624B042139
:10AFE8003AF9030090FBF1F16648805D4143A4EB18
:10AFF800A1129BF8511008EE102A69B16248634CFF
:10B008000393B8EEC80A00EBC600D4ED000AFEF7B9
:10B0180097F9039BBDEEC08A5D4933F80A303AF9C7
:10B0280001002AF801300FFA83FEC0EB0E0E04204F
:10B038009EFBF0F001F1040E0C3158F80E4058F860
:10B04800013048F8014023449BF8501048F80E009E
:10B05800034400EE103A59B14C4B4E48D3ED000A68
:10B06800B8EEC00A00EBC600FEF76AF9BDEEC00AEA
:10B0780049494A48895D4A4C10EE103A18EE102AA0
:10B088004B435B11D119C91A2AF8001048F804205B
:10B098004449454A48F801705B4248F8023009F1D2
:10B0A80001090EB9012604E72D4B2E4EB3F90450C1
:10B0B800019BD6F808E09B790F335B006B435B116B
:10B0C800294D002BB5F904504FF0040795FBF7F70D
:10B0D800A3EB0707B8BF5B42322B9BF80D500BDC84
:10B0E800324B05FB07E5AB42A8BF2B46304DAB42C0
:10B0F800ACBFB360B56001E00023B3609BF80350B8
:10B1080005FB07F32B4D2D78032D4FEAA3130CD91C
:10B11800BBF84E50B5F5FA7F07D26F42BB4203DB4E
:10B12800AB42A8BF2B4600E03B46B568A36045F399
:10B138004F35B5F5807FA8BF4FF480756FF0FF06D7
:10B14800B542B8BF35465E19002386808D6093608E
:10B1580005B0BDEC028BBDE8F08F00BF081B0020D6
:10B1680048120020D82700208811002080C1FFFF46
:10B17800E22F00204E2E002068900108CC1E0020EF
:10B18800F0D8FFFFC41E0020BC270020D4270020D1
:10B19800E81E002008280020C71E002020280020C4
:10B1A800282800203428002040280020FEFFFF0F18
:10B1B800020000F0C41F00202DE9F04F2DED028B96
:10B1C80087B000260493B24B0392B3F90270B3F927
:10B1D80000300190002FB8BF7F42002BB8BF5B4200
:10B1E8009F42B8BF1F46B7F5FA7F8146A8BF4FF404
:10B1F800FA77B0460296B3463446A64D2B8899078F
:10B208005BD0022C59D0A24BA34A33F8143032F940
:10B218001420022013FB0022039B5B429A424FEA50
:10B22800440103DB039B9342A8BF13469B4A31F9B1
:10B2380002A0049A32F91420CAEB030303EB020AB2
:10B2480007F000FA88B107EE90AA954BB8EEE70A26
:10B25800B2EE048A185D80EE080A06F0A7FF20EE19
:10B26800080AFDEEC07A17EE90AA99F80830642211
:10B2780003FB0AF393FBF2F399F81C206FF0040B1D
:10B288000BFB02FB5B4504DB02EB820B9B45A8BF73
:10B298009B46844A52F8243042F2107153448B4240
:10B2A800A8BF0B4680498B42B8BF0B4642F82430F2
:10B2B80099F8122053431B1302932B8803F00302BF
:10B2C800012A01D1022C3FD17848714A30F9140083
:10B2D80032F914807649019A51F824E0567880EAC8
:10B2E800E075A5EBE075B5F5206F4FEA84021EDC2A
:10B2F800022C16D008EB8801090191FBF6F604210F
:10B3080090FBF1F0361AB644BEF57A5F6849694891
:10B31800A8BF4FF47A5E8645ACBF42F801E05050B2
:10B3280007E088EAE875A5EBE875642DE2DD002002
:10B3380088505F497D26525892FBF6F6019AD27AD8
:10B348007243402692FBF6F69A0713D5022C11D0C9
:10B358000298C7F5FA7307FB06F507FB08F203FB2B
:10B368000B224FF4FA7103FB005392FBF1F293FBAB
:10B37800F1F508E0DB0704D5022C02D0029D5A46FD
:10B3880001E035464246494B33F91410042391FB3A
:10B39800F3F34949615C4B436FF04F0193FBF1F3C1
:10B3A80099F85110D3184FEA440A08EE103AB1B18F
:10B3B800022CB8EEC80A414B08D14A0803D0914282
:10B3C800A8BF114600E001213D4802E03D4800EBDE
:10B3D800C400D3ED000AFDF7B3FFBDEEC08A334BBE
:10B3E800394A3AF803003AF902302AF8020001B261
:10B3F80002F108001432CB1A50F824E0042193FB20
:10B40800F1F152F8243040F8241073440B4499F8B1
:10B41800501042F824E04FEA840C00EE103A79B15B
:10B42800264B2A48D3ED000ACDF814C0B8EEC00A5E
:10B4380000EBC400FDF784FFDDF814C0BDEEC00AC0
:10B44800234A2449125D10EE103A5343202293FBFD
:10B45800F2F318EE102A2A44D21A2AF801201E4ABA
:10B4680018EE101A4CF802101C4A4CF802501C4AEC
:10B478005B424CF80230019B01340133032C0193E9
:10B488007FF4BBAE07B0BDEC028BBDE8F08F00BF08
:10B4980048120020081B0020E22F00204E2E00201A
:10B4A80068900108CC1E0020F0D8FFFF881100200A
:10B4B800D827002080C1FFFFC41E0020D427002009
:10B4C800CC270020BC270020FC1E002008280020D4
:10B4D800C71E00202028002028280020342800200B
:10B4E8004028002010B5084B1968002201EBC20360
:10B4F80093F90240844201D1981C10BD0132042AFC
:10B50800F4D1002010BD00BF1C2B002038B14388A7
:10B5180011EA030003D08B420CBF012002207047C0
:10B5280030B50A4B0A491C680A78032A0AD8134618
:10B5380004EBC303551CEAB29D882842F5D00A7073
:10B54800981C30BD0A70002030BD00BF1C2B0020A5
:10B558001C1F0020014B00221A70E1E71C1F00206D
:10B568002DE9F047877890F803C0214DBBB2C7F1A9
:10B57800640E03EB83065C42C3F178005FFA8EFE2B
:10B588007600CCF16408A4B280B2A3B20FFA83F9B2
:10B59800B9F1000F05DC002B14BFBA464FF0010AC1
:10B5A80000E0F24613FB03F303FB0CF21AFB0AF369
:10B5B80092FBF3F3434403FB09F30A2293FBF2F3F0
:10B5C80033449BB225F8023FB1F800904A880A3408
:10B5D800C9EB020AA4B21AB202FB0AF24FF47A7358
:10B5E800844292FBF3F34B442B80CED1BDE8F08725
:10B5F8001C1F002010B544780078002202FB02F3DB
:10B60800193B634303F6C413534340F6C411434341
:10B6180093FBF1F3034921F812300132072AEDD1E7
:10B6280010BD00BF361F00200430114B33F9100045
:10B63800B0F5617F10B506DB40F633039842024649
:10B64800A8BF1A4601E04FF461720C78192340F242
:10B65800833013FB0404944207DA497813FB01038F
:10B668009342B4BF0020012010BD002010BD00BFD0
:10B67800942E002010B500F1500302788A4203D1BD
:10B688008478C278944204D304309842F5D10020DB
:10B6980010BD012010BD0B4B1B6813F4805F0A4BD3
:10B6A800B3F9063005D0C089421A934207DD084431
:10B6B80000E0008A8342B4BF0020012070470120C7
:10B6C800704700BF582E0020942E00201FB5094B4C
:10B6D8001B681B030AD58DF8040001230D2001A95E
:10B6E8008DED030A8DF80530FDF798F905B05DF882
:10B6F80004FB00BF582E00201FB5084B1B681B0316
:10B7080009D58DF80400029100230D2001A98DF8B8
:10B718000530FDF783F905B05DF804FB582E0020CD
:10B7280010B5064B00241C7007F0B0FA044B83F8E0
:10B738002840DC621C865C6310BD00BFB82F002067
:10B748001C1F002010B510B9BDE81040E8E7002321
:10B758000C225A430A4C1119125D824203D001335C
:10B76800102BF5D110BD074B586B18B14A784078AB
:10B77800824203D2002259631A86DA6210BD00BFE2
:10B788002C9101081C1F002010B540001428A8BFE8
:10B7980014200023074A022199540B4499181424B1
:10B7A800834201F8014CF5DBFF21D1540F20BDE89D
:10B7B8001040C7E77C2B002010B50A4A0A4B1168D5
:10B7C8009B6800BF12689142F7D1084A946B4FF406
:10B7D8007A7000FB04F2D31AB3FBF4F300FB0130D8
:10B7E80010BD00BF7C2E002010E000E01C1F0020D0
:10B7F80038B50446FFF7E0FF0546FFF7DDFF401BBD
:10B80800A042FAD338BD10B504462CB14FF47A7073
:10B81800FFF7EEFF013CF8E710BD2DE9F04F87B0C8
:10B8280088469DF8444011461A469DF840308146A6
:10B8380000250C206843814E87198057484505D15B
:10B8480097F808A0BAF1000F04D0F3E00135042DF1
:10B85800EFD1EFE0B9F1010F00F0DA8006DCB9F1C1
:10B86800000F40F0E78000947548D6E0B9F1020F68
:10B8780000F0D180B9F1140F40F0DC80714FBB6942
:10B8880043F00103BB617B694FF0904443F40033FC
:10B898007B61012603224FF4805B04A94FF090409E
:10B8A8008DF815200392CDF810B08DF814608DF83E
:10B8B80016608DF817A0FCF703FEA4F828B0C8207E
:10B8C800FFF7A1FFC4F818B07B69039A43F400336B
:10B8D8007B6120464FF4C0534FF0020B04A9049338
:10B8E8008DF815208DF814B08DF816A08DF817A0D6
:10B8F800FCF7E6FD636A23F470436362636A43F40A
:10B9080060436362636A23F470236362636A43F487
:10B91800602363624C4B4D4C4FF480221A6002F155
:10B928008042A2F53F321223E366082384F871307F
:10B93800136884F8726023F480231360536823F437
:10B948008023536094F8703003F1804303F5823309
:10B958001A6842F480221A60E26E3D4B22F01F0002
:10B9680002F01F02C15806FA02F221EA0202C2508E
:10B97800E26E384922F01F0002F01F0250F801E081
:10B9880006FA02F22EEA02024250E26E22F01F018B
:10B9980002F01F02C85806FA02F20243CA502E4BA0
:10B9A8002E4AC3F800A0FB6943F40003FB612C4B4B
:10B9B80004A8DA608DF810908DF811B08DF812A0F7
:10B9C8008DF8136006F0A8FB2A238DF810309DF837
:10B9D80013308DF811608DF812A01BB104A806F081
:10B9E8009BFB04E01F4B4FF48062C3F884201E4A7F
:10B9F8001E4B136002221A721D4A1E4B13601E4A08
:10BA08001E491B68116098471D4BE3631D4807E0FA
:10BA180000941D4801E01D48009401F05BFE48B108
:10BA2800064B80F804900C2202FB053585F8088047
:10BA3800686000E0002007B0BDE8F08F202B0020F0
:10BA48000038014000100240140401401C1F00206F
:10BA5800080401400C040140D80042420005FA05E0
:10BA680000ED00E000E100E00C2A0020102A002090
:10BA7800A0270020A80000209C2700203C000020D0
:10BA880050870108581F002000440040004800402B
:10BA980038B5134B202240F2DB151A856843102273
:10BAA8009A61851E0B24013C14F0FF0411D00C4A46
:10BAB800938A9BB283F020039382938A9BB283F08C
:10BAC800100328469382FFF79EFE1920FFF79BFE7E
:10BAD800E9E7044B044A1A60044B054ADA6038BDAA
:10BAE80000040048FC9F0020EFBEADDE00ED00E042
:10BAF8000400FA05024A136801331360704700BF57
:10BB08007C2E0020024B5B6F03B11847704700BFC3
:10BB18001C1F002003681B6918470368DB68184767
:10BB280003689B68184703685B68184703681B68C5
:10BB380018472DE9F84FB0F90230934218BF002397
:10BB48002DED028B18BF0370057804460E4691460A
:10BB5800002D40F08B8007EE902A9FED770AF8EED3
:10BB6800E77AB6EE008A27EE800ADFED747A20EED7
:10BB7800270AA04620EE080A0AF078FBDFED706A73
:10BB880060EE266AB7EE006AB0EE667AA0EE007A3A
:10BB980040F2DC536365D0EE006A1023A4F85230FB
:10BBA80037EE067A76EE866AC6EE077A1823A4F888
:10BBB8005030274684ED046A27EE807A27EE007A13
:10BBC80077EE075A84ED017AC4ED025A70EE005AF6
:10BBD80084ED037AB8EE007AA5EE807A27EE877AAC
:10BBE80067EEA67A84ED057AC4ED067ADFED557A1C
:10BBF80098ED047A27EE277AF0EE678AB5EEC07AD8
:10BC0800F1EE10FA4CBF77EE487A77EE087A0135F4
:10BC180017EE900A07F096F8D8ED017A67EEA87A41
:10BC2800C7E90E01F5EEC07AF1EE10FA4CBF77EED7
:10BC3800C87A77EE887A08F1040817EE900A07F0B8
:10BC480081F8032DC7E9080107F10807CED1A6F24C
:10BC5800DC531B042367E3676367C4F88030A3677A
:10BC6800C4F884300123A4F802902370D4F85490C7
:10BC7800B4F95280636A276A206FE26FD4F840C033
:10BC8800D4F88010C4F88020C9EB060606FA08F636
:10BC98004FEAE67B734307FB0B332667A7FB066770
:10BCA8001F44636C656F60674FEAE27B53430CFB8C
:10BCB8000B3EACFB02237344B61A67EB0307E36A37
:10BCC800A26AC4F884104FEAE07B434302FB0B3EB0
:10BCD800A2FB00237344B6185F41E36CA06CB4F96F
:10BCE8005020A5674FEAE17B4B4300FB0B33A0FBD9
:10BCF80001011944636B361A206B4FEAE57B05FB9B
:10BD080003F300FB0B3367EB0107A0FB05011944A4
:10BD18008019794106F0ECFF08F1FF3201239340C6
:10BD2800E067C01841EBE371424606F0E1FFBDEC65
:10BD3800028B4844BDE8F88F6F12833ADB0F494005
:10BD4800F404B53F0000804B2DE9F8430024234B51
:10BD580093F8A860E0B2B0420CD203EB8003204A0B
:10BD68009B6F32F810101BB10B2801D8DB6898477D
:10BD78000134ECE71B4B1B685B032DD500242346DD
:10BD8800E2B2B24228D2DFF8549009F178074FEABC
:10BD9800840857F8242055689D4215D0284605F098
:10BDA80065FFEFF31283502282F3128828216A6A12
:10BDB80001FB00900132C0F8D0206A6942F001020C
:10BDC8006A61DBB283F3118857F808301B680022D8
:10BDD8001A6001342B46D3E7BDE8F8831C1F002006
:10BDE800A8110020582E002008B50E4B1B6813F42C
:10BDF800805F0D4B14BFD3F87421D3F8782193F8E2
:10BE0800A81092880023D8B2884204D2074820F8A4
:10BE180013200133F7E7FFF797FF3220BDE808400A
:10BE2800F1E400BF582E00201C1F0020A81100209C
:10BE38000A4B1A680A4B30B502F48052D3F87441A1
:10BE4800D3F8785100230AB1A18800E0A9880548F1
:10BE580020F8131001330C2BF5D130BD582E0020DB
:10BE68001C1F0020522B002070B5124D00242146C3
:10BE780005F27D10702285F87C4109F072FF214699
:10BE8800D5F8F0310B4A0B4493F9020080B102F265
:10BE98007D141E680E5108199C8884809B798371D3
:10BEA80092F87C3107310133702982F87C31E7D16F
:10BEB80070BD00BF1C1F0020094B1A680E2303FB2E
:10BEC8000020437AFF2B07D0064A12789A4203D9FA
:10BED800054A32F8130000E0808800B2704700BFBE
:10BEE8008C210020142B0020942E0020022803D03F
:10BEF800431E584258417047064B1B681B7823B1B4
:10BF0800054B1868C0F3C0407047044B1878C0F35D
:10BF1800800070477006002068110020EA2F00207A
:10BF280010B50A4C5E280146206805D15D21FFF74F
:10BF3800FDFD20683E2105E05D2903D1FFF7F6FDF0
:10BF480020683D21BDE81040FFF7F0BD102100201A
:10BF580030B50028104C114AB8BF40423C2590FB30
:10BF6800F2F304FB030068430D4D90FBF2F22D68D9
:10BF78002D7B25B903EB830303EB830301E0C3EBBC
:10BF8800031302EB83030B8004FB02024FF47A7362
:10BF980092FBF3F24A8030BD806967FF8096980073
:10BFA800341A002010B50446C0B2FFF7B9FFC4F335
:10BFB8000720BDE81040B3E7024B5E211868FFF781
:10BFC800B5BD00BF1021002038B5064C05465E21DE
:10BFD8002068FFF7ABFD20682946BDE83840FFF729
:10BFE800A5BD00BF10210020674B73B51878674DB9
:10BFF800FFF77CFF2B788342044620D0C8B1644BFE
:10C008001B68E3B193F9000002230093614B1B689E
:10C018005B78003318BF0123019304214FF41653B2
:10C028000022FFF7FAFB5C4B186040B101232B702C
:10C0380005E0594E306802F098FA34602C70574B7E
:10C04800574D1878FFF752FF2B788342044618D0D3
:10C0580088B1544B1B68A3B10022012493F9000056
:10C0680000944FF4964301920821FFF7D6FB4E4BFC
:10C07800186028B905E04C4E306802F076FA346052
:10C088002C704A4B4A4D1878FFF730FF2B788342C3
:10C0980004462E4642D0002837D0464B1A68002A5C
:10C0A8003CD0D37992F90000434C002B08BF0223FF
:10C0B80002220092002254F8233001921021FFF747
:10C0C800ACFB3E4B0546186040B33D4C94F84A30F3
:10C0D800022B0BD094F89620022A01D14C3405E0AB
:10C0E80023B1002A04F14C0418BF0024354B1C600E
:10C0F80044B1204600214C2209F033FE022325607A
:10C1080084F84A300123337008E02C4E306804F07C
:10C1180049FC306802F029FA34602C702A4B2B4D08
:10C128001878FFF7E3FE2B788342044629D000B342
:10C13800274B1B682BB3274A93F9000012685278E3
:10C14800002A0CBF082209220323009301924FF40E
:10C15800614320210022FFF760FB1F4B186080B16C
:10C168001E4A012313702B701D4B1A681D4B1A6051
:10C1780007E0194E306802F0F8F9184B34601C706B
:10C188002C7002B070BD00BF780600202812002075
:10C1980074060020341A002010210020790600209F
:10C1A800541A0020D81A0020C81A0020840600203B
:10C1B800DE1A0020800600206C900108E01A00209A
:10C1C800782A0020E41A002090060020F41A0020A3
:10C1D8008C06002088060020F81A0020FC1A00208F
:10C1E8007C2E0020001B0020642928BF6421F8B59C
:10C1F80010FB01F56424064695FBF4F40027E4B22D
:10C20800FBB2A34204D29F2005F0FBFB0137F7E7FE
:10C21800B4420BD2C4EB84101421C4EB800095FB0C
:10C22800F1F5663D2844C0B205F0EBFB0134E4B2F9
:10C23800B44201D29A20F7E7F8BD2DE9F743934CB1
:10C24800FFF7BAFA6368C31A002BC0F2688300F5D7
:10C25800433303F5A07363608D4B1D78237AC5F3D0
:10C268008005EB1A18BF012325724DB1002B00F091
:10C278005683884B5A789A7001225A701A702BE0AC
:10C28800844A2BB1D37843F00203D3709378537068
:10C29800D67806F0020101F0FF0339B97D498968B3
:10C2A800411A002903DB06F0010300E0012303F033
:10C2B8000107784917707BB1F2070DD50A79013269
:10C2C800D2B20523B2FBF3F303EB8303D31ADBB239
:10C2D800714A0B71D35C4B706E4EDFF8088233786D
:10C2E8007BB3F37823F00203F3706C4B0344AE2066
:10C2F800B36005F0AAFB08B105F0ACFB88F80000B4
:10C30800002800F00C83B02005F09FFB402005F0CA
:10C318009CFB002005F099FB102005F096FB4FF4DC
:10C328008067013F0020BFB205F066FB002FF8D1FF
:10C33800384605F0FEFB7278594B53F8220005F099
:10C348007BFB98F80030002B00F0E9827378062B0D
:10C3580000F2B382DFE813F00700B102180078009A
:10C368006C018901EE014F494F4A504B5048FDF787
:10C3780006FA012005F0DDFB4D4805F05DFB0220C3
:10C3880005F0D7FB4B48AEE14B4F3B689B0735D5D3
:10C39800DFF85481DFF85491B8F8001044480A23B4
:10C3A800B1FBF3F203FB121399F80010009192B25B
:10C3B80042499BB2FDF7E3F9FDF7F6FD012005F0D0
:10C3C800B8FB3B4805F038FB3D4B99F8002018684E
:10C3D800B8F80030067906FB123164234B43C17864
:10C3E8008E1B56430220B3FBF6F6F6B205F0A1FB0E
:10C3F80031461520FFF7F8FE032600E001263B68CA
:10C408001F0540F15A822F4B2F491F680968009178
:10C4180064232E4997FBF3F2254803FB1273FDF7BB
:10C42800AEF9FDF7C1FD304605F083FB204805F065
:10C4380003FBFCF71DF90746701C05F07AFB152075
:10C448003946FFF7D1FE38E20120214F05F071FB94
:10C45800204805F0F1FA3B68980749D51E4A144868
:10C46800B2F90210B2F900300091B2F904201B4968
:10C4780001921B4AFDF783F9FDF796FD022005F0AE
:10C4880058FB0B4805F0D8FA032632E010210020AB
:10C49800EA2F00204821002075A90108404B4C00D4
:10C4A800688701087AA9010883A90108B9A40108C5
:10C4B800192100208AA90108582E002091A90108F5
:10C4C8002C1A0020381A00203C1A0020A9A90108BB
:10C4D800401A0020BEA9010832120020D4A9010880
:10C4E800E3A90108E9020020301A0020FC0000201E
:10C4F80002263B68D9071AD57C4A7D48B2F9021052
:10C50800B2F900300091B2F904207A4901927A4ACE
:10C51800FDF735F9FDF748FD304605F00AFB74488C
:10C5280006F1010805F088FA5FFA88F846463B6884
:10C538001A0718D5714A6E48B2F90210B2F90030DC
:10C548000091B2F904206B4901926D4AFDF717F981
:10C55800FDF72AFD304605F0ECFA6548771C05F032
:10C568006BFAFFB23E46674A6249B2F90030B2F947
:10C5780002200092644A5E48B2F900200192634AA0
:10C58800634FFDF7FCF8FDF70FFD304605F0D1FAD3
:10C59800574805F051FA97ED000A5548FCF784FF13
:10C5A800534809F022FC06F101085FFA88F8C0B286
:10C5B800B946092809D8431C2044DBB2202242721C
:10C5C800E218002191721846F3E7494F99ED010AE4
:10C5D8003844FCF769FFFDF7E7FC404605F0A9FA87
:10C5E800384605F029FA99ED020A3846FCF75CFF4F
:10C5F800384609F0FAFB0236F6B2C0B2092809D863
:10C608002318421CD2B220215972A3180021997212
:10C618001046F3E73F4AB2F9003000EE103A3844CA
:10C62800B8EEC00AFCF740FFFDF7BEFC304657E005
:10C638000026394F3B78B34240F23F810E2E00F07E
:10C648003C817008013005F074FA304605F0C2FFED
:10C658003B78B34206D9202005F0D3F9701CC0B24C
:10C6680005F0B8FF0236F6B2E3E72C4E2C4996F8EF
:10C67800B0271F48FDF783F8012005F05AFA1C4837
:10C6880005F0DAF9274B28491F7819483A46FDF78B
:10C6980076F8022005F04DFA154805F0CDF90C237F
:10C6A80003FB0766214996F8B32796F8B237104876
:10C6B800FDF765F8FDF778FC032005F03AFA0C4819
:10C6C80005F0BAF996F8B81796F8B62796F8B73776
:10C6D800074800911649FDF752F8FDF765FC04205C
:10C6E80005F027FA024805F0A7F9E6E088110020CE
:10C6F80019210020D4A90108E7A901088E110020FA
:10C70800C1BF01084E2E002040120020EBA90108ED
:10C718000429002010290020142B0020501200208A
:10C72800EFA90108502B0020FBA901080CAA010859
:10C738001DAA01087B4B1B681B0640F1BA80236ABF
:10C74800616A794A8B421FBF536292F828300133DD
:10C7580003F003034FF001014FF0000018BF82F807
:10C76800283005F0F2F994F82830704AD05C05F0CA
:10C7780048F90220012105F0E8F900266C4B9B5D81
:10C788003620C3EBC30393FBF0F0C0B2062828BFE2
:10C7980006206038C0B2013605F033F9102EEDD10D
:10C7A800644B65491B78654813F0020F644B1A788F
:10C7B80014BF59234E23FCF7E2FFFDF7F5FB0220D7
:10C7C80005F0B7F95D4805F037F95E495E4B4E68EC
:10C7D8000A685A4892FBF3F25C4996FBF3F3FCF7BC
:10C7E800CEFFFDF7E1FB032005F0A3F95348584EAF
:10C7F80005F022F9574B58491A885048FCF7BFFFF3
:10C80800FDF7BEFB042005F094F94C4805F014F937
:10C81800524B53491A884948FCF7B1FFFDF7B0FB62
:10C8280004210A2005F091F9444805F005F94D491D
:10C83800E26A4248FCF7A3FFFDF7A2FB052005F0DA
:10C8480078F93E4805F0F8F87268B36846493B48FD
:10C85800FCF795FFFDF794FB05210A2005F075F913
:10C86800364805F0E9F83369F26840493348D21A86
:10C87800FCF785FFFDF784FB062005F05AF92F48E1
:10C8880005F0DAF8B2683A492C48FCF778FFFDF76A
:10C8980077FB06210A2005F058F9284805F0CCF85E
:10C8A80034492648152209F0CDFAFDF769FB07201F
:10C8B80016E7F37843F00203F370002D2FD12E4BC7
:10C8C80093F82030052B9BBF2C4A9B183F251D7FD2
:10C8D8000021122005F039F9284605F092F81320B6
:10C8E800002105F032F9264B1B78002B254B1B78CD
:10C8F80014BF72202120002B18BF522005F081F8A8
:10C908001420002105F021F994F83050074B585DA8
:10C91800013505F0030505F074F884F8305003B0CC
:10C92800BDE8F083582E0020102100202FAA01080E
:10C9380015120020441A002034AA010819210020E9
:10C948004A1A00204C1A00208096980045AA01082F
:10C9580000080020461A002052AA0108CC11002025
:10C968005AAA010861AA010868AA010871AA01085F
:10C9780078AA010830030020DC2E0020688701080F
:10C98800BB0E0020200F002038B500240B4D605945
:10C99800254404F0FBF8696811B10948FCF704FF65
:10C9A800A96811B10748FCF7FFFE0748103404F0E6
:10C9B800EDF8B4F5D87FE9D138BD00BF8C87010800
:10C9C800B1AA0108B7AA01087AB40108F0B585B080
:10C9D800044609F00AFA082826D1621EE01D1F49FC
:10C9E80012F8013F09681944497801F00301022946
:10C9F80008BF203B82421370F1D1254604F1080795
:10CA080015F8016B1648314609F0E1F920B12846BE
:10CA1800314609F0DCF910B101F026F91CE0BD42FD
:10CA2800EED1204603F006FE0E4804F0AFF80023CE
:10CA38000D4A1A4404A992F88A210A440849595C03
:10CA480002F80C1C0133082BF2D1002307488DF89B
:10CA58000C3001A9FCF7A8FE05B0F0BD0C010020C0
:10CA6800CEBF0108BDAA010850120020BCB30108BE
:10CA78002A4B2B4C1E68206880B501F06BFD3046B0
:10CA880001F068FD206841798D0704D4036841F0FE
:10CA980002015B699847234B234D10229A6120229B
:10CAA8009A612B689A0341BF06236371E37923F0E7
:10CAB800010344BF43F00203E3712068FFF733F832
:10CAC80090B1184F10233B85154B1868FFF728F8CD
:10CAD8008046FAF729FB08B102F09AFF3046414632
:10CAE800FFF724F81023BB613046FFF71CF878B134
:10CAF8000C4FD4F800904FF02008A7F82880304653
:10CB0800FFF70EF801464846FFF710F8C7F81880F7
:10CB18002B689B03D1D5FFF790FBCEE76C2B002049
:10CB28004421002000040048582E00202DE9F04739
:10CB3800054609F05AF9314E0446D6F8088090B9EE
:10CB48002F4804F023F82F4B53F8241049B1012340
:10CB5800A34013EA080F02D02B48FCF725FE013446
:10CB6800F1E72A4822E028462949224609F046F9F1
:10CB780058B92848284C04F009F854F8041F00292B
:10CB8800EFD02148FCF710FEF7E72B782D2B03BFD9
:10CB9800013504F1FF344FF0010A4FF0000A4FF05D
:10CBA8000009184B53F8297027B91C48BDE8F0470D
:10CBB80003F0ECBF28463946224609F01FF9C8B9E8
:10CBC800012000FA09F0830501D51548EEE7BAF10E
:10CBD800000F03D0FCF73EFF124803E040EA0800CC
:10CBE800B060114803F0D2FF39461048BDE8F0475D
:10CBF800FCF7DABD09F10109D3E700BF50120020A4
:10CC0800C3AA01083C890108CDAA01087AB4010821
:10CC1800D1AA0108D6AA010838890108E2AA0108A0
:10CC2800F1AA0108FFAA010808AB0108BBB3010873
:10CC380010B5084803F0AAFF074B00241C741C64B5
:10CC4800064B1C70FFF7F4F804F084F9044B1C60E1
:10CC580010BD00BF10AB010844210020EB2F0020BD
:10CC68006C2B002070B5064600240B4BE518AA88EB
:10CC780016420AD0E1580948FCF796FD28460021DB
:10CC880003F011FF064803F081FF143440F6BC435B
:10CC98009C42EAD170BD00BFCC9201083CAB0108B0
:10CCA8007AB40108F0B504788BB005460CB10024BD
:10CCB80036E04B4B19680E2303FB041101F58C7009
:10CCC800B1F91D51B1F91921B1F91B31009591F84C
:10CCD8002051019591F82151029590F90700039090
:10CCE80001F590713F4891F90210049121460134F1
:10CCF800FCF75AFD082CDCD170E02D2B14D1072C41
:10CD08001BDC284609F0C8F80AAB661C03EB440490
:10CD180024F8100C15F8013F303B092BFAD934469A
:10CD28002B78002BE9D104E0A3F13002092A09D8B5
:10CD3800E5E7082CBDF8182009D00BB0BDE8F04095
:10CD480000F092BF202BF8D101352646E7E7072AE5
:10CD5800F3D8BDF81A00224BA0F2EE2189B240F2B6
:10CD6800DC55A9421B68E8D8BDF81C10A1F2EE24D6
:10CD7800A4B2AC42E1D8BDF81E6004B237B2A742F3
:10CD8800DBDB0DB2AF42D8DCA542D6DBBDF82470A0
:10CD980007F16404A4B2C82CCFD8BDF826E00FFA76
:10CDA8008EF4112CC9DCBDF82050B42DC5D8BDF8BF
:10CDB8002240B42CC1D812B24FF00E0C0CFB023337
:10CDC800A3F81901A3F81B11A3F81D6183F82051DA
:10CDD80083F8214183F81F7183F822E10BB0F0BD7D
:10CDE800A411002046AB0108F0B504468FB02046D8
:10CDF80008F0FBFFC5B225BBAC48AD4C03F0C6FE3E
:10CE080094F8D61009B9AB4854E049B294F8D42044
:10CE180094F8D530009194F8D710019194F9D8106E
:10CE2800029194F9D910039194F8DA100491A24868
:10CE380029460135FCF7B8FC102D04F10704DFD1B1
:10CE4800E1E720469D49052208F0D8FF0546B8B914
:10CE580029469B48702208F084FF9A4B1968284697
:10CE68000E2303FB001301300022082883F8232136
:10CE780083F8242183F8252183F82621F0D113E1B2
:10CE880020469149042208F0B9FF05462046002DA6
:10CE98004AD1202108F09BFF002800F00581461C9C
:10CEA800304608F0A2FF2C460746884B53F824501A
:10CEB8002DB987480FB0BDE8F040FCF775BC304687
:10CEC8002946FAB208F09AFF01340028EDD1784AD1
:10CED80002F170011646002382F8DA3082F8D63063
:10CEE80082F8D53082F8D43007328A42F3D17949B2
:10CEF80001EBC40191F80822934210DAD1F80C72C0
:10CF0800C3EBC302B0183A4400F1D4011768C0F863
:10CF1800D4709088888092798A710133E7E729462E
:10CF28006D48FCF741FC90E06C49072208F066FF69
:10CF380005462046002D4AD1202108F048FF064624
:10CF480008F053FFC4B274BB6548FCF72DFC2146BA
:10CF580064480134FCF728FC0E2CF8D15548FCF73E
:10CF680023FC002460482146FCF71EFC0025554A96
:10CF78005E4811680E2202FB04120123D2F8232115
:10CF88005B49AB4013425B4B05F1010508BF1946ED
:10CF9800FCF70AFC0E2DEAD146480134FCF704FCE4
:10CFA800082CDFD180E03046534908F079FF2C4641
:10CFB80000284CD0022C4FD008F06EFF06AB4E492B
:10CFC80043F82400002008F06BFF0134F0E74A49D9
:10CFD80008F066FF002460B1082C38D008F05CFF28
:10CFE80006AB454943F82400002008F059FF0134F6
:10CFF800F1E7082C2BD1069B0F2B28D8DDF81CE075
:10D00800BEF1070F23D8089F0D2F20D8099E06F1DF
:10D018006402C82A1BD80A9DFF2D18D80B986428CB
:10D0280015D80C99642912D8884210DA0D9C032C63
:10D038000DD8324AC3EBC303134483F804E05F718D
:10D048009E71DD71187259729C722D4CCFE60FB02B
:10D05800BDE8F04000F008BE069B072B20D80799D2
:10D068000D291DD80278722A0DD06E2A18D1154ABA
:10D0780012680E2000FB032301228A40D3F82311F3
:10D0880021EA020209E00F4A12680E2000FB03237E
:10D0980001228A40D3F823110A43C3F8232101E06F
:10D0A80000F0E2FD0D4CA2E60FB0F0BD6EAB01083A
:10D0B800501200207AB4010899AB0108B5AB0108F9
:10D0C80024130020A4110020BBAB0108889F01088D
:10D0D800E2AA01088C870108C0AB010866AB010809
:10D0E800BBAA0108CCAB01085EAA0108D1AB0108B4
:10D0F800D5B701088FB80108D5AB01082013002067
:10D10800D2A701082DE9F743047805468CB9324DBA
:10D1180095F8AB12B5F8A82295F8AA322F480091D5
:10D1280021460134FCF740FB102C05F10405EFD132
:10D138004EE008F0B1FE0F28044636DC28462021D0
:10D1480008F045FE264EE4B2D6F84480451CA400FB
:10D158000027284608F0A0FE5FFA87F9B9F1010F09
:10D1680083B208D0B9F1020F0BD0B3F5B47F24D243
:10D17800726C13530AE0FF2B1FD8736C234498700A
:10D1880004E0FF2B19D8736C2344D87028462C214F
:10D1980008F01DFE054608B1013502E0B9F1020F9D
:10D1A8000BD10137032FD4D112E00E4800210F22F2
:10D1B80003B0BDE8F04300F0D4BC08EB0400002144
:10D1C800042208F0CEFD03B0BDE8F04300F04CBDEA
:10D1D80003B0BDE8F08300BF50120020D7AB0108B0
:10D1E80044210020EBAB01082DE9F0412DED048B23
:10D1F800B1498AB0044608F0BDFDB0490028204670
:10D208000CBF0126072608F0B5FDAD4900282046C9
:10D2180008BF022608F0AEFD002808BF0426F10763
:10D2280040F1EF80A748A84C03F0B0FC002003F0C1
:10D23800B9FAA64803F0AAFCA54803F0A7FC63794D
:10D24800A44AA548013B254652F82310FCF7ACFA3E
:10D25800A248FCF7A9FA4FF00008274695ED058A81
:10D26800B5EE408AF1EE10FA04D19D48FCF79CFA1D
:10D27800002570E09B48D5ED069A95ED079AD5ED07
:10D28800088A4146FCF790FAB5EEC08AF1EE10FA2A
:10D2980002D5202003F072FCB0EE480A06A8FCF77D
:10D2A80003F901469048FCF77FFAF5EEC09AF1EED3
:10D2B80010FA02D5202003F061FCB0EE690A06A836
:10D2C800FCF7F2F801468848FCF76EFAB5EEC09A0A
:10D2D800F1EE10FA02D5202003F050FCB0EE490A16
:10D2E80006A8FCF7E1F801467F48FCF75DFAF5EE81
:10D2F800C08AF1EE10FA02D5202003F03FFCB0EE10
:10D30800680A06A8FCF7D0F808F101080146774832
:10D31800FCF74AFAB8F10C0F05F110059ED1A4E705
:10D3280049B294F8D42094F8D530009194F8D710E5
:10D33800019194F9D810029194F9D910039194F8B5
:10D34800DA1004916A4829460135FCF72DFA102DA8
:10D3580004F1070403D094F8D6100029E0D16548F9
:10D36800654C03F013FCD7F8088054F8041F19B172
:10D378006248FCF719FAF8E70D46614B53F8254067
:10D3880054B10123AB4013EA080F03D05D4821468E
:10D39800FCF70AFA0135F0E75B4803F0F7FB214692
:10D3A8007B180AAA93F88A311344584A8A5C03F80E
:10D3B800102C01310829F3D1002306A954488DF80F
:10D3C8002030FCF7F1F9534803F0E0FB524800F035
:10D3D80081FF524803F0DAFB4F4800F04BFC5048FD
:10D3E80003F0D4FB4C48FFF78DFE4E48FCF7DCF900
:10D3F8004020FFF737FC4C4803F0C8FB464801F0D3
:10D408000BF8B20739D5494803F0C0FB484803F088
:10D41800BDFB414803F006FA464803F0B7FB3E4817
:10D4280000F0ACFB444803F0B1FB3B4800F0A4FE1D
:10D438004248FCF7B9F9384800F028FD404803F0A5
:10D44800A5FB3548FFF72EFC00270E257D43002459
:10D458003C4A926C2A440123D2F80A20A340134282
:10D468001ED101340E2CF3D10137082FEDD12D48F0
:10D47800FCF79AF98020FFF7F5FB730716D53248B9
:10D4880003F084FB314803F081FB234803F0A4F93F
:10D498002448FCF789F94FF48070FFF7E3FB05E0B7
:10D4A800394622462A48FCF77FF9DAE70AB0BDEC8C
:10D4B800048BBDE8F08100BFF1AB0108FDAF0108A6
:10D4C800F8AB0108FEAB0108501200200CAC0108B3
:10D4D8001EAC0108889F01082AAC010835AC010878
:10D4E80042AC01084FAC0108BAAA0108BCB3010854
:10D4F80067AC010857AC01083889010886AC0108F7
:10D508003C89010894AC0108A1AC0108CEBF010810
:10D51800ADAC0108B6AC0108D2A70108C5AC01083A
:10D52800D1AC01087AB40108DFAC0108ECAC010801
:10D53800FFAC01080DAD010817AD010826AD0108C3
:10D5480034AD01084421002040AD010851AD010867
:10D5580063AD0108026BC168034610B5406942B16A
:10D568001A6C8C1A013A005D08BF0A46C0B21A64E8
:10D5780010BD1A6A805C01328A4228BF0022C0B2FC
:10D588001A6210BD436B13B190F844007047836A68
:10D59800406A1B1A584258417047036B13B15B68C5
:10D5A800016C01E0C369016A8B423CBFC2689B18E9
:10D5B800581AC0B27047836A8169426B1944D160B6
:10D5C800416A99429DBF0169CB1A5360CB1A96BF35
:10D5D8000023536083624FF0000380F844301368DF
:10D5E80088BF816243F0010313607047436A826910
:10D5F800D154436A02690133934228BF002343622E
:10D60800436B1BB11B68DB0705D4D4E7026D1368B5
:10D6180043F08003136070474171F7F73DB98160AB
:10D62800F7F73AB9026D036B70B50446D5699BB933
:10D63800A90611D5C36A1BB1908C80B298470BE03C
:10D64800E169928C40694E1CD2B2E6614254E169AC
:10D65800E268914228BFE361616BA1B92A0612D53D
:10D66800636AA26A9A42236D09D0501CA669A06217
:10D67800B25C1A852369984205D3A16203E01A684F
:10D6880022F080021A602B0742BF236D08221A621B
:10D6980070BD0D4B0D484FF400525A600C4A11688A
:10D6A8004FF6FE730B401360426B11684FF6FE7322
:10D6B8000B401360426A836A9A4200D07BE70123D9
:10D6C80080F84430704700BF00000240402C002022
:10D6D800440002402DE9F0471E46A14B8CB0984209
:10D6E800894690469DF850507ED19E4B9E4A1A60BE
:10D6F8009E4A5A6102F580729A614FF48072DA602C
:10D708001A619B4A1A63143A5A63A2F54842203AAE
:10D71800DA6404329A64C3F808801865954B9A69EC
:10D7280042F480429A615A6942F001025A61022326
:10D738008DF80830032315F0010A8DF809304FF0F1
:10D7480000038DF80A3014BF022301232C078DF83B
:10D758000B3017D5884C402701978AF001038DF8C4
:10D768000A30236A23F070632362236A43F0E0637C
:10D778002362204601A9FAF7A3FEBAF1000F23D1CC
:10D78800A76121E0B0070ED50CA9402341F82C3D34
:10D798007948036A23F070630362036A43F0E06325
:10D7A8000362FAF78DFEF1070ED50CA9802341F824
:10D7B8002C3D7148036A23F070430362036A43F007
:10D7C800E0430362FAF77CFE0E238DF80030002256
:10D7D800012368468DF801308DF802208DF803305A
:10D7E800604C04F099FC08E1644B984274D1644B96
:10D7F8005D4A1A604FF48072DA601A61614A5A61B0
:10D8080002F580729A615B4AC3F808801865D3698B
:10D8180043F40033D36102238DF80830032315F055
:10D82800010A8DF809304FF000038DF80A3014BF53
:10D83800022301232A078DF80B3019D54FF09044A5
:10D84800042701978AF001038DF80A30236A23F42C
:10D8580070632362236A43F4E063236220460DEB7E
:10D868000701FAF72DFEBAF1000F25D1A76123E0D1
:10D87800B3070FD50CA9042341F82C3D4FF0904075
:10D88800036A23F470630362036A43F4E063036288
:10D89800FAF716FEF7070FD50CA9082341F82C3D17
:10D8A8004FF09040036A23F470430362036A43F421
:10D8B800E0430362FAF704FE26238DF800300022C5
:10D8C800012368468DF801308DF802208DF8033069
:10D8D8002B4C04F021FC90E02B4B984240F00E8139
:10D8E8002A4B214A1A604FF48072DA601A61284A7A
:10D8F8005A6102F580729A611E4AC3F80880186559
:10D90800D36943F48023D36102238DF808300323BD
:10D9180015F0010A8DF809304FF000038DF80A3030
:10D9280014BF022301232C078DF80B3032D5124C7B
:10D938004FF4806701978AF001038DF80A30636A13
:10D9480023F470636362636A43F4E06363622046AE
:10D9580001A9FAF7B5FDBAF1000F3FD1A7613DE083
:10D9680000380140402C0020248B01089021002021
:10D9780058000240001002400004004800440040E3
:10D98800EC2B00209023002000480040982B00201A
:10D9980090250020B0070FD50CA94FF4806341F8FB
:10D9A8002C3D5848436A23F470634362436A43F446
:10D9B800E0634362FAF784FDF1070FD50CA94FF431
:10D9C800006341F82C3D4F48436A23F47043436297
:10D9D800436A43F4E0434362FAF772FD27238DF864
:10D9E80000300022012368468DF801308DF80220AE
:10D9F8008DF8033004F090FB434CC4F82C900027BA
:10DA0800012384F844302762E761A7626762667180
:10DA1800C4F80880A5712046F6F73EFFF20734D512
:10DA2800236B002B2AD001A8FAF7E6FAE36C0193DE
:10DA38004FF480530A9380230693E368ADF81030BF
:10DA480020230993206B636902930B970597079727
:10DA580008970397FAF7FBFA01A9206BFAF7D9FAA6
:10DA6800236B216D1A6842F001021A608A6842F03D
:10DA780040028A605B689BB2236406E0236D202223
:10DA88001A621A6842F020021A60B3072FD5636B36
:10DA980043B301A8FAF7B0FAA36C01934FF480538B
:10DAA8000A93802306932369ADF8103000251023CC
:10DAB800606B03930B950595079508950995FAF7FB
:10DAC800C6FA606B01A9FAF7A4FA636B1A6842F008
:10DAD80002021A60226D5D605D60936843F0800306
:10DAE800936004E0226D136843F080031360226D95
:10DAF800136843F001031360204600E000200CB0D7
:10DB0800BDE8F08700040048982B0020F8B50446CB
:10DB18000E46174600252046202108F058F90446ED
:10DB2800D0B10134204608F0B7F9B0F5617F05DBC4
:10DB380040F634039842A8BF184601E04FF46170DC
:10DB4800A0F56170192390FBF3F00DB9307000E077
:10DB580070703B7801333B700DB90125DBE7204637
:10DB6800F8BD30B505460C461346294622460248FC
:10DB7800BDE83040FBF718BE40B201087FB5047815
:10DB88000646E4B9354B1B6803EB8403192193F867
:10DB98007B0093F87C6093F8792093F87A304FF4FF
:10DBA800617511FB005011FB0651009001912C4842
:10DBB80021460134FBF7F8FD142CE3D14BE008F0C3
:10DBC8006BF91328054641DC244B701C1C68202186
:10DBD80000238DF80F3008F0FAF81E35064670B1AC
:10DBE8000136304608F058F91A289FBF04EB850320
:10DBF80058709DF80F30013398BF8DF80F303046BC
:10DC0800202108F0E4F8064670B10136304608F0E5
:10DC180043F90D289FBF04EB850398709DF80F30DA
:10DC2800013398BF8DF80F3004EB85043046E11CB2
:10DC38000DF10F02FFF76AFF9DF80F30042B0AD091
:10DC4800601C0021042208F08CF804E0054800213B
:10DC58001322FFF786FF04B070BD00BFA411002097
:10DC68005FB20108EBAB0108014802F08FBF00BFAB
:10DC780074B201082DE9F04304788FB00546002CF2
:10DC880059D17B4B0021142209A807AED3F8008094
:10DC980008F067F807223046002108F062F805A866
:10DCA8000023A700059308EB070583801A467149EE
:10DCB800B5F802E031F813C01CEA0E0F0AD00DF1D6
:10DCC800380C0E3102F1010E6244595C02F81C1C3A
:10DCD8005FFA8EF20133072BE9D100210B46664A21
:10DCE800B5F802E011F802C01CEA0E0F0AD00DF1D7
:10DCF800380C063203F1010E63448A5C03F8242CC5
:10DD08005FFA8EF301310629E9D118F807305B492B
:10DD18008DE841006A78029209A81A0903F00F03F6
:10DD2800FBF72DFD2146564809AA0134FBF73CFDB7
:10DD3800202CA6D198E008F0AFF81F28044600F37D
:10DD4800868028462021E4B208F041F81F2C02D929
:10DD5800FFF78AFF88E0464B1B6803EB8404451CE9
:10DD680000212046042207F0FCFF0027454B09AE9E
:10DD7800304600210A2217F803905FFA87F807F067
:10DD8800F0FF002315F8012B32B10A2B04D04A45C5
:10DD980002D0F2540133F5E74A455ED108F1FF336A
:10DDA800032B09D8DFE803F01005023F0DF123012A
:10DDB80034E00DF123011EE0304608F06DF82378B9
:10DDC800C0B243EA001006E0304608F065F8237850
:10DDD80000F00F001843207031E00133062B0AD001
:10DDE800244800F11B069E5D9642F6D103445A7DF5
:10DDF80063881343638011F8012F02B30023EFE710
:10DE08000133072B0AD01B4800F10E069E5D96428F
:10DE1800F6D130F8132063881343638011F8012F7B
:10DE28006AB10023EFE7304608F036F80F2804DC23
:10DE3800304608F031F8607001E000236370013764
:10DE4800052F93D1012401F089FD6CB980E70E48B4
:10DE580000211F22FFF785FE06E02046002104224C
:10DE680007F07FFF0024EEE70FB0BDE8F08300BFA6
:10DE7800902700203C8B0108518B010882B20108D1
:10DE880091B201085D8B0108EBAB0108F8B5047885
:10DE9800064674B9304DB5F8C621B5F8C8312F48D3
:10DEA80021460134FBF780FC042C05F10405F2D16E
:10DEB800F8BD2B4907F05EFFA8B9274B4FF47A71DC
:10DEC8004FF4FA62A3F8C611A3F8C821A3F8CA113F
:10DED800A3F8CC21A3F8CE11A3F8D021A3F8D2112E
:10DEE800A3F8D421F8BD304607F0D6FF032805462D
:10DEF8002BD83046202107F06AFF044630B10134A0
:10DF0800204607F0C9FF0126074600E006462046DE
:10DF1800202107F05CFF10B9BDE8F840A4E6013005
:10DF280007F0BAFF012EF7D1A7F2EE2240F2DC5338
:10DF38009A42F1D8A0F2EE229A42EDD8064B7035FB
:10DF480003EB8503DF801881F8BD06480021032212
:10DF5800BDE8F84005E600BF501200209DB2010858
:10DF6800B5AB0108A2B601082DE9FF4104780546C2
:10DF7800002C39D17348744D02F008FED5ED057AAE
:10DF8800F5EE407AF1EE10FA00F0D88021466F489D
:10DF9800FBF70AFC95ED050A6846FBF785FA01468A
:10DFA8006B48FBF701FC95ED060A6846FBF77CFA1F
:10DFB80001466748FBF7F8FB95ED070A6846FBF74B
:10DFC80073FA01466248FBF7EFFB95ED080A6846CD
:10DFD800FBF76AFA013401465E48FBF7E5FB0C2CB7
:10DFE80005F11005CAD1A9E05B49052207F006FF33
:10DFF80040B9554B03F1C0020021596110339342D7
:10E00800FAD19BE028465549042207F0F7FE04465A
:10E018002846002C40D1202107F0D9FE002800F026
:10E028008D80451C284607F0E0FE07464C4B53F808
:10E0380024601EB94B4802F0A9FD7FE0284631460E
:10E04800FAB207F0DBFE01340028EFD13E4B03F1B2
:10E05800C0029E460021596110339342FAD1424BC7
:10E0680003EBC4029846D2F804C0BCF1000F04D1F7
:10E0780031463E48FBF798FB57E0002718F8343044
:10E088009F42F5DA3B010EEB030563440FCB1435D1
:10E0980085E80F000137F1E707F0FEFE0B2806467A
:10E0A80047DC2846202107F092FE054650B101358D
:10E0B8002846FBF76FF9244B03EB061383ED050A9B
:10E0C800012400E004462846202107F080FE05468A
:10E0D80048B101352846FBF75DF91B4B03EB0613E6
:10E0E80083ED060A01342846202107F070FE054614
:10E0F80048B101352846FBF74DF9134B03EB0613DE
:10E1080083ED070A01342846202107F060FE10B984
:10E11800FFF7AAFD12E00130FBF73CF90A4B032C8C
:10E1280003EB061686ED080AF2D11148FFF71CFF2B
:10E1380004E0104801210C22FFF713FD04B0BDE8EC
:10E14800F08100BFB0B2010850120020CBB2010824
:10E15800D1B20108BCB30108B5AB0108BBAB0108DB
:10E16800889F0108E2AA010870B10108C0AB010844
:10E17800D2A70108EBAB0108F0B5047887B00646D2
:10E188001CBB514B1968062303FB0411192091F895
:10E19800CA5091F8CB7091F8CE2091F8C9304FF45D
:10E1A800617610FB056510FB07600095019091F8FA
:10E1B800CC000290C8314548497903912146013481
:10E1C800FBF7F2FA0C2CDCD17CE007F065FE0B289B
:10E1D800044672DC3C4B701C1D68202100238DF81E
:10E1E800173007F0F4FD064680B10136304607F0D7
:10E1F80053FE03289FBF062303FB045383F8CE0076
:10E208009DF817309CBF01338DF817303046202118
:10E2180007F0DDFD074680B10137384607F03CFEC0
:10E228000D289FBF062303FB045383F8C9009DF8FC
:10E2380017309CBF01338DF8173006266643A9199D
:10E248003846CA310DF11702FFF760FC202107F0AC
:10E25800BEFD074670B10137384607F01DFE142889
:10E268009FBF9DF817307619013386F8CC0098BF08
:10E278008DF817303846202107F0A9FD78B1013014
:10E2880007F00AFE0D289FBF062303FB045383F8FB
:10E29800CD009DF817309CBF01338DF817309DF8DD
:10E2A8001730062B0ED0062202FB04500021C9307D
:10E2B80007F057FDFFF7D8FC04E0054800210B22C2
:10E2C800FFF74FFC07B0F0BDA4110020D5B201083C
:10E2D800EBAB0108F0B5027887B08AB94A4C04F173
:10E2E800200694F8F62100234849595650B2814235
:10E2F8006DD00C33302BF7D10834B442F1D180E023
:10E30800002204920592451C07F0C6FDC4B260B213
:10E31800FDF7E8F8074618B18DF81040012400E031
:10E3280004462846202107F052FD054638B101353C
:10E33800284607F0B1FD0134ADF81200E4B200261A
:10E348002846202107F043FDB0B3451C284607F0B6
:10E35800A3FD00222E4951F8223083425FFA82FE43
:10E3680004D00132082AF5D1002300E0734651F8A1
:10E378002320824220D1022E0FD0032E12D05A1E03
:10E38800012ED2B204D0042A13D88DF814300EE02E
:10E39800042A0ED88DF8153009E0052B09D88DF818
:10E3A800173004E09A1E052A03D88DF81630013478
:10E3B800E4B20136042EC3D1052C03D807B0BDE85A
:10E3C800F04051E404AB03CB3860796019E094F86D
:10E3D800FB010F4B94F8FA5153F82000B4F8F821D8
:10E3E800009094F8FD0153F82000019094F8FC0186
:10E3F80053F82000029053F825300648FBF7D4F96B
:10E408007AE707B0F0BD00BF50120020202B002093
:10E418006C900108F5B201082DE9F3470478064627
:10E428004CB9204601A904F0FBF80134FFF7F4FFCA
:10E43800122CF6D180E007F02FFDC5B2112D76D849
:10E448003F4C05F1D00704EB4703701C202193F8DB
:10E4580002803C4E07F0BBFC034630B9A8F102022B
:10E46800D2F1000848EB020848E006F1260800F15E
:10E47800010A5978404607F0AAFC68B1032D8CBF01
:10E4880003230023C8EB0000334453FA80F090F8CC
:10E498002A90B9F1030F02D1FFF7E6FB4CE0A9F18E
:10E4A8000203D3F1000850464FF0200148EB03085F
:10E4B80007F08DFCD8B1B8F1000FEDD0013007F0AE
:10E4C800EBFC40F2ED2380B2984205DD40F6CA032A
:10E4D8009842A8BF184601E040F2EE2004EB47033B
:10E4E800A0F2EE20192290FBF2F0D87002E0B8F109
:10E4F800000FD1D104EB470383F8029004EB4704E3
:10E50800A3781E4496F82620B8F1000F0AD0E378C5
:10E518000D48294640F2EE24192505FB0343FBF775
:10E5280043F909E029460948FBF73EF904E00848A1
:10E5380000211122FFF715FB02B0BDE8F08700BFEC
:10E54800501200203C8B010814B3010826B30108BF
:10E55800A2B6010810B504462046FDF7DBFA18B943
:10E568000A20FDF750F9F7E710BD002207490C23F0
:10E5780003FB02135968814204D10022C2621A7255
:10E588005A6070470132042AF0D17047202B0020CE
:10E59800704708B50B4B002093F82C10F9F778FC5E
:10E5A800094B1B68187A082801BF084B4FF48052A2
:10E5B8001A80102208BF5A80A0F109035842584116
:10E5C80008BD00BFA80000200C2A002094270020C6
:10E5D800024B4FF480221A60704700BF14040140B8
:10E5E800704770477047FEE7FEE7FEE7704730B5B3
:10E5F8000024E3B293420DD2030F092B94BF3033AA
:10E60800373301F8143001EB4403002500015D7035
:10E618000134EEE730BD30B5002202F1805303F536
:10E62800B8539B0042F400441D6840F60F7144F053
:10E638008004294001322143042A1960EDD1024B9C
:10E6480040F08000186030BD4C5C00402DE9F34775
:10E65800884D894C2B68894E9BB2A380A28831884B
:10E668000A40970507D54FF6FF53854A2B60137864
:10E678000133DBB21370A3880B40180440F1008308
:10E688000023ADF802302B687B4F9AB21804A280A1
:10E6980040F1F682BB8803F00F03BB71002B40F0FA
:10E6A800C182784A13689BB23B803B8803F03003F1
:10E6B8007B803B8803F440533B8011684BF6BF7363
:10E6C8000B4083F4005383F0200343F4004343F0EA
:10E6D80080031360BB88D90621D4116848F60F73EC
:10E6E8000B40694913600B681A7A022A884601D0E0
:10E6F800042A02D1F9F758FB5AE2062A40F06B8245
:10E708005A78052A08D11A78520605D1D878FFF721
:10E7180082FFBB681B6A9847E3689B685AE21368E4
:10E728009BB2ADF80230BDF802301F0540F1D08130
:10E738001168554F40F68F730B40544913600A68AF
:10E74800534B92B213445B0088461A683B68187AA8
:10E75800092817D092B2520002F1804202F5C04255
:10E7680011781970517859709188C8B2090A41EA2C
:10E77800002159801189C8B2090A41EA002199800B
:10E788009289DA8001221A72DA8893F80190002AB5
:10E7980040F0DC801A7812F07F024AD1B9F1090FF3
:10E7A8000FD1DA78012A00F2B8809978002940F070
:10E7B800B4809988002940F0B0809A72A3685B6899
:10E7C800A9E0B9F1050F10D193F90320002A01DA65
:10E7D8000823B9E09A78002AFAD19A88002AF7D152
:10E7E8009B7A002B00F0A280F2E7B9F1030F0ED15B
:10E7F800DA78012A40F091809A88002A40F08D80CA
:10E808005A7A42F020025A72A368DB6983E0B9F1B0
:10E81800010F40F08280DA78012A7ED19A88002A96
:10E828007BD15B7A980678D5F9F754FB00287DD020
:10E8380073E0012A2ED1B9F10B0F6ED1E268587935
:10E848009269D97890473B689A7A002A65D000285F
:10E8580063D11A79002A60D19B78002B5DD1064BD1
:10E868009B68DB689847084B1B685A79DA72DA7834
:10E878001A735BE0445C004094270020742A00204F
:10E88800ED2F0020005C00400C2A0020505C004066
:10E8980004300020022A40D1B9F1010FC4D0B9F1E7
:10E8A800030F3AD1587920F0800E4FEA8E0202F118
:10E8B800804101F5B84110F0800F096814BF01F0DC
:10E8C800300101F44051BEF1030F26D8B3F802E03D
:10E8D800BEF1000F21D101B39B7AF3B102F180425E
:10E8E80002F5B842010613684BBF23F4E04323F452
:10E8F800804323F0400323F070034BBF9BB29BB2CD
:10E9080083F0100383F4805343F4004343F08003FF
:10E918001360A3689B69984708E0E36848465B6909
:10E92800984703280FD000287FF452AFD8F800206A
:10E93800A14B92B213445B001A6800221A6030237C
:10E948006380062300E009233A6847E1B9F1060F1E
:10E9580012D11A78520678D19B78012B02D1E3683C
:10E96800DB6967E0022B02D1E3681B6A62E0032BD4
:10E978006BD1E3685B6A5DE0B9F1000F38D1598863
:10E98800002962D15A6822F47F42B2F5003F5CD177
:10E998001A7812F07F0204D19B88002B00F0D581F1
:10E9A80053E0012A08D1E268587992699047002813
:10E9B8004BD13B689B7A17E0022A46D15A7902F07C
:10E9C8000F010BB29B0003F1804303F5B84312F02B
:10E9D800800F1B6814BF03F0300303F4405303296E
:10E9E80033D812F0700F30D1002B40F0AE812CE0FC
:10E9F800B9F1080F04D11B785B0600F0A88124E068
:10EA0800B9F10A0F21D11A7802F07F02012A1CD12C
:10EA18009A7AD2B15988C1B95A6822F47F42B2F5BC
:10EA2800803F12D1E268587992699047002800F037
:10EA380090810AE04BB13A684FF00008A2F81280C2
:10EA480093614046984740460BE0E3683A681B6983
:10EA580050789847032804D1584B1B6809221A722A
:10EA6800BDE03A68138A4FF6FF718B4201D1092342
:10EA7800B4E0022800D00BB90823AFE092F90010E7
:10EA880000291FDAD18801910198834202D9019B9C
:10EA9800138210E08B420ED2E16891F82C00834279
:10EAA80001D2002105E093FBF0F100FB113313B90B
:10EAB8000121434B1970E36893F82C309382F9F7DE
:10EAC80073F98CE0032313724FF44053238086E0DC
:10EAD800BDF802301BB2002BBFF6D5AD116840F669
:10EAE8008F730B401360354A17683B7A022B9046A8
:10EAF80071D0042B6FD0032B01D0052B66D1BB69D5
:10EB08003A8A8BB9398A00293BD04FF44053238085
:10EB18002C4B1A68284B92B213445B001A680022E7
:10EB28001A60302363802CE0002AEBD0B7F81490E9
:10EB3800914528BF91461FFA89FA504698473B8A63
:10EB4800CAEB03033B827B8A53447B821D4B1A68C2
:10EB58001D4B92B213445B0009F101021B689BB282
:10EB680003F1005303F5405352105B004FF0000EC1
:10EB78009645C7D053F82E1020F81E100EF1010E3E
:10EB8800F6E7BB8A8B42D8F8003001D8032201E0AF
:10EB980011B105221A720BE006221A72094B1A6883
:10EBA800054B92B213445B001A68196030236380E6
:10EBB800D8F800301B7A0FE0023000200C2A002021
:10EBC800EC2F0020505C004004300020072B02D1BD
:10EBD800E368DB6898470823D8F800201372FFF72A
:10EBE800D8FC5E4B1A684BF6BF7313402288D704D3
:10EBF800228848BF83F480539004628848BF83F416
:10EC08000053D106628848BF83F01003920648BFBC
:10EC180083F0200343F4004343F080034F4A9BB240
:10EC280013602DE09A0002F1804202F5B8421168A3
:10EC380089B2ADF80210BDF8021009B2002909DA4C
:10EC4800106840F68F7101401160013B444A52F848
:10EC580023309847BDF802301F067FF514ADA1791F
:10EC68008B0003F1804303F5B84348F60F72186828
:10EC780002401A603A4B03EB81039B69984702E50F
:10EC8800A28833881340590505D54FF6FF332B600A
:10EC9800344B5B689847A28831880A40920444BF85
:10ECA8004DF6FF732B60A3882F4A0B40DB0452D527
:10ECB8004EF6FF732B6000231374137C052B41D889
:10ECC800DFE803F0030D1418222D6369264D1BB9E4
:10ECD80001F04CFD062300E005232B743BE001F016
:10ECE80045FD042323740123636134E00223637424
:10ECF800032328E0637C013BDBB26374637C53BB72
:10ED0800194B04221A7426E0184A13689BB243F080
:10ED180010031360052323740A2363741BE0637CC8
:10ED2800114A013BDBB26374637C03F0FF0093B9C3
:10ED38000E490C684FF6EF7323400B6006231374DB
:10ED4800506108E00623237405E0094B73E6094B7C
:10ED580071E6094B6FE602B0BDE8F087005C004041
:10ED68002C900108A800002094270020405C004057
:10ED7800597A0008117B0008ED7A000838B5294C4B
:10ED88002DED048B94ED008AB0EE480A0546FAF79B
:10ED98009DFDF0EE408AB0EE480AFAF734FD94ED96
:10EDA800019AB0EE408AB0EE490AFAF78FFDF0EE0C
:10EDB800409AB0EE490AFAF726FD95ED017AD5EDAD
:10EDC800027A95ED006A68EE676A27EE088AE7EE30
:10EDD800286A68EE000A67EE807AE6EE290AB0EE45
:10EDE800660AE7EEA80A07F0CDFADFED0F7A20EE03
:10EDF800270ADFED0E7A80EE270AD4ED027A30EE8C
:10EE0800270AF2EE047A80EE270A07F0B9F9BDEC7A
:10EE1800048B83B21A0444BF00F5B47083B218B2ED
:10EE280038BD00BFAC2700200000E144DB0F49409B
:10EE38002DE9F04F2DED028B85B007460293A14BCB
:10EE48001B889807934636D5109B9F48DC89B0F9F4
:10EE580000301B1B03F2F31540F2E632954203D84B
:10EE6800002BB8BF5B4201E04FF4FA73B0F90220FF
:10EE7800121B02F2F31440F2E630844203D8002A4F
:10EE8800B8BF524201E04FF4FA729342B8BF13463A
:10EE9800C3F5FA73052293FBF2F30A22643B53434A
:10EEA8003A7FD2105343642293FBF2F3134423EACC
:10EEB800E373DBB200E064230093CB1C0193B846F4
:10EEC8000024019BDFF828A213F8016F0193022C9C
:10EED8004FEA440905D1BAF904301B365E4376116E
:10EEE80046E07A493AF8142031F91410022012FB4E
:10EEF8000011CBF10002914203DB59450A46A8BF35
:10EF08005A467349029B31F90950551B33F91420AD
:10EF1800154403F097FB88B107EE905A6D4AB8EE96
:10EF2800E70AB2EE048A105D80EE080A03F03EF9A3
:10EF380020EE080AFDEEC07A17EE905A614A128850
:10EF4800D10712D43AF909301B365E4393074FEACA
:10EF580026160DD5BB7C5D439DF900305D436423C7
:10EF680095FBF3F506EB251602E03E7A75432E1164
:10EF7800594B042533F9093093FBF5F5574B03F149
:10EF88000C02751BA25C924698F8012051466A4310
:10EF98004A43642192FBF1F297F85110D21108EE1E
:10EFA800102AB1B1022CB8EEC80A08D14A0803D019
:10EFB8009142A8BF114600E00121494803E003F14E
:10EFC800100000EBC400D3ED0A0AFAF7B9F9BDEE58
:10EFD800C08ADFF808E1434B98F80B6018880EF1F7
:10EFE8002C0300FB05F253F82410D21206FB02167C
:10EFF800B6F5001F3C4AA8BF4FF400169642B8BFAA
:10F0080016460EF1380243F8246052F8243042F8CC
:10F018002450EB1A0EF144014FF6FF720009B2FBBF
:10F02800F0F043430EF1500051F8245050F82420DA
:10F0380040F824509B112A4441F8243097F8501086
:10F048001A444FEA840C761300EE102A79B10EF1B7
:10F058005C00B8EEC00A00EBC400DEED0A0ACDF889
:10F068000CC0FAF76DF9DDF80CC0BDEEC00A98F8CF
:10F07800153010EE102A18EE101A5A43534653430F
:10F088001A463144642392FBF3F3184A1B121944BD
:10F0980022F8091018EE100A02F1080101344CF8A0
:10F0A800010002F114012032032C4CF801604CF8E5
:10F0B800023008F101087FF404AF05B0BDEC028B03
:10F0C800BDE8F08F081B0020942E0020E22F0020BE
:10F0D8004E2E00206890010888110020AC270020DF
:10F0E800CC2700205C1100200000E0FF2028002031
:10F0F800481200202DE9F04F2DED048B944CDFF8D9
:10F108005482D4F8A4308DB0064692489847914866
:10F1180094F8B4200146F9F70FFA8F4B19889946ED
:10F1280004F58272002973D0D4F8B8301B7808EE41
:10F13800103A04F1BC0A04F1C8054FF0000BB9F805
:10F14800007038F91B00B7F57A7F02BF0023CAF8B0
:10F1580000302B61DAF800300344CAF800302B691C
:10F1680007EE900A0133012B4FEA4B01F8EEE77ADC
:10F178002B6106D10023C5ED017AC5ED007AAB609D
:10F188001BE0D5ED006A07EE103A37EEE66AB8EEF6
:10F19800C77A86EE077A36EE877AD5ED026A85ED6C
:10F1A800017A77EEC77A85ED007AE6EE276AF0EE07
:10F1B800667AC5ED036AC5ED026A0023012F28F8B7
:10F1C800013053522FD12B69012BC3BF03F1FF33F9
:10F1D80000EE103AD5ED037A9FED600AC8BFB8EE8D
:10F1E800C00A8DE80600C8BF87EE800A07F06EFAED
:10F1F8009DE8060018EE103A63B1F8EEC87AB4EE4E
:10F20800E70AF1EE10FA05DD4FF47A73A9F8003039
:10F2180000231CE0DAF800304FF47A7003F5FA7333
:10F2280093FBF0F353520BF1010BBBF1030F0AF1FF
:10F23800040A05F1140582D1012F04D13846009241
:10F24800FCF780FA009A013FA9F80070E0E738F867
:10F25800131032F813003E4D091A28F81310013321
:10F26800032BF4D13E4F3B6813F0020300F0C88231
:10F278003C4B05F585705B6898473B4B05F58570F9
:10F288001A780146F9F758F9B5F8103105F5857976
:10F29800002B41D0D5F814010023B4F810213349CC
:10F2A80039F913E02A4DB2F5C87F04BF002241F8AE
:10F2B80023204FEA830C51F80C20724441F80C20AB
:10F2C800002129F8131020F813100133032BE4D17F
:10F2D800B5F81031012B1AD1D5F818314FF4C87E82
:10F2E800C83393FBFEF30380D5F81C21C83292FB88
:10F2F800FEF242801E4AD5F820311288C83393FBAB
:10F30800FEF39B1A838031807180FAF72FFEB4F8E0
:10F318001031013BA4F81031164B1B68590740F116
:10F328008D80B4F824210A4B322A25D1D3F8142130
:10F338001188A3F8261151889288A3F82A213288C7
:10F34800A3F82C217288A3F82811A3F82E2115E020
:10F35800AC27002088110020E62F002000000000C4
:10F36800401A0020702B0020EE2F0020C428002017
:10F3780004000020582E0020002A3ED0D4F814A102
:10F388000023B4F82421AA4939F91300A94D322AD7
:10F3980004BF002241F823204FEA830E51F80E20C3
:10F3A800024441F80E20002229F813202AF81320DD
:10F3B8000133032BE5D1B5F82431012B18D10C20EA
:10F3C80085F83D3185F83C21FCF7BCF9B5F82631C4
:10F3D800AAF80030B5F82831AAF80230B5F82A3171
:10F3E800AAF80430B5F82C313380B5F82E31738083
:10F3F800B4F82431013BA4F8243194F83E318D4A05
:10F40800E3B1D2F81451D2F83001002182F83E114C
:10F418004FF0320E90FBFEF02880D2F8340190FBBA
:10F42800FEF06880D2F83831834A93FBFEF31288E5
:10F438009B1AAB8031807180FAF798FDD4F81421BB
:10F44800B4F80A3111885B1AA4F80A315188B4F863
:10F458000C315B1AA4F80C319288B4F80E319B1A5F
:10F46800A4F80E31FCF7A8F9D4F8403194ED516AAC
:10F47800D4F84861C4F84001C3EB000A07EE90AA2B
:10F48800B8EE678A002528EE066A96F800C06B4831
:10F498006B490DF10C0E2A4638F9123007EE903AF6
:10F4A800F8EEE77A67EE867AEEEC017ABCF1000FA7
:10F4B8001CD007EE90CAF8EEE76AB7EE007AC7EEFE
:10F4C800266A39F9123007EE903AF8EEE77A37EE05
:10F4D800667A67EEA67AD1ED006AE6EE877AC1ED24
:10F4E800007AFDEEE77A17EE903A01E039F812302B
:10F4F800438030F8023F0132032A13FB035501F120
:10F508000401C9D1DFF830814E4864236B43B8F851
:10F5180000506D4393FBF5F5493D03A9ADB2FAF7E9
:10F528003BFA3B2DD6ED016A11D9B4F96431D4ED1B
:10F53800580A07EE903AF8EEE77A434BF4EEE70AFA
:10F54800F1EE10FA1EDD1A7842F008021DE0F7EE1F
:10F55800007A36EEA77A3B4A87EE877A00233B4942
:10F5680031F913100133032B07EE901A92ED006A5C
:10F57800F8EEE77AE6EE267A67EE877AE2EC017A29
:10F58800EDD1D2E71A7822F0080294ED570A1A70E2
:10F5980006F0F8FEB0EE409A84ED000A94ED580AA1
:10F5A800D4ED577AD4ED568ADFED299A294D20EE0D
:10F5B800000AF1EE688AA7EEA70A07F087F8F0EECE
:10F5C800400AB0EE680A06F0DDFEF0EE408A84EDEF
:10F5D800010A29EE290A06F0D3FD28EEA90A288097
:10F5E80006F0CEFD3B6868801A0739D51A4803A98A
:10F5F800FAF7D2F9D6ED026A174AF7EE007A36EE34
:10F60800A77A002387EE877A144931F9131001335A
:10F61800032B07EE901A92ED006AF8EEE77AE6EE11
:10F62800267A67EE877AE2EC017AEDD10A4842E061
:10F63800DC280020AC270020040000203012002025
:10F64800F828002004290020441A00203212002043
:10F658004C3D0F444E2E0020142900208E1100200E
:10F668006D4D03A92846FAF797F995ED010A95ED2E
:10F67800007AD5ED027A20EE000AA7EE070AA7EE77
:10F68800A70A07F023F8B5EE400AF1EE10FA11D0F8
:10F69800D5ED007AC7EE807AC5ED007AD5ED017A0E
:10F6A800C7EE807AC5ED017AD5ED027A87EE800A39
:10F6B80085ED020A5848FFF761FB584BDFED587A91
:10F6C8001880564B9FED577AB3F9003028EE278AF9
:10F6D80007EE903A544BF8EEE77AB3F9002067EE5C
:10F6E800C77AB1EE499ACDED087A07EE902AB3F9B8
:10F6F8000220B3F904308DED069AF8EEE77AF1EEC0
:10F70800688ACDED097A07EE902AF8EEE77A09A81B
:10F71800CDED0A7A07EE903AF8EEE77A06A9CDED34
:10F72800078ACDED0B7AFAF737F973789DED0B7AE6
:10F73800012B19D13D4B1B785B070FD4D4F87431DA
:10F74800402293FBF2F29B1A07EE903AF8EEE77A22
:10F7580077EE877AFDEEE77AC4ED5D7AD4F87431F6
:10F76800402293FBF2F301E0B8F800309DED090A5E
:10F7780007EE903AF8EEE77A37EE677AD4ED5E7ADC
:10F788008DED0B7A94ED5F7A38EE077A88EE078A6A
:10F798009DED0B7A37EE677AE8EE077AB0EE678A66
:10F7A800C4ED5E7A06F0ECFCD4F880512978FAF7BB
:10F7B8001BF8D4F884319DED0A0A1844C4F8840172
:10F7C80006F0DEFC2978FAF70FF8D4F88831B0EEA5
:10F7D800480A1844C4F8880106F0D2FC6978FAF798
:10F7E80003F8D4F88C31124A18441368C4F88C0111
:10F7F80053441360D4F890310133C4F8903105E0D4
:10F80800A5F80A31A5F80C31A5F80E310DB0BDECFC
:10F81800048BBDE8F08F00BF60000020401200207C
:10F82800BD37863535FA8E3C32120020EA2F00208B
:10F83800CC2F002001380A4B042804D8DFE800F058
:10F848000507090B0D00074A08E0074A06E0074AC2
:10F8580004E0074A02E0074A00E0074A1A607047D6
:10F8680000010020C1B1000839EE00087126010826
:10F8780073AE0008D1AA000841A5000810B54B884E
:10F88800DC0641BF2F4B14791B6853F8244044BF52
:10F898002D4B43F820404B889B0641BF294B547998
:10F8A8001B6853F8244044BF274B43F820404B883B
:10F8B8001C070ED5254B0C781B78B3EB141FA1BF82
:10F8C800204BD4781B6853F82440A4BF1E4B43F840
:10F8D80020404B889B070ED51D4B0C781B78B3EB4B
:10F8E800141FDFBF174B54781B6853F82440DCBF44
:10F8F800154B43F820404B88DC070FD5154C0B7887
:10F90800247803F00F03A342DFBF0E4B14781B6863
:10F9180053F82440DCBF0C4B43F820404B885B076E
:10F928000FD50B780C49097803F00F038B42A1BF60
:10F93800044B92781B6853F82220A4BF024B43F86B
:10F94800202010BD882100200A0E00209F1E0020C4
:10F958009D1E00209C1E00209E1E0020254A264831
:10F9680026490023F0B5156803700B701C461A462B
:10F978002E1976884EB92F5D3FB9037000230A709F
:10F988004B7007781C461A460CE0360548BF013212
:10F9980004F1040403F1010348BFD2B2802CDBB2A6
:10F9A800E6D1EAE7E0B2B8420CD215F8240006091D
:10F9B8009E4200F00F00A8BF731C9042A8BF421CD3
:10F9C8000134EFE78A704B70C2F3470102F001027D
:10F9D8000A444C1E0A490B480A70C3F3470203F055
:10F9E8000103134404700849501E084A0870137034
:10F9F800F0BD00BF90270020941E00204029002061
:10FA08009E1E00209C1E00209F1E00209D1E002080
:10FA18002DE9F04FC24BDA682DED028B1A61C14A0D
:10FA28001168D960C0490B6843F020030B60BF4BD5
:10FA38001978012990460CBF002201221A70BC4B8C
:10FA48001A78910789B040F13D83BA4909780429A9
:10FA580040F23883B849097801F0040101F0FF0049
:10FA680011B922F001021A701B78DB0702D408B121
:10FA7800F7F770FFB149CA78531C052293FBF2F2DD
:10FA880002EB82029A1AAE4BCA701B78039392005B
:10FA98000023AC4CDFF8CCC2DFF8D8925CF8231016
:10FAA80091FBF9F504F1080004F1100640F8235021
:10FAB800A54844F8231000FB051142F2107091FB91
:10FAC800F0F080B226F813004FF0140E04F114067B
:10FAD80004F13C0A0EFB036E5AF823605EF80270CC
:10FAE8004EF80210F61B314444344AF82310052618
:10FAF80091FBF6F109FB051144F82310039C012C36
:10FB08004FEA830BE24605D10238B0F5797F98BFFA
:10FB18004BF80C100BB90123BBE7884CD8F8003020
:10FB2800226D9FED8A7A8A4E8A4D9B1A07EE903A8B
:10FB3800F8EE677AD8F800302365C7EE877A7C4BF1
:10FB48001B78B7EE008AF4EEC87AF1EE10FA58BFC7
:10FB5800F0EE487A13F00103C4ED157A12D005AA25
:10FB680000927D4B06AA01920CCB9AE80300F7F7A6
:10FB7800EFFD6421059A069BB2FBF1F293FBF1F3CA
:10FB8800328000E033802B8094F858306B48002B8B
:10FB98003BD0D0ED157AC26DDAF80030C8EE276A8E
:10FBA8009B1A026E022507EE103AB8EEC77ADAF809
:10FBB800043027EE267A9B1AFDEEC77AB0F9662044
:10FBC80017EE901A07EE903A644BB8EEE77AD3ED49
:10FBD800007A67EE277A67EEA67AFDEEE77A17EEE7
:10FBE800903A02FA83F3B0F9642093FBF5F302FA32
:10FBF80081F29BB292FBF5F292B2A0F86A30A0F8BB
:10FC08006820A0F86630A0F86420012384F85830F2
:10FC1800534BDAF804101B88DAF80000474D514EB0
:10FC2800216603F03003E065002B00F04B8205F1FC
:10FC38007403009305F178030193EA6E2B6FF7F7CD
:10FC480087FD72682B6F9B1A07EE903A434B326818
:10FC580093ED007AEB6EF8EEE77A9B1AEB67384B78
:10FC680067EE877A1B78FDEEE77A012BC5ED207ADF
:10FC780003D0022B00F0DF8024E2D5ED287A3A4B3E
:10FC8800D5ED215A95ED255A95ED156A95ED264A3B
:10FC9800D5ED274A35491D68B1EE677ABDEEC77ABA
:10FCA800FDEEE77A17EE10EA17EE90CA0020304A08
:10FCB80091ED007A52F8207007EE907AF8EEE77A24
:10FCC800A2F1140367EEA57A33F81060FDEEE77A27
:10FCD800283217EE903A9B1B9BB222F810301BB2C9
:10FCE80007EE903AF8EEE77A3B4467EE857A4400EF
:10FCF800FDEEE77ACDED037A07EE903AF8EEE77A73
:10FD0800BDF80C8067EE847AA7EE867AFDEEC77A96
:10FD180017EE902A724531DB6245A8BF62462EE095
:10FD2800000800207C2E0020401A0020CE11002060
:10FD3800441A00204A1A0020EA2F002040290020F7
:10FD48008C0F002044290020806967FF00007A4456
:10FD5800BE1A0020C01A0020D01100206C0000201C
:10FD6800081B00204C1A0020900F0020C00F002014
:10FD7800BC29002080969800DB0FC940724607EE28
:10FD8800902AF8EEE77A5FED046AC1ED007AFDEE9D
:10FD9800E77A313617EE903A43449AB2AB78D1ED10
:10FDA800027A07EE103AB8EE477A4B684F6027EEB2
:10FDB800267AFB1A88EE077AB6B2622E06EE903AD9
:10FDC800F8EEE66A37EE067AC6EE866A86EE077AB7
:10FDD80076EEE76AE7EE267AC1ED047AC1ED027A9B
:10FDE8000FD964EEA77ABA4EFDEEE77A17EE903A8D
:10FDF800B3F5FA6FA8BF4FF4FA63B342B8BF3346FE
:10FE080000E0002313441BB240F6B8329342A8BF67
:10FE18001346B04A9342B8BF1346AF4AA352AF4AFB
:10FE2800142303FB002351F8142B1A60002840F018
:10FE3800498101203BE7AA4BD5F874801F68D4F8A4
:10FE480078903E89DFEDA78A4FEA58039E4228BF83
:10FE58001E46B5F8A8301AB29642C3BFD5ED157A3A
:10FE68009FEDA17A67EE877AB6B2C1BFFDEEE77A59
:10FE780017EE906AF618B6B2C8BFA5F8A860D4F80D
:10FE8800AC50C5EB09052846F7F7A6FC0028D8BFF3
:10FE9800404241F293129042CCBF0020012088B327
:10FEA80007EE905AB8EEE70A20EE280AF9F7ABFCFD
:10FEB80007EE908AF8EE677A40F6B83320EE270A04
:10FEC800FDEEC07ACDED037ABDF80C20A4F8B02081
:10FED80012B29A42A8BF1A467E4B9A42ACBF09EBAF
:10FEE80002034B4448F6A042934203DDA3F50C43BA
:10FEF800A03B04E0002BBCBF03F50C43A033C4F8BF
:10FF0800B43001E0C4F8B490D4F8B450C5F50C533B
:10FF1800283307EE903AF8EEE77A67EEA88AB0EE53
:10FF2800680AF9F7D3FC8DED070AB0EE680AF9F70D
:10FF38006AFCD4ED317AD4ED2E4AD4ED155A94EDFD
:10FF48002F4A94ED305A65498DED060AB1EE677A6D
:10FF5800BDEEC77AFDEEE77A0DF1180E17EE10AA7E
:10FF680017EE90BA0020614AFEEC016A32F91030AF
:10FF7800DFF88C9107EE903A07EE106AF8EEE77A10
:10FF8800B8EEC77A3C32D6EE877A4FEA400CFDEEDF
:10FF9800E77ACDED037ABDF90C30B3F57A7FA8BFC7
:10FFA8004FF47A734B45B8BF4B461FFA83F922F8D2
:10FFB80010900FFA89F207EE902AF8EEE77A27EE0A
:10FFC800A47ABDEEC77A8DED037A27EE847AD1ED57
:10FFD800007ABDF80C90E7EE257AFDEEE77A17EE89
:10FFE800902A524503DB5A45A8BF5A4600E05246BC
:08FFF80007EE902AF8EEE77A0B
:020000040801F1
:100000009FED3D6AC1ED007ABA7891ED027A06EE75
:10001000902AF8EE666A4A684B6066EE866A9A1A1B
:10002000C8EE266A143106EE102AB8EEC66A76EEDD
:10003000A56A86EE256AC5EEA66A36EE476AA6EE82
:10004000867A01ED017A01ED037A25EE077ABDEE9D
:10005000C77A17EE103ABDEEE77A4B4417EE102A36
:1000600013441BB240F6B8329342A8BF13461B4A52
:100070009342B8BF13461A4A2CF802301F4A142381
:1000800003FB0023C3ED007A08B901206FE73B7939
:1000900023B1642395FBF3F5194B1D803B889845EC
:1000A0000DD9D4F8AC30A06FC01AF7F799FB80EAED
:1000B000E072A2EBE07242F210739A4206DD114B3D
:1000C00001221A700E4BB4F8C8201A8009B0BDEC9A
:1000D000028BBDE8F08F00BF30F8FFFF48F4FFFF50
:1000E00014100020E80F0020900F0020D3023739B1
:1000F0000000C842A8290020DB0FC940C00F002023
:10010000880F00208C0F002018FCFFFF20B9034B44
:100110001B6808221A827047014870470C2A002089
:100120007000002020B9034B1B6808221A82704718
:10013000014870470C2A00207000002021B90128D6
:100140008CBF0220002070470220704710B5094B79
:100150001A68D378042B0BD8074C518ADB00234450
:1001600018B99B895B1A138210BD9B68581810BD83
:10017000002010BD0C2A002070000020054B1968DB
:10018000054B4A8A18B99B8D9B1A0B827047986A57
:10019000104470470C2A002070000020054B19689D
:1001A000054B4A8A18B99B8E9B1A0B827047186BB5
:1001B000104470470C2A002070000020074B1B6879
:1001C0001B7803F07F03212B06D100F0DF0002280B
:1001D00014BF022000207047022070470C2A002024
:1001E000212810B508D1114B1B681B7803F07F0341
:1001F000212B10D0022010BD2028FBD10B4B0C4A24
:100200001B6810701B7803F07F03212B094B18BF6C
:1002100000230BB9EEE7084B044A126800249361EF
:10022000548220469847204610BD00BF0C2A00206B
:10023000EF2F00200D010108250101087047034B35
:100240001A78202A04BF00221A707047EF2F00206E
:10025000014B04221A607047D02F0020034B9B7B78
:1002600013B1034B05221A60704700BF0C2A00200F
:10027000D02F00200D4B0E491A680E4B92B213443A
:100280005B000D4A1B68C3F3090310B51362136AC0
:100290009BB201335B1000229A4206D0074851F806
:1002A000044B20F812400132F6E710BD505C0040CC
:1002B000206200401E3000200C2A0020302A00203E
:1002C000014B00225A6670470C2A00202DE9F843A2
:1002D000664B674E1B68DFF8B881664A00254FF011
:1002E000C0099D7283F80990DD723560D8F800303E
:1002F00023F4EC4323F0700343F400739BB2C8F87B
:100300000030D8F8003023F4E04323F040039BB2E0
:1003100048F2800483F010032343C8F800303368A8
:1003200012FA83F35B0040271A681F6033689BB2A0
:1003300003F1005303F540535B0028461A688022FE
:100340001A60D8F8003023F4F8731B051B0D234303
:10035000C8F80030484B93F86410F7F79DFDD8F8C3
:100360000030464A464923F4804323F070039BB291
:1003700083F440532343C8F80030136823F4EC435C
:1003800023F070039BB21360336811FA83F35B00B0
:1003900003201968C3F8009013683A4923F4E04336
:1003A00023F040039BB283F02003234313601368C0
:1003B00023F4804323F0700323439BB213605368FC
:1003C00023F4EC4323F0700343F4C0639BB2536007
:1003D000336811FA83F35B0019684FF48071196078
:1003E000536823F4804323F0700323439BB253608C
:1003F000536823F4E04323F040039BB283F02003CF
:1004000023435360D8F80C301F4A23F4EC4323F005
:1004100070039BB2C8F80C30336812FA83F35B00A8
:1004200039461A684FF488721A60F7F735FDD8F824
:100430000C3023F4804323F070039BB283F44053C9
:100440002343C8F80C30D8F80C3023F4E04323F0F1
:1004500040031C43A4B2C8F80C402846FEF7DFF85E
:100460000A4B01221A60BDE8F88300BF0C2A002065
:10047000505C00400430002070000020045C00400C
:1004800008300020103000201C300020D02F002029
:10049000005C0040134A144B50681B68181810B5D4
:1004A000146808D011490822FEF7A5F82046104923
:1004B0000422FEF7A0F80F480268002393720E4A48
:1004C000012111600D4913604FF4E0540B6014607A
:1004D0000B604FF43641A0F868101160084A1360B1
:1004E00010BD00BFB0F7FF1FACF7FF1FDA00002000
:1004F000EA0000200C2A0020405C0040445C0040E0
:10050000D02F002010B50446B0F9000001F027F903
:10051000B4F9020001F023F9B4F90400BDE8104079
:1005200001F01DB910B50446006801F018F96068C3
:1005300001F015F9A068BDE8104001F010B92DE9EF
:10054000F74F0120FBF70AF8002488B3012C2FD8BD
:10055000194E4FF04C0909FB04FA06EB0A0808F1A2
:10056000B407BD7815B10134E4B2EEE790F900307C
:1005700090F804E01846114B03228DE82400012175
:100580002A4653F82E30FBF74CF9834660B106F14A
:100590006C00504429464A4605F0E7FB01231C4401
:1005A000C8F86CB0BB70E4B20120FAF7BDFFCCE72D
:1005B00003B0BDE8F08F00BF0C2A00206C9001084A
:1005C0000021222210B5114805F0CFFB104B00226C
:1005D000194610480424105C83F8F6010132052006
:1005E00083F8FB41042A4FF0000483F8FA0183F8F2
:1005F000FD4183F8FC0103F10803EAD10123A1F8CE
:10060000F831522381F8F43110BD00BF44140020AA
:100610005012002047B3010810B5F7F795FD4FF4CD
:100620003024012806D11CB1F7F78EFD013CF8E714
:10063000052010BD002C08BF052010BD70B5064672
:10064000441E14F8011F89B1094D284605F0C3FB6B
:100650000028F6D005F1080398423FBF054B401B28
:10066000C018A31B38BF80F88A31EAE770BD00BF0D
:10067000CEBF01085012002007B51D4B03F5847250
:10068000C3F804211B4A92F892215AB1012A14D1CD
:10069000032183F80A11072183F80C2183F80B1139
:1006A0000C2208E0022183F80A11032183F80C21AF
:1006B00083F80B11072283F808210F4B0F4AC3F868
:1006C00084204020FAF74AFF70B10122002390F9FC
:1006D000000040218DE80C00094A4FF4E133FBF79C
:1006E000A0F8003018BF012003B05DF804FB00BF84
:1006F0000C2A00205012002070000020ED7B000822
:10070000197D00080120002100F09EB9F0B5184ABB
:1007100092F80D31D2F810711546032B11D807EB62
:10072000C3025E1C941CF6B209D013469288D1070E
:1007300005D5104203D008E00131042908D1334621
:10074000EBE785F80D310020F0BD93F802E00021C1
:10075000074C0C2204F58A7C02FB01F31CF80320F1
:100760009645E9D1234484F80D61D3F81801F0BD12
:100770000C2A00200A4B10B519684FF6FB720A408C
:100780001A60084A927B1C46074B0AB1052200E01A
:1007900001221A6000F0B4FE4FF43643236010BD0E
:1007A000405C00400C2A0020D02F002007B5064BEB
:1007B0000093064B01930649064A074B0748F8F792
:1007C000F7FF03B05DF804FBE4A40108B9A4010835
:1007D0008AA9010883A90108D8A401084BB301081C
:1007E00008B5037833B90C4B0C481978BDE80840BC
:1007F000F8F7DEBF05F054FB02280CD8064B187042
:10080000074B0C2202FB0030064B0230186000F050
:10081000D7FB0548E5E708BD502B00206BB3010866
:10082000001A0020C8110020D2A7010808B50378DB
:100830003BB90B4B0B4893F8B017BDE80840F8F7ED
:10084000B7BF05F02DFB022808D8054B83F8B00789
:10085000F9F736F9F9F7D4F90348E8E708BD00BF1E
:10086000501200206FB30108D2A7010838B50378F1
:1008700003BB214B1B6801330F2B07D81F490C22E8
:1008800002FB03121C4695682DBB00E01C46013498
:100890000F2C01DD002400E005D818490C2202FBD2
:1008A00004129568BDB99C42F1D11548BDE83840A5
:1008B000F8F77EBF05F0F4FA0F28044605D80F4A72
:1008C0000C2303FB00239D682DB921460D48BDE88C
:1008D0003840F8F76DBF084B1C60FAF725FF21463A
:1008E0002A460948F8F764FF0C235C43034B185D64
:1008F000BDE83840FAF72ABFF80000202C91010823
:100900007CB3010892B30108AAB3010873B5037858
:1009100013B9FDF7ADF93DE01F4901AA05F021FB30
:10092000002401462646254699B134B1012C08D150
:10093000084605F0B5FA064603E0084605F0B0FAA9
:1009400005461549002001AA05F00BFB01340146BC
:10095000EAE70B2D02D911480C220BE0022C10D132
:10096000A6F57A73B3F57A7F07D90D484FF47A71FB
:100970004FF4FA62FDF7F9F80CE00A4B03EB45037C
:100980005E80084B084803EB45032946B3F9022073
:10099000F8F70EFF02B070BDD5AB0108EBAB010854
:1009A0001FAF0108502B0020C1B3010838B50D4C12
:1009B00023688342054606D1FDF7DBFD2046002172
:1009C0004C2205F0D2F9E36CAB4209D12846FDF781
:1009D000D0FD054800214C22BDE8384005F0C5B9DE
:1009E00038BD00BF782A0020C42A0020034B1A68B3
:1009F000D379591C1344D171187A7047E81A002032
:100A000010B5FFF7F3FF84B2FFF7F0FF04EB00200F
:100A100080B210BD10B5FFF7F3FF0446FFF7F0FFFB
:100A200004EB004010BD064B10B504462146186883
:100A3000FBF780F8034B1B6898796040987110BDF4
:100A4000EC1A0020E81A002038B5044624200D4690
:100A5000FFF7E9FF4D20FFF7E6FF002C084C14BF1D
:100A600021203E20FFF7DFFF2368002228469A71ED
:100A7000FFF7D9FF236893F84900BDE83840D2E773
:100A8000E81A002001460020DEE710B50446C0B297
:100A9000FFF7C9FF200ABDE81040C4E710B50446BF
:100AA00080B2FFF7F2FF200CBDE81040EDE737B54C
:100AB00082888368044610060D4641BF2B4991F891
:100AC000B0174FF4CC7000FB0133D10544BF284967
:100AD000097802F03F0244BF01EB410103EB8103BF
:100AE000042A12D006D8012A0DD0022A32D193F955
:100AF000001030E0102A0AD0202A0AD0082A29D172
:100B0000B3F9001027E0197825E0198823E0196867
:100B100021E093ED000A6846F8F7CAFC0146154843
:100B2000F8F746FE05B3D4ED037A6846B8EEE70A57
:100B3000F8F7BEFC01461048F8F73AFE94ED040AB7
:100B40006846B8EEC00AF8F7B3FC01460A48F8F761
:100B50002FFE09E000210948F8F72AFE25B10848D0
:100B6000E1682269F8F724FE03B030BD501200207E
:100B7000502B0020BAAA0108B3AA01085EAA0108F6
:100B8000D0B30108024B0146D869FAF7D3BF00BFC2
:100B9000502B002010B5441E14F8011F21B1034B47
:100BA000D869FAF7C7FFF7E710BD00BF502B002048
:100BB000F7B52B492B4B08782B4D1C682B4B05EBBD
:100BC00080001A882A4BD0F8C0101B782948009161
:100BD0004FF47A71B4FBF1F1F8F7EAFD26484821A9
:100BE000F8F7E6FD254B1F680026F3B205EB8302FC
:100BF000D2F8D010E9B101249C403C4217D0220722
:100C000015D01F4AD25C0B2000FB0323164A1D4857
:100C100002EB8303D3F8F020F8F7CAFD022C06D1CB
:100C2000194B93F8281011B11848F8F7C1FD013697
:100C3000DBE71748FFF7AEFF164B17481A68174B4C
:100C40009A420CBF164B174B1A88174B198892B251
:100C500040F2DC7303B0BDE8F040F8F7A9BD00BF77
:100C6000901A00207C2E00202C910108301A0020C0
:100C7000FC000020D7B301081AB40108401A002074
:100C8000040100202AB40108502B002032B40108CE
:100C90007AB401086011002036B401080054004005
:100CA00064110020661100205C1100202DE9F04144
:100CB0000024804625460F4EA7594146384605F088
:100CC000D7F858B139460C48F8F772FD30190021B1
:100CD000FFF7EDFE0948FFF75DFF0135143440F6DC
:100CE000BC439C42E7D11DB90548BDE8F04151E73E
:100CF000BDE8F081CC92010840AB01087AB401084C
:100D0000E2AA01082DE9F04F2DED028B83B00546D4
:100D100005F06FF8064620B1012818D12B782A2B50
:100D200015D15C48FFF736FF00245B4D5B486159E5
:100D3000F8F73EFD28193146FFF7B9FE5848FFF78E
:100D400029FF143440F6BC439C42EED19CE0284677
:100D50003D2105F040F8002800F08F8003469946B9
:100D600013F8012D202AFAD0441C204605F098F8EB
:100D700080462046F8F712FBC5EB0909B0EE408A21
:100D80000026DFF834A1142202FB06F40AF5D07B1A
:100D900054F80B70384605F02CF803461A462846DE
:100DA0003946019305F02EF8019B00285BD15FFACC
:100DB00089F29A4257D10AEB0402D2ED6B7AF8EE2F
:100DC000E77A0BEB0405B4EEE78AF1EE10FA48DBA4
:100DD000D2ED6C7AF8EEE77AB4EEE78AF1EE10FA2B
:100DE0003FD8B2F8A431D2F8A82113F0200F08BFE1
:100DF00008EE108A1C0641BF2A4991F8B0174FF43B
:100E0000CC7404FB0122D90544BF2749097803F0BB
:100E10003F0344BF01EB410102EB8102042B18EEBA
:100E2000100A0BD004D8013B012B0ED810700CE037
:100E3000102B05D0202B06D0082B06D1108004E003
:100E400082ED008A01E082ED008A39461748F8F702
:100E5000AFFC2846002103B0BDEC028BBDE8F04F8B
:100E600025E6134803E00136A32E8AD1114803B0CA
:100E7000BDEC028BBDE8F04F8CE6284603B0BDEC1C
:100E8000028BBDE8F04F11E703B0BDEC028BBDE86B
:100E9000F08F00BF68B40108CC92010840AB010894
:100EA0007AB4010850120020502B00207DB40108B4
:100EB00088B40108E2AA01082C91010870B5054622
:100EC000284604F096FF064658B9194B19485A7936
:100ED000194B03EB8203BDE87040D3F8581EF8F7B6
:100EE00067BC28461549324604F08CFF60B91448A7
:100EF000144CFFF74FFE54F8041F19B11248F8F7CD
:100F000057FCF8E7114805E00024114B53F8241072
:100F100019B91048BDE870403CE62846324604F056
:100F200071FF01340028F0D1014B0B4D5C71C7E714
:100F300050120020A8B401082C910108D1AA010880
:100F4000B4B40108849F0108CDAA01087AB401084D
:100F5000889F0108E2AA0108D2A7010808B507483E
:100F6000FFF718FE064BD869FDF7F8FAFAF740FFCD
:100F7000F8F77CFD034B044ADA6008BDC7B40108EA
:100F8000502B002000ED00E00400FA0508B50548EC
:100F9000FFF700FE00F05CF8F8F792FDBDE80840AE
:100FA000DCE700BFD3B4010808B50448FFF7F2FD41
:100FB000F8F786FDBDE80840D0E700BFE9B40108B6
:100FC00010B50E4C2068FAF719FB2068047A00224D
:100FD00002FB02F3193B634303F6C4135343192185
:100FE00093FBF1F3064921F812300132072AEFD1C1
:100FF0000449BDE81040FAF7B7BA00BFC811002095
:1010000018100020941300200F4B1A78692A17D16A
:10101000598840F2DC72914212D11A79BE2A0FD15E
:1010200093F8D927EF2A4FF000000BD113F8012BCA
:101030005040064A9342F9D1B0FA80F04009704717
:1010400000207047704700BF00F80308DCFF03086A
:101050002DE9F04F2DED028BE94D002140F2DC72BD
:1010600085B0284604F081FEE64B05F53A721A6019
:10107000E54A00231370E54A05F2B2711160692256
:101080002A7003226A7140F20112AA604FF41672AC
:10109000A5F86621FA22A5F86821BC22A5F86421EA
:1010A0004FF4FA722021A5F86E21012285F8622101
:1010B00085F86A1185F87E216E2185F88621052242
:1010C00085F87C1185F827220A2140F2DC5285F848
:1010D0007D11A5F898212B2140F24C4285F87F1113
:1010E000A5F89A21212140F26C7285F88011A5F8AB
:1010F0009C21232140F2753285F88111A5F89E21AB
:101100004FF4C87140F64302A5F8A021A5F882115A
:101110002A462C46032BCCBF0121002103F10103F9
:1011200082F8A21114BF1E217521122B82F8A3117F
:1011300002F10202EED14FF4FA63A4F8C831A4F828
:10114000CC31A4F8D031A4F8D43140F27E4105234B
:1011500040F27E5684F8E231A4F84411C82340F2EC
:101160003A71A4F84C6140F2EA5601274FF47A79BB
:101170004FF0320BA4F8E631A4F846114FF4C873CF
:1011800040F2DC51A4F84E61DFF878A2A4F8EA310D
:1011900040F2B4561E201922A4F84A11A4F8506156
:1011A000A4F8C691A4F8CA91A4F8CE91A4F8D2915B
:1011B00084F8E47184F8E57184F8E871A4F8489142
:1011C000A4F852B184F89501039084F8E3210192C8
:1011D0000291A4F8543184F8E17184F8EE71A4F816
:1011E00056B184F8F171FFF7EBF9DAF800300398A3
:1011F00027740026E773A673A681D872187355204A
:10120000019AD8700F205871DA712220212298712A
:101210005A740E2053224FF0170E1874DA763520C8
:101220000A224FF0280883F815E083F816E0987634
:101230004FF02D0E5A209A740192642283F80DE02B
:1012400018721A771E7083F8018083F80280DE75A9
:1012500083F804B09E731E76DE735E7683F8098091
:1012600083F814E04FF4FA7EA3F84EE04FF0080E36
:1012700083F850E0DFF8B0E1C3F838E0C3F83CE0B1
:10128000DFF8A8E1C3F828E04FF0780C4FF07E5E5D
:1012900083F80AC0C3F834E0DFF894C1DFF894E1C2
:1012A0009FED5B8AC3F82CC0C3F830C0C3F848E098
:1012B000F7EE087ADFF880C102999F774FF04B0E66
:1012C00083F8526083F85180C3ED087AC3ED097A40
:1012D00083ED108AC3F844C083F84CE084F8B20769
:1012E000A4F8BC174120042184F8B30784F8B4B7EC
:1012F00084F8B56784F8B96784F8BA6784F8B66784
:1013000084F8B76784F8B867A3F85860A3F85A6000
:10131000A3F8566083F85C10152183F868103D49E6
:10132000D9663D4919673D495967C3F860C083F8DC
:10133000648083F8658083F878703948FFF77EF918
:10134000DAF80030019A83F811614FF44871A3F87C
:10135000161183F8126183F8138183F8147183F8EE
:10136000186184F8D821C82284F8D9216422A4F80D
:10137000DA9184F8DC61A4F8DE2119460E2202FB22
:1013800006326FF0170082F81901032082F81A0163
:101390006FF02F0082F81B01072082F81C016FF00C
:1013A000230082F81D01052082F81E0101365A2013
:1013B00081F8200181F821016422FF20082E81F8A4
:1013C0001F2181F8220101F10E01D7D1002183F8FC
:1013D0008911C821A3F88A11142183F88C11A3F86C
:1013E00090211E214FF4967283F88D11A3F892215B
:1013F0000121282283F88E11A3F89421094B1DE0C6
:1014000050120020A4110020502B0020C8110020F1
:10141000000000009A99193FF6287C3F3D0A773F6B
:10142000C5BF0108101300208FC2F53C00006040CA
:10143000CDCCCC3E000040400000A04085ED058AA8
:1014400010359D42FAD12A480021402204F08DFC3B
:101450000023284D284C59591A1904330868C2F83A
:10146000A802382BF5D104F50A700021802204F07F
:101470007CFC05F13801702204F50A7004F06AFC66
:10148000FEF770FADAF8006000230125314604F512
:1014900090604FF4CC7284F8D83784F8D65784F82B
:1014A000D75704F057FC04F5C36031464FF4CC72B3
:1014B00004F050FC114B1B681A68C4F8BE275A6828
:1014C000C4F8C2279A68C4F8C6271A68C4F8CA279D
:1014D0005A68C4F8CE279A68C4F8D227022384F841
:1014E000D45484F86C3605B0BDEC028BBDE8F08FA7
:1014F000F814002050A0010850120020C81100204C
:101500001549D1F8883043F47003C1F88830134B83
:101510001A6842F001021A605868114A02405A6083
:101520001A6822F0847222F480321A601A6822F457
:1015300080221A605A6822F4FE025A60DA6A22F0A7
:101540000F02DA62186B074A02401A6300229A609F
:101550004FF000638B60704700ED00E00010024028
:101560000CC07FF8CCFC00FF38B5094B93F8D85776
:1015700065B9084C2068FCF7FCFF074B25601B7819
:10158000022B03D1BDE83840FEF7D9BF38BD00BFFC
:1015900050120020A02C00209C2C0020044B93F81B
:1015A000D8371BB9034B1868FAF7B8BA0020704750
:1015B00050120020A02C002038B5054604462046D5
:1015C00014F8011B21B1034B1868FAF7B3FAF6E7D8
:1015D000401B38BDA02C00200FB407B504AB064952
:1015E00053F8042B01930020F7F7E0FF03B05DF8F8
:1015F00004EB04B0704700BF67170108024B0146B7
:101600001868FAF797BA00BFA02C0020F8B5011FA0
:1016100006460023083051F8042F02F120043F2C25
:101620003AD802F108040F2C06D80232032A04D952
:10163000002B08BF012300E002238142EBD1012BE4
:1016400030680ED0022B1AD0736803F003039B009E
:1016500000F0030043EA0010B36803F003031843EB
:1016600017E000F00F0040F04000FFF7C7FFB06840
:10167000736800F00F0040EA0310C0B209E000F008
:101680003F0040F08000FFF7B9FF3079FFF7B6FF69
:10169000307ABDE8F840B1E706F10C0734463A4627
:1016A000002552F8043D03F18001FF294FEA85052A
:1016B00010D903F50041B1F5803F02D245F0010594
:1016C00008E003F50003B3F1807F34BF45F0020565
:1016D00045F00305B242E4D165F03F00C0B2FFF728
:1016E0008DFF05F00303022B207807D0032B0CD0CD
:1016F000012B13D1FFF782FF60780FE0FFF77EFF29
:101700006078FFF77BFFA07808E0FFF777FF60784D
:10171000FFF774FFA078FFF771FFE0780434FFF75C
:101720006DFFBC424FEAA505DBD1F8BD10B50446FC
:10173000C0B2FFF763FFC4F30720BDE810405DE7C8
:1017400010B504467F2C06D964F07F00C0B2FFF7C5
:1017500055FFE409F6E7E0B2BDE810404EE743006C
:1017600083EAE070ECE7084648E700BF77204821AD
:101770000122F3F767BC772058210122F3F762BCFE
:1017800007B5002101AB03227720F3F7DFFB9DF8BB
:1017900005309DF804001B0243EA00439DF8060053
:1017A000184303B05DF804FB08B5FFF7E9FF014BF0
:1017B000186008BD181B002008B5FFF7E1FF014BBA
:1017C000186008BD141B002013B5062204464321EF
:1017D00068206B46F3F7BAFBA0B19DF800209DF896
:1017E000013043EA022323809DF802209DF8033054
:1017F00043EA022363809DF804209DF8053043EA04
:101800000223A38002B010BD13B5062204463B217B
:1018100068206B46F3F79AFBA0B19DF800209DF875
:10182000013043EA022323809DF802209DF8033013
:1018300043EA022363809DF804209DF8053043EAC3
:101840000223A38002B010BD13B501220DF10703DE
:101850003A2104466820F3F779FB0520F9F7CCFF1D
:101860009DF8073003B10123237002B010BD0F4B68
:101870001A7813B51C46BAB90D4B1B68A3B11A6888
:101880001AB10C49486902434A619A88ADF80420AC
:1018900002228DF807209868002201A98DF8062001
:1018A000F3F73EFA0123237002B010BD942B002001
:1018B000F00200200010024008B5FFF7D8FF6B21AE
:1018C00080226820F3F7BEFB6420F9F7A0FF6B21AC
:1018D00003226820F3F7B6FB0F20F9F798FF104BAF
:1018E00019211A786820F3F7ADFB0F20F9F78FFF65
:1018F0000C4B1A211A786820F3F7A4FB1B2118223D
:101900006820F3F79FFB1C2110226820F3F79AFB55
:10191000682037210222BDE80840F3F793BB00BFDF
:10192000240300200000002008B5FFF7A0FF074BAC
:101930001B7813B1012B03D008BD4FF4006201E006
:101940004FF48052024B1A8008BD00BFF402002001
:10195000040000202DE9F0410369C76805460E46E2
:101960001F40002F35D0B7FA87F24FF00043D34025
:10197000DB432B611F40A2F11B03042BF1D8DFE8EE
:1019800003F0221F1C190300746A24B1013C0023D8
:10199000A4B2736201E0EC6AA4B2D6F82080B8F178
:1019A000000FDED0D8F80030404621469847D8F8DE
:1019B0000480F4E73068696B07E07068A96B04E0A5
:1019C000B068E96B01E0F068296C036889B2984758
:1019D000C7E7BDE8F08107B52320F9F718FF6820B5
:1019E000752101220DF10703F3F7B0FA28B19DF834
:1019F0000700A0F168035842584103B05DF804FBAA
:101A0000024640213C20F3F71DBB70B500EB80007F
:101A1000094CA0F1A1059C3825440444074B15F856
:101A2000010F1E787040FFF7EBFFA542F6D130465C
:101A3000BDE87040E4E700BF28A10108F02F0020B6
:101A400010B5441E14F8010F10B1FFF7DEFFF9E7DF
:101A500010BD024680213C20F3F7F4BA10B5D42023
:101A6000FFF7F7FF8020FFF7F4FFA820FFF7F1FF53
:101A70003F20FFF7EEFFD320FFF7EBFF0020FFF73B
:101A8000E8FF4020FFF7E5FF8D20FFF7E2FF14207D
:101A9000FFF7DFFFA120FFF7DCFFC820FFF7D9FF2A
:101AA000DA20FFF7D6FF1220FFF7D3FF8120FFF7E0
:101AB000D0FFCF20FFF7CDFFD920FFF7CAFFF120DD
:101AC000FFF7C7FFDB20FFF7C4FF4020FFF7C1FF90
:101AD000A420FFF7BEFFA620FFF7BBFFAF20FFF754
:101AE000B8FFA620FFF7B5FFAE20FFF7B2FF20201A
:101AF000FFF7AFFF0020FFF7ACFFB020FFF7A9FF13
:101B00004020FFF7A6FF0020FFF7A3FF1020FFF7FC
:101B1000A0FF4FF48064013C0020A4B2FFF770FFE7
:101B2000002CF8D18120FFF794FFC820FFF791FF28
:101B3000AF20FFF78EFF012010BD08B55038C0B2AE
:101B4000FFF787FF0020FFF784FF1020BDE8084063
:101B50007FE7503910B50446C8B2FFF77AFF04EBAF
:101B60004400400004EB440400F00E00FFF771FF56
:101B7000C4F3C3001030BDE810406AE701480249D1
:101B8000E8E600BF00480140682000200148024903
:101B9000E0E600BF0040014040200020014802492B
:101BA000D8E600BF00040040182000204FF080401D
:101BB0000049CFE6F01F002001480249CAE600BFF5
:101BC000002C0140C81F002001480249C2E600BFA6
:101BD000002C0140C81F0020224B10B5224C5A4354
:101BE000224BB3FBF2F203880139013AA04289B2D9
:101BF00092B29BB20ED004F50064A0420AD0B0F1BC
